:100000000C94BF140C94F0140C94F0140C94F01491
:100010000C94F0140C94F0140C94F0140C94F01450
:100020000C94F0140C94F0140C94F0140C94F01440
:100030000C94F0140C9487850C94F0140C94F01428
:100040000C94F0140C9417B60C94F0140C94F01457
:100050000C94F0140C94F0140C94C98D0C941CC5E1
:100060000C94F0140C94D9550C94F0140C94F014D6
:100070000C94F0140C94F0140C94F0140C94F014F0
:100080000C94F0140C94F0140C94F0140C94F014E0
:100090000C94F0140C94F0140C94F0140C94F014D0
:1000A0000C94F0140C94F0140C94F0140C94F014C0
:1000B0000C94F0140C94F0140C94F0140C94F014B0
:1000C0000C94F0140C94F0140C94F0140C94F014A0
:1000D0000C94F0140C94F0140C9478560C9439563B
:1000E0000C94F014B832D5320633233338336133ED
:1000F000CE333434DD34253933392C39533957393B
:100100007139D73D8639D239043A2B3A543AAA3A52
:10011000BB3ACC3ADD3AEE3AFF3AD73DE23CD73D26
:10012000ED3C5D3D633D833D35C138C127C12BC1E9
:1001300031C16FC13CC140C146C14AC14EC154C169
:1001400058C15CC16FC162C166C16AC138C43DC4D7
:1001500042C44CC456C4CFC460C468C470C47AC41A
:1001600084C48EC49DC4A7C4CFC4B1C4BBC4C5C419
:10017000084AD73B3BCE016E84BCBFFDC12F3D6C0E
:1001800074319ABD56833DDA3D00C77F11BED9E474
:10019000BB4C3E916BAAAABE000000803F05A84C54
:1001A000CDB2D44EB93836A9020C50B99186880820
:1001B0003CA6AAAA2ABE000000803F004E414E493C
:1001C0004E495459494E46CDCCCC3D0AD7233C1715
:1001D000B7D13877CC2B329595E6241FB14F0A0062
:1001E0000020410000C84200401C4620BCBE4CCA52
:1001F0001B0E5AAEC59D74434F4D4D554E4943415C
:1002000054494F4E0044525952554E004552524F98
:10021000525300494E464F004543484F0047322F46
:1002200047332062616420706172616D657465722C
:10023000730A00206F6620004D424C20473239205F
:10024000706F696E74200059206F7574206F66207E
:1002500072616E67652028312D35292E0A005820DD
:100260006F7574206F662072616E67652028312D6E
:1002700035292E0A004D6573682070726F62696EB1
:100280006720646F6E652E0A005374617274206D6E
:100290006573682070726F62696E67207769746831
:1002A0002022473239205331222066697273742E1E
:1002B0000A004732380A47323920533200537461FA
:1002C00074653A20004D65736820626564206C6532
:1002D00076656C696E6720686173206E6F2064615B
:1002E00074612E0A0053206F7574206F662072614E
:1002F0006E67652028302D35292E0A004D657368FC
:1003000020706F696E742063616E6E6F7420626519
:10031000207265736F6C7665640A00456E642066B2
:10032000696C65206C6973740A00426567696E20A8
:1003300066696C65206C6973740A00286E6F2066AC
:10034000696C6529005344207072696E74696E6728
:10035000206279746520004E6F74205344207072BF
:10036000696E74696E670A0043757272656E7420F7
:1003700066696C653A20002569730025696D202542
:100380006973002569682025696D2025697300253A
:100390006964202569682025696D20256973002519
:1003A000697920256964202569682025696D2025E3
:1003B0006973005072696E742074696D653A20002B
:1003C000180213020C020502F7016F66660044452D
:1003D0004255473A004B494C4C45442E20004D3184
:1003E00031332053006F6B002C20002C2000544828
:1003F00045524D414C5F50524F54454354494F4E26
:10040000004155544F5245504F52545F53445F532F
:10041000544154555300454D455247454E43595F4D
:1004200050415253455200434153455F4C49474860
:10043000545F4252494748544E45535300544F4726
:10044000474C455F4C494748545300534F46545717
:100450004152455F504F574552004255494C445F09
:1004600050455243454E54004C4556454C494E4725
:100470005F44415441005A5F50524F42450041553C
:10048000544F4C4556454C005052494E545F4A4FCC
:10049000420050524F4752455353004155544F521A
:1004A00045504F52545F54454D5000564F4C554D9A
:1004B000455452494300454550524F4D0053455213
:1004C00049414C5F584F4E5F584F4646004649528F
:1004D0004D574152455F4E414D453A4D61726C69F1
:1004E0006E20312E312E39202847697468756229B3
:1004F00020534F555243455F434F44455F55524C3F
:100500003A68747470733A2F2F6769746875622E35
:10051000636F6D2F4D61726C696E4669726D7761A4
:1005200072652F4D61726C696E2050524F544F436B
:100530004F4C5F56455253494F4E3A312E30204D65
:10054000414348494E455F545950453A3344205041
:1005500072696E7465722045585452554445525F15
:10056000434F554E543A3120555549443A636564DA
:1005700065326132662D343161322D343734382D95
:10058000396231322D63353563363266333637663C
:10059000660A002F2F200020540020520041636380
:1005A000656C65726174696F6E3A20500020466C0C
:1005B0006F773A20000001363726032BFFFFFF3C00
:1005C0003D382AFFFFFFFF2E303E12FFFFFFFFFFE7
:1005D000FFFF0809FF2C071A1C18FFFFFF08440A39
:1005E0002C4324221E43290A0061626C6564202882
:1005F0006D696E2074656D702000436F6C642065BA
:100600007874727564657320617265200020643AA5
:100610000020693A0020703A004E6F2063617365D4
:10062000206C696768740A00454550524F4D204F51
:100630004B0A00205A004475616C20456E64737447
:100640006F702041646A7573746D656E7420286DD7
:100650006D293A20003F4B2076616C7565206F75DF
:1006600074206F662072616E67652028302D3130EE
:10067000292E0A00416476616E6365204B3D00417E
:1006800063746976652045787472756465723A2082
:1006900000496E76616C6964206578747275646572
:1006A000720A0043616E6E6F7420656E746572200D
:1006B0007375626469723A20004739310A47312004
:1006C0005A2D302E30320A47393000537065636935
:1006D000616C204D656E753A205A20446F776E200C
:1006E000302E310A004739310A4731205A2D302E39
:1006F00030320A473930005370656369616C204DB0
:10070000656E753A205A20446F776E20302E303255
:100710000A004739310A4731205A2B302E30320A2D
:10072000473930005370656369616C204D656E75A3
:100730003A205A20557020302E30320A0047393185
:100740000A4731205A2B302E310A47393000537076
:10075000656369616C204D656E753A205A2055704D
:1007600020302E310A004732392053320053706551
:100770006369616C204D656E753A204E6578742012
:100780004D65736820506F696E740A0047323920D6
:100790005331005370656369616C204D656E753A25
:1007A000205374617274204D657368204C657665C2
:1007B0006C696E670A004D31343020533630005377
:1007C00070656369616C204D656E753A2050726585
:1007D00068656174204265640A004D35303100530C
:1007E00070656369616C204D656E753A2052656174
:1007F0006420454550524F4D0A004D35303000536E
:1008000070656369616C204D656E753A2053617641
:100810006520454550524F4D0A004D333033204539
:100820002D31205338302043382055310053706526
:100830006369616C204D656E753A204175746F2057
:1008400054756E6520486F74626564205069640A4F
:10085000004D33303320453020533233302043387D
:10086000205531005370656369616C204D656E756C
:100870003A204175746F2054756E6520486F746519
:100880006E64205049440A003C5370656369616C92
:100890005F4D656E753E003C5370656369616C5FCA
:1008A0004D656E753E002F002F002F002F2E2E0A53
:1008B000002F2E2E002F2E2E003C53706563696191
:1008C0006C5F4D656E753E0A003C537065636961EF
:1008D0006C204D656E753E003C5370656369616CBC
:1008E000204D656E753E003C526561642045455063
:1008F000524F4D3E003C5265616420454550524F79
:100900004D3E003C4175746F2054756E6520486FF4
:1009100074626564205049443E003C4175746F2008
:1009200054756E6520486F74626564205049443E7A
:10093000003C4175746F2054756E6520486F746576
:100940006E64205049443E003C4175746F205475DC
:100950006E6520486F74656E64205049443E003CCB
:10096000457869743E003C457869743E003C5361AB
:10097000766520454550524F4D3E003C53617665AB
:1009800020454550524F4D3E003C4E657874204DF9
:1009900065736820506F696E743E003C4E657874D4
:1009A000204D65736820506F696E743E003C53742F
:1009B000617274204D657368204C6576656C696E54
:1009C000673E003C5374617274204D657368204C1F
:1009D0006576656C696E673E003C5072656865615E
:1009E00074206265643E003C5072656865617420E5
:1009F0006265643E003C5A20446F776E20302E3191
:100A00003E003C5A20446F776E20302E313E003C31
:100A10005A20446F776E20302E30323E003C5A20F0
:100A2000446F776E20302E30323E003C5A20557095
:100A300020302E30323E003C5A20557020302E306F
:100A4000323E003C5A20557020302E313E003C5A38
:100A500020557020302E313E0056313136004A3359
:100A60003320004D3530300A4D3432302053310AB6
:100A70004731205A313020463234300A473120582D
:100A800030205930204636303030004A3232004A69
:100A90003232004731205A3520463234300A47314D
:100AA0002058313930205932302046363030300A23
:100AB0004731205A302046323430004731205A35F1
:100AC00020463234300A47312058313930205931EC
:100AD00039302046363030300A4731205A302046EF
:100AE000323430004731205A3520463234300A47FC
:100AF00031205831393020593230204636303030AC
:100B00000A4731205A302046323430004739310A02
:100B10004731205A313020463234300A4739300AC2
:100B20004732380A4732390A473120583230205983
:100B300032302046363030300A4731205A30204695
:100B4000323430004A3032004A3132004731205AC4
:100B50003130004F4B004731205A31300047393097
:100B60000047312045256946353030004731204562
:100B70002D302E314625690047312045302E314633
:100B80002569004731205A256946256900473120EB
:100B90005A2D302E31462569004731205A302E31EA
:100BA00046256900473120592569462569004731A6
:100BB00020592D302E314625690047312059302EDD
:100BC0003146256900473120582569462569004787
:100BD0003120582D302E31462569004731205830BC
:100BE0002E314625690047393100473238004732F7
:100BF00038205A00473238205900473238205800F0
:100C00004132305620004731205A3130004A3034CA
:100C1000004A3231004A3230004B494C4C45442E98
:100C200020004A303400454E4400464E20004A30F1
:100C300032003939393A393939004D0048004137E5
:100C4000562000413656202D2D2D004A30320041CD
:100C5000365620005A3A2000593A2000583A2000CF
:100C60004135560041345620004133562000413270
:100C7000562000413156200041305620004D383476
:100C8000004A3136004A3138004739310A473120AD
:100C90005A313020463234300A473930004A313434
:100CA000004A3030004A3031004A31300024F4D458
:100CB0003050C38E20C2A24017828B7011127A91DD
:100CC0000D816CD90AA861E108C7586607615143D4
:100CD000061E4B5D05C145A7041A411104093D9844
:100CE00003713931034036DB0265339102D430544D
:100CF00002802E1D02632CEE01752AC501B028A0CA
:100D000001102781018F2564012B244B01E022343F
:100D100001AC211F018D200D01801FFC00841EED00
:100D200000971DDF00B81CD200E61BC600201BBCCC
:100D300000641AB200B219A8000A19A0006A189932
:100D400000D117910040178B00B516840031167E34
:100D500000B31579003A157300C7146F0058146A70
:100D600000EE1366008813630025135E00C7125B54
:100D7000006C12570015125400C111510070114F30
:100D80000021114B00D61049008D10470046104439
:100D90000002104200C00F4000800F3E00420F3C96
:100DA00000060F3B00CB0E3800930E37005C0E356B
:100DB00000270E3400F30D3200C10D3100900D30CC
:100DC00000600D2E00320D2D00050D2C00D90C2BCE
:100DD00000AE0C2900850C29005C0C2700350C277F
:100DE000000E0C2600E80B2400C40B2400A00B23EB
:100DF000007D0B23005A0B2100390B2100180B201A
:100E000000F80A1F00D90A1E00BB0A1E009D0A1D19
:100E100000800A1D00630A1C00470A1B002C0A1BE5
:100E200000110A1A00F7091A00DD091900C409198E
:100E300000AB091900920917007B09180063091714
:100E4000004C09160036091600200916000A09157B
:100E500000F5081500E0081400CC081400B80814C8
:100E600000A4081400900813007D0812006B0813FA
:100E70000058081200460812003408110023081117
:100E8000001208110001081100F0071000E007101F
:100E900000D0071000C0071000B0070F00A1071016
:100EA0000091070E0083070F0074070F0065070EFF
:100EB0000057070E0049070E003B070D002E070ED6
:100EC0000020070D0013070D0006070D00F9060CA2
:100ED00000ED060D00E0060C00D4060C00C8060C60
:100EE00000BC060C00B0060C00A4060B0099060C12
:100EF000008D060B0082060B0077060B006C060BBC
:100F00000061060A0057060B004C060A0042060A5A
:100F10000038060A002E060A0024060A001A060AED
:100F2000001006090007060A00FD050900F405097E
:100F300000EB050900E2050900D9050900D0050903
:100F400000C7050900BE050900B5050800AD050884
:100F500000A50509009C050800940508008C0508FB
:100F600000840508007C050800740508006C05076E
:100F700000650508005D050700560508004E0507D9
:100F80000047050700400508003805070031050740
:100F9000002A050700230507001C050600160507A3
:100FA000000F0507000805060002050700FB040600
:100FB00000F5040700EE040600E8040600E204075A
:100FC00000DB040600D5040600CF040600C90406B1
:100FD00000C3040600BD040600B7040600B1040502
:100FE00000AC040600A6040600A00405009B04064D
:100FF0000095040500900406008A04050085040598
:1010000000800406007A04050075040500700405DC
:10101000006B04050066040500610405005C04051E
:101020000057040500520405004D0405004804055E
:1010300000430405003E0404003A0405003504059D
:1010400000300404002C04050027040400230405D8
:10105000001E0404001A0404001604050011040410
:10106000000D040400090405000404040000040445
:1010700000FC030400F8030400F4030400F003047C
:1010800000EC030400E8030400E4030400E00304AC
:1010900000DC030400D8030400D4030400D00304DC
:1010A00000CC030400C8030300C503030024F404B8
:1010B000D9201BC40C5C0E9804C4095F026507713B
:1010C00001F405F900FB04B30048048700C103697B
:1010D000005803550003034500BE023A0084023164
:1010E0000053022A002902250004022000E4011C0A
:1010F00000C8011900AF0117009801140084011302
:1011000000710110006101100051010E0043010D3A
:101110000036010B002B010B0020010B001501090B
:10112000000C01090003010800FB000800F300089F
:1011300000EB000700E4000600DE000600D8000611
:1011400000D2000600CC000500C7000500C2000563
:1011500000BD000400B9000400B5000400B10004A3
:1011600000AD000400A9000400A5000300A20003D4
:10117000009F0004009B00030098000300950002FC
:101180000093000300900003008D0002008B000319
:101190000088000200860002008400030081000233
:1011A000007F0002007D0002007B00020079000247
:1011B0000077000100760002007400020072000156
:1011C00000710002006F0002006D0001006C00025F
:1011D000006A00010069000200670001006600016A
:1011E000006500010064000200620001006100016E
:1011F00000600001005F0002005D0001005C000172
:10120000005B0001005A0001005900010058000174
:101210000057000100560001005500010054000174
:101220000053000000530001005200010051000172
:1012300000500001004F0001004E0000004E000170
:10124000004D0001004C0001004B0000004B00016C
:10125000004A000100490001004800000048000168
:101260000047000100460000004600010045000064
:10127000004500010044000100430000004300015C
:101280000042000000420001004100000041000156
:1012900000400001003F0000003F0001003E000050
:1012A000003E0001003D0000003D0001003C000048
:1012B000003C0000003C0001003B0000003B00013E
:1012C000003A0000003A0001003900000039000136
:1012D000003800000038000000380001003700002E
:1012E0000037000100360000003600000036000123
:1012F000003500000035000000350001003400001A
:10130000003400000034000100330000003300000E
:101310000033000100320000003200000032000102
:1013200000310000003100000031000100300000F9
:101330000030000000300001002F0000002F0000EE
:10134000002F0000002F0001002E0000002E0000E2
:10135000002E0001002D0000002D0000002D0000D7
:10136000002D0001002C0000002C0000002C0000CB
:10137000002C0001002B0000002B0000002B0000BF
:10138000002B0001002A0000002A0000002A0000B3
:10139000002A0001002900000029000000290000A7
:1013A000002900000029000100280000002800009A
:1013B000002800000028000000280001002700008D
:1013C0000027000000270000002700000027000180
:1013D0000026000000260000002600000026000075
:1013E0000026000100250000002500000025000067
:1013F0000025000000250000002500010024000059
:10140000002400000024000000240000002400014B
:101410000023000000230000002300000023000040
:101420000023000000230000002300010022000030
:101430000022000000220000002200000022000024
:101440000022000100210000002100000021000016
:101450000021000000210000002100000021000107
:1014600000200000002000000020000000200000FC
:1014700000200000002000000020000000200001EB
:10148000001F0000001F0000001F0000001F0000E0
:10149000001F0000001F0000001F0001001E0000D0
:1014A000001E0000001E0000001E000000232C0093
:1014B00000B8220000561800003A0F0000B80800DB
:1014C00000B1040000710200003E010000656E7171
:1014D00075657565696E672022004B494C4C454423
:1014E0002E20005072696E7465722073746F707074
:1014F00065642064756520746F206572726F727305
:101500002E2046697820746865206572726F72209B
:10151000616E6420757365204D39393920746F20F0
:10152000726573746172742E202854656D706572D3
:1015300061747572652069732072657365742E20FD
:1015400053657420697420616674657220726573D6
:1015500074617274696E67290A004E6F2043686572
:10156000636B73756D2077697468206C696E652094
:101570006E756D6265722C204C617374204C696EBF
:10158000653A20004E6F20436865636B73756D206C
:1015900077697468206C696E65206E756D6265721E
:1015A0002C204C617374204C696E653A200063688E
:1015B00065636B73756D206D69736D617463682C01
:1015C000204C617374204C696E653A20004C696E42
:1015D00065204E756D626572206973206E6F742090
:1015E0004C617374204C696E65204E756D62657236
:1015F0002B312C204C617374204C696E653A2000AD
:101600004D313130004D33310053442072656164F7
:10161000206572726F720A00446F6E652070726985
:101620006E74696E672066696C650A0020496E7683
:10163000616C69642065787472756465722000520B
:101640006573656E643A20006F6B0020746F6F20C5
:101650006C6F6E6720657874727573696F6E207039
:10166000726576656E7465640A0020636F6C642031
:10167000657874727573696F6E2070726576656EC9
:101680007465640A00627573793A207061757365D8
:101690006420666F7220696E7075740A00627573DB
:1016A000793A2070617573656420666F7220757376
:1016B00065720A00627573793A2070726F636573A0
:1016C00073696E670A004A3135004B494C4C4544FA
:1016D0002E20004B494C4C20636175736564206279
:1016E00079204B494C4C20627574746F6E2F706971
:1016F0006E0A004B494C4C45442E20004B494C4C43
:101700002063617573656420627920746F6F206D4A
:1017100075636820696E6163746976652074696DAC
:1017200065202D2063757272656E7420636F6D6D18
:10173000616E643A20004A3131005072696E7465FE
:10174000722068616C7465642E206B696C6C28294A
:101750002063616C6C6564210A000000A0C0000079
:101760000000000000005761726E696E673A204801
:101770006F6D696E672042756D702044697669737C
:101780006F72203C20310A000202040000A04000D9
:1017900000A0400000004000005C430000574300F0
:1017A000004E43FFFFFF20746F6F206C6F6E672049
:1017B000657874727573696F6E2070726576656E88
:1017C0007465640A0020636F6C64206578747275B8
:1017D00073696F6E2070726576656E7465640A0059
:1017E0000000A0C0000000000000000000005743FF
:1017F0000000574300004E43486F6D696E672066D6
:1018000061696C656400206E6F7420656E7465722A
:1018100065642E0A0046696C652064656C657465B4
:10182000643A0044656C6574696F6E206661696C2A
:1018300065642C2046696C653A200050726F7465AF
:10184000637465642050696E0A004A3036004A307D
:1018500034004A30370020573A004A3038004A30C6
:10186000390020573A00205A3A0020593A002043C4
:101870006F756E7420583A0020453A00205A3A009D
:1018800020593A00583A003A004361703A005741F3
:10189000524E494E4721204C6F77205A204A65729C
:1018A0006B206D6179206C65616420746F20756EAA
:1018B00077616E746564207061757365732E0A00BC
:1018C000454550524F4D206461746173697A6520BB
:1018D0006572726F722E0A00290A0020627974659F
:1018E000733B20637263200053657474696E677381
:1018F0002053746F726564202800290A00206279E1
:101900007465733B2063726320002073746F72658B
:10191000642073657474696E67732072657472698C
:1019200065766564202800202863616C63756C61AE
:1019300074656429210A0020213D2000454550524C
:101940004F4D20435243206D69736D61746368206D
:101950002D202873746F7265642920002053697AE2
:10196000653A2000496E6465783A2000204D617226
:101970006C696E3D563535290A0028454550524F51
:101980004D3D00454550524F4D2076657273696F4D
:101990006E206D69736D617463682000024A313591
:1019A000004A3132004A3137002020506C616E6E9F
:1019B000657242756666657242797465733A200095
:1019C0002046726565204D656D6F72793A2000433F
:1019D0006F6D70696C65643A204E6F7620323820E6
:1019E000323031380A00207C20417574686F723AB9
:1019F0002028646176696472616D69726F2C20665B
:101A00006F7220416E796375626963206933204D7E
:101A1000656761290A00323031392D31312D323874
:101A200000204C61737420557064617465643A20C1
:101A300000312E312E390A004D61726C696E002022
:101A4000536F6674776172652052657365740A001E
:101A5000205761746368646F672052657365740A08
:101A6000002042726F776E206F7574205265736527
:101A7000740A002045787465726E616C205265733B
:101A800065740A00506F77657255700A007374614F
:101A900072740A004D3234004D32332025730061D8
:101AA00075746F25692E67006572726F7220777288
:101AB0006974696E6720746F2066696C650A00201E
:101AC0005A3A0020593A0020583A00656E647374FF
:101AD0006F7073206869743A2000446F6E652073DC
:101AE0006176696E672066696C652E0A004D323931
:101AF000006F70656E206661696C65642C204669B4
:101B00006C653A200043616E6E6F74206F70656E75
:101B10002073756264697220004A3035004A32339E
:101B2000004739310A4731205A2D313020463234AE
:101B3000300A4739300053442063617264206F6B70
:101B40000A006F70656E526F6F74206661696C6514
:101B5000640A00766F6C756D652E696E6974206617
:101B600061696C65640A004572726F723A00534491
:101B700020696E6974206661696C0A006563686F2C
:101B80003A001000C90210012C014001220170012D
:101B90001801B0010E01F00104015002FA00B00278
:101BA000F0003003E600D003DC009004D2007005A2
:101BB000C800A006BE000008B400B009AA00D00BFF
:101BC000A000600E960060118C00001582002019A4
:101BD0007800C01D6E00A0226400B0275A00902C2F
:101BE000500000314600E0343C0010383200903A9A
:101BF0002800603C1E00A03D1400803E0A00203FEB
:101C000000002CFFFFFFFFFF0001010101016265E1
:101C1000640A002C2073797374656D2073746F707F
:101C200070656421204865617465725F49443A209B
:101C3000004265642068656174696E672066616949
:101C40006C65640048656174696E67206661696CE3
:101C500065640045312048656174696E672066617E
:101C6000696C65640048656174696E6720666169C6
:101C70006C65640070012C0190012701B001220104
:101C8000C0011D01F00118011002130130020E0104
:101C90006002090190020401C002FF000003FA0083
:101CA0004003F5008003F000D003EB002004E600C1
:101CB0007004E100E004DC004005D700C005D2005C
:101CC0004006CD00D006C8008007C3003008BE0023
:101CD000F008B900C009B400B00AAF00B00BAA0008
:101CE000D00CA500000EA000500F9B00C010960065
:101CF0005012910000148C00C0158700B0178200AC
:101D0000B0197D00D01B7800001E730040206E00CB
:101D100090226900F024640040275F0090295A0057
:101D2000E02B5500102E500020304B0010324600A2
:101D3000E033410090353C001037370070383200F6
:101D4000A0392D00B03A2800A03B2300603C1E00C3
:101D5000103D1900903D1400103E0F00703E0A0027
:101D6000C03E0500003F0000403FFBFF803FF6FF04
:101D7000C03FF1FF453120544845524D414C20525F
:101D8000554E415741590042454420544845524D13
:101D9000414C2052554E4157415900546865726D6F
:101DA000616C2052756E6177617900453120457212
:101DB000723A204D415854454D50004572723A20B8
:101DC0004D415854454D5020424544004D415854D2
:101DD000454D5020747269676765726564004531CE
:101DE000204572723A204D494E54454D500045727F
:101DF000723A204D494E54454D5020424544004DC5
:101E0000494E54454D502074726967676572656428
:101E1000004D383420582059205A204500202F00EA
:101E20002042403A0020403A00205A0020590058F1
:101E30000020204D61783A2000205A002059005897
:101E40000020204D696E3A20004F6E20004F6666DC
:101E500000536F667420656E6473746F70733A20FC
:101E60000020643A0020693A0020703A00496E76FA
:101E7000616C69642065787472756465720A004BE0
:101E800064200023646566696E65204445464155BB
:101E90004C545F004B69200023646566696E6520C1
:101EA00044454641554C545F004B70200023646507
:101EB00066696E652044454641554C545F00504963
:101EC00044204175746F74756E652066696E697320
:101ED000686564212050757420746865206C617396
:101EE00074204B702C204B6920616E64204B642061
:101EF000636F6E7374616E74732066726F6D2062AF
:101F0000656C6F7720696E746F20436F6E666967CA
:101F100075726174696F6E2E680A005049442041E1
:101F200075746F74756E65206661696C65642120D7
:101F300074696D656F75740A0045312054484552C7
:101F40004D414C2052554E41574159004245442085
:101F5000544845524D414C2052554E41574159002D
:101F6000546865726D616C2052756E61776179009D
:101F700045312048656174696E67206661696C65EA
:101F800064004265642068656174696E67206661FB
:101F9000696C65640048656174696E672066616993
:101FA0006C656400504944204175746F74756E65AA
:101FB000206661696C6564212054656D706572618D
:101FC0007475726520746F6F20686967680A0020F5
:101FD0004B643A2000204B693A2000204B703A2095
:101FE000000A20436C617373696320504944200ADE
:101FF000002054753A2000204B753A2000206D6176
:10200000783A2000206D696E3A200020643A200062
:1020100020626961733A2000504944204175746F11
:1020200074756E65206661696C6564212042616427
:10203000206578747275646572206E756D62657264
:102040000A00504944204175746F74756E652073A1
:10205000746172740A004F66660A00466164652006
:102060004865696768742000426564204C65766540
:102070006C696E6720004661696C656420746F202E
:10208000656E61626C6520426564204C6576656CA6
:10209000696E670A004D65736820426564204C656F
:1020A00076656C20646174613A0A004D657368203E
:1020B000706F696E742063616E6E6F74206265204C
:1020C0007265736F6C7665640A004D343231206935
:1020D0006E636F727265637420706172616D657496
:1020E00065722075736167650A0020666972737492
:1020F0000A005A0059005800486F6D652000546F5F
:102100006F206661722066726F6D207265666572FF
:10211000656E636520706F696E740A007C3C3E5E7C
:102120002B3D3F2F5B5D3B2C2A225C0054524947DC
:102130004745524544006F70656E003A20007A3280
:102140005F6D696E007A5F6D696E00795F6D696EB3
:1021500000785F6D696E005265706F7274696E67AA
:1021600020656E6473746F70207374617475730A84
:10217000000A4D6561737572656420706F696E74D5
:10218000733A0A005A206F66667365743A20004EEF
:10219000756D20582C593A20352C350A0000000066
:1021A000010000000100008000555555000000406E
:1021B0000033333300AAAA2A0049922400000020E9
:1021C00000C7711C0099991900D145170055551584
:1021D000003BB1130024491200111111000000103E
:1021E000000F0F0F00E3380E0043790D00CCCC0C2C
:1021F00000C3300C00E8A20B0064210B00AAAA0A5D
:1022000000703D0A009DD80900427B090092240914
:1022100000DCD3080088880800104208000000088D
:1022200000F0C107008787070075500700711C0781
:10223000003EEB0600A1BC0600699006006666063B
:1022400000703E06006118060017F4050074D10501
:10225000005BB00500B2900500627205005555059F
:102260000078390500B81E0500050505004EEC0490
:102270000087D40400A1BD040090A7040049920483
:1022800000C17D0400EE690400C756040044440404
:10229000005C320400082104004110040000000426
:1022A000003FF00300F8E0030026D20300C3C3039D
:1022B00000CCB503003AA803000A9B0300388E0344
:1022C00000C08103009F750300D0690300505E03C6
:1022D000001D53030034480300913D0300333303D2
:1022E0000016290300381F030097150300300C0364
:1022F00000030303000BFA020049F10200BAE802EE
:10230000005CE002002DD802002DD0020059C80266
:1023100000B0C0020031B90200DAB10200AAAA027C
:1023200000A0A30200BC9C0200FA9502005C8F0290
:1023300000DF88020082820200457C0200277602CC
:102340000027700200436A02007C640200D05E0233
:10235000003F590200C853020048617264636F6411
:1023600065642044656661756C7420536574746996
:102370006E6773204C6F616465640A00B80B0000DF
:10238000B80B00003C000000102700000000FA43DA
:102390000000FA430000C040000070420000A0426C
:1023A0000000A0420000C843E17AD24220286D6DAF
:1023B000290020204D393030204B004C696E65617A
:1023C0007220416476616E63653A0A002044002001
:1023D000490020204D333034205000204400204953
:1023E0000020204D33303120500050494420736587
:1023F0007474696E67733A0A00205A0020204D36C3
:10240000363600456E6473746F702061646A75734C
:10241000746D656E743A0A00205A0020590020201D
:10242000473239205333205800205A0020204D34A1
:1024300032302053004D65736820426564204C653E
:1024400076656C696E673A0A00205A0020590020B0
:10245000204D323036205800486F6D65206F66661B
:102460007365743A0A00204500205A002059002064
:10247000580020540020530020204D323035205188
:102480000020453C6D61785F655F6A65726B3E0058
:1024900020583C6D61785F785F6A65726B3E2059A9
:1024A0003C6D61785F795F6A65726B3E205A3C6D66
:1024B00061785F7A5F6A65726B3E00416476616E37
:1024C0006365643A20513C6D696E5F7365676D6545
:1024D0006E745F74696D655F75733E20533C6D6902
:1024E0006E5F66656564726174653E20543C6D691B
:1024F0006E5F74726176656C5F6665656472617447
:10250000653E0020540020520020204D32303420FF
:102510005000416363656C65726174696F6E202859
:10252000756E6974732F7332293A20503C7072694A
:102530006E745F616363656C3E20523C72657472B9
:102540006163745F616363656C3E20543C747261C7
:1025500076656C5F616363656C3E0A002045002010
:102560005A0020590020204D3230312058004D6152
:1025700078696D756D20416363656C65726174691E
:102580006F6E2028756E6974732F7332293A0A00B2
:10259000204500205A0020590020204D32303320A1
:1025A00058004D6178696D756D206665656472616E
:1025B0007465732028756E6974732F73293A0A0045
:1025C000204500205A0020590020204D3932205843
:1025D0000053746570732070657220756E69743A6B
:1025E0000A0020204D3230302044300A0020204D97
:1025F0003230302044002044697361626C65640AA3
:102600000046696C616D656E742073657474696EE3
:1026100067733A002020473231202020203B00FF02
:10262000FDFCFAF8F6F4F2F0EEECEAE9E7E5E3E1B6
:10263000E0DEDCDAD9D7D5D4D2D0CFCDCBCAC8C76B
:10264000C5C3C2C0BFBDBCBAB9B7B6B4B3B2B0AFF0
:10265000ADACAAA9A8A6A5A4A2A1A09E9D9C9A994A
:10266000989795949392908F8E8D8B8A8988878680
:1026700084838281807F7E7D7B7A7978777675749A
:10268000737271706F6E6D6C6B6A69686766656492
:10269000636261605F5E5D5C5B5A5958585756557E
:1026A0005453525150504F4E4D4C4B4A4A49484753
:1026B0004646454443424241403F3E3E3D3C3B3B13
:1026C0003A39383837363535343332323130302FC5
:1026D0002E2E2D2C2B2B2A29292827272625252469
:1026E000232322212120201F1E1E1D1C1C1B1B1A00
:1026F000191918181716161515141313121211118B
:10270000100F0F0E0E0D0D0C0C0B0A0A090908080C
:10271000070706060505040403030202010000453D
:1027200072726F722077726974696E6720746F209D
:10273000454550524F4D210A00000021002400273A
:10274000002A002D003000330001010000040107C1
:10275000010A0100002200250028002B002E003174
:1027600000340002010000050108010B01000020F7
:10277000002300260029002C002F00320000010059
:1027800000030106010901050505050705080808FC
:1027900008020202020A0A080804040404010101F2
:1027A00001010101010303030303030303040707FA
:1027B000070C0C0C0C0C0C0C0C0202020206060698
:1027C00006060606060B0B0B0B0B0B0B0B01021080
:1027D000202008081020401020408002010201083B
:1027E00004020101020408102040808040201008EB
:1027F0000402018004020180402010080402010844
:1028000004020101020408102040800102040810A3
:1028100020408000000A0B02090C0D0E080703047B
:1028200001000000000000000000000000000000A7
:102830000000000000000000000000000000001286
:102840001110000000000000000000000000000067
:10285000000000000000000000556E6B6E6F776E88
:1028600020636F6D6D616E643A2022000000484263
:102870000000484200008040000000005772697468
:10288000696E6720746F2066696C653A20006F700E
:10289000656E206661696C65642C2046696C653ADA
:1028A00020006F70656E206661696C65642C20463F
:1028B000696C653A200046696C652073656C6563D8
:1028C0007465640A002053697A653A200046696C91
:1028D00065206F70656E65643A20002066696C65DE
:1028E0003A2000646F696E67006672657368004E17
:1028F0006F772000454E4420535542524F5554495E
:102900004E450A002220706F7300222070617265AC
:102910006E743A2200535542524F5554494E452049
:1029200043414C4C207461726765743A22004B49F4
:102930004C4C45442E2000747279696E6720746F88
:102940002063616C6C207375622D67636F64652012
:1029500066696C6573207769746820746F6F206D89
:10296000616E79206C6576656C732E204D41582020
:102970006C6576656C2069733A00E6CF00CA112455
:102980001FBECFEFD1E2DEBFCDBF00E00CBF14E031
:10299000A0E0B2E0EAE0FBEB01E00BBF02C0079071
:1029A0000D92AC30B107D9F728E1ACE0B4E001C03A
:1029B0001D92AD33B207E1F714E1CEEBD4E100E0B4
:1029C00006C021970109802FFE010E94DDDCCD3B6E
:1029D000D10780E00807A9F70E944CCA0C9474DD67
:1029E0000C9400002F923F924F925F926F927F92D1
:1029F0008F929F92AF92BF92CF92DF92EF92FF920F
:102A00000F931F93CF93DF93CDB7DEB7C45AD1098D
:102A10000FB6F894DEBF0FBECDBF91E09093C50511
:102A2000809136188D3411F40C94D024843511F42F
:102A30000C94DE2F873411F00C942A302090341837
:102A40003090351825E02216310409F43EC66CF4A6
:102A500044E0241631040CF0F9C552E02516310487
:102A6000B4F537FE2DC00C94CC246AE2261631044E
:102A700011F40C946C2374F48CE12816310411F4D5
:102A80000C9471219DE12916310411F40C947621E6
:102A90000C94CC24ABE52A16310411F40C94F723E2
:102AA000BCE52B16310411F40C94FB23EAE52E1639
:102AB000310411F00C94CC2410921E040C942C3090
:102AC0008091350281110C9431300C942C3080911E
:102AD0003502882311F40C942C300E948D7482E509
:102AE0000E946951882309F454C10E94E9504B01A6
:102AF0005C0120E030E0A9010E949BD5882309F405
:102B000078C1C0902904D0902A04E0902B04F09062
:102B10002C04CCAEDDAEEEAEFFAEC0902D04D09056
:102B20002E04E0902F04F09030042496CCAEDDAE5D
:102B3000EEAEFFAE2497C090E005D090E105E090A6
:102B4000E205F090E3052C96CCAEDDAEEEAEFFAE26
:102B50002C97C090E405D090E505E090E605F09054
:102B6000E7052896CCAEDDAEEEAEFFAE28972C96EC
:102B70002CAD3DAD4EAD5FAD2C976CAD7DAD8EAD4A
:102B80009FAD0E949BD581110DC0A701960124968F
:102B90006CAD7DAD8EAD9FAD24970E949BD58823F3
:102BA00009F427C111E022E02216310409F010E0F7
:102BB00020E030E0A901C501B4010E949BD5881F27
:102BC0008827881F181739F0C12CD12C90E8E92EDE
:102BD0009FEBF92E06C0C12CD12C80E8E82E8FE3A4
:102BE000F82E6896CCAEDDAEEEAEFFAE68972CAD9B
:102BF0003DAD4EAD5FAD2C966CAD7DAD8EAD9FAD58
:102C00002C970E94C4D964966CAF7DAF8EAF9FAFF6
:102C1000649724962CAD3DAD4EAD5FAD24972896BC
:102C20006CAD7DAD8EAD9FAD28970E94C4D96B0170
:102C30007C0164962CAD3DAD4EAD5FAD6497CA018D
:102C4000B9010E9400D62B013C01A7019601C701E2
:102C5000B6010E9400D69B01AC01C301B2010E94E3
:102C6000C5D90E9430DC60966CAF7DAF8EAF9FAF50
:102C7000609720E030E040E05FE30E9400D62B0147
:102C80003C01A5019401C501B4010E9400D64B018D
:102C90005C01A3019201C301B2010E9400D69B0115
:102CA000AC01C501B4010E94C4D90E9430DC689611
:102CB0002CAD3DAD4EAD5FAD68970E9400D64B0187
:102CC0005C01C701B601905860962CAD3DAD4EAD8C
:102CD0005FAD60970E94A1DAA50194010E9400D621
:102CE0006B017C012C962CAD3DAD4EAD5FAD2C97AC
:102CF0006CAD7DAD8EAD9FAD0E94C5D920E030E0BA
:102D000040E05FE30E9400D69B01AC01C701B60121
:102D10000E94C5D92CAD3DAD4EAD5FAD0E94C4D96A
:102D20006B017C0128962CAD3DAD4EAD5FAD289773
:102D300024966CAD7DAD8EAD9FAD24970E94C5D914
:102D400020E030E040E05FE30E9400D62B013C0130
:102D500060962CAD3DAD4EAD5FAD609764966CADA9
:102D60007DAD8EAD9FAD64970E94A1DAA50194015F
:102D70000E9400D69B01AC01C301B2010E94C5D9DB
:102D800024962CAD3DAD4EAD5FAD24970E94C4D9C5
:102D900014C089E40E946951882329F00E94E950F7
:102DA0006B017C0103C0C12CD12C76018AE40E9406
:102DB0006951882309F10E94E9502C966CAF7DAFD0
:102DC0008EAF9FAF2C9720E030E0A901C701B6017C
:102DD0000E949BD581111FC020E030E0A9012C96F4
:102DE0006CAD7DAD8EAD9FAD2C970E949BD58111B2
:102DF00012C0E7E6FBE116C420E030E0A901C701FC
:102E0000B6010E949BD58823A1F32C961CAE1DAE63
:102E10001EAE1FAE2C97A701960150582CAF3DAFA8
:102E20004EAF5FAF2C964CAD5DAD6EAD7FAD2C97C8
:102E3000705824964CAF5DAF6EAF7FAF24972CAD2A
:102E40003DAD4EAD5FADCA01B9010E9400D64B0148
:102E50005C0124962CAD3DAD4EAD5FAD2497CA010B
:102E6000B9010E9400D69B01AC01C501B4010E94CA
:102E7000C5D90E9430DCA8966CAF7DAF8EAF9FAFF6
:102E8000A8976091290470912A0480912B04909155
:102E90002C0428966CAF7DAF8EAF9FAF2897A7010B
:102EA00096010E94C5D968966CAF7DAF8EAF9FAF7B
:102EB0006897C0902D04D0902E04E0902F04F090DD
:102EC00030046496CCAEDDAEEEAEFFAE64972C96C9
:102ED0002CAD3DAD4EAD5FAD2C97C701B6010E9444
:102EE000C5D9A4966CAF7DAF8EAF9FAFA497C090AD
:102EF000E005D090E105E090E205F090E3056C96E6
:102F0000CCAEDDAEEEAEFFAE6C9768962CAD3DADAF
:102F10004EAD5FAD6897C701B6010E94C4D96B0181
:102F20007C012091E4053091E5054091E605509142
:102F3000E705A0962CAF3DAF4EAF5FAFA097A4962C
:102F40002CAD3DAD4EAD5FADA497A0966CAD7DAD03
:102F50008EAD9FADA0970E94C4D94B015C014091FA
:102F60003104509132046091330470913404AC9672
:102F70004CAF5DAF6EAF7FAFAC979A01AB01609184
:102F8000E8057091E9058091EA059091EB050E94B2
:102F9000C4D960966CAF7DAF8EAF9FAF6097A7012D
:102FA00096016CAD7DAD8EAD9FAD0E9400D62B011C
:102FB0003C01A501940124966CAD7DAD8EAD9FAD15
:102FC00024970E9400D69B01AC01C301B2010E946C
:102FD000C5D92B013C01A50194016CAD7DAD8EAD31
:102FE0009FAD0E9400D64B015C01A701960124967B
:102FF0006CAD7DAD8EAD9FAD24970E9400D69B0138
:10300000AC01C501B4010E94C4D9A30192010E9480
:1030100038DA6B017C0120E030E0A9010E949BD5E9
:1030200087FF0AC02BED3FE049EC50E4C701B60131
:103030000E94C5D96B017C0152E02516310451F480
:103040002BED3FE049EC50E4C701B6010E94C4D922
:103050006B017C0120E030E0A901C701B6010E94AC
:103060009BD5811128C06C962CAD3DAD4EAD5FADAA
:103070006C9728966CAD7DAD8EAD9FAD28970E9464
:103080009BD5811118C0A0962CAD3DAD4EAD5FAD66
:10309000A09764966CAD7DAD8EAD9FAD64970E9498
:1030A0009BD5811108C00BEDC02E0FE0D02E09EC8E
:1030B000E02E00E4F02EA7019601A8966CAD7DAD40
:1030C0008EAD9FADA8970E9400D64B015C0120E019
:1030D00030E0A90160966CAD7DAD8EAD9FAD60977F
:1030E0000E949BD58823E9F0A5019401C501B40194
:1030F0000E9400D64B015C0160962CAD3DAD4EADFB
:103100005FAD6097CA01B9010E9400D69B01AC0176
:10311000C501B4010E94C5D90E9430DC4B015C019D
:103120000DC020E030E0A901C501B4010E94EBDB35
:1031300087FF04C0B7FAB094B7F8B0942FE632E135
:1031400043E85AE3C501B4010E949BD587FF02C042
:103150000C942C30C501B4010E943ADB0E940EDBB6
:1031600062967FAF6EAF6297672B31F461E070E0DB
:1031700062967FAF6EAF62974090350450903604F0
:1031800060903704709038046296AEADBFAD629720
:10319000BD0180E090E00E949FD54B015C019B0146
:1031A000AC01C701B6010E94A1DA28966CAF7DAFD1
:1031B0008EAF9FAF2897A501940160966CAD7DAD51
:1031C0008EAD9FAD60970E94A1DAA8966CAF7DAFDF
:1031D0008EAF9FAFA897A30192016091EC0570910B
:1031E000ED058091EE059091EF050E94C4D9A501EF
:1031F00094010E94A1DAE0966CAF7DAF8EAF9FAFD5
:10320000E09728962CAD3DAD4EAD5FAD2897CA0135
:10321000B9010E9400D620E030E040E05FE30E9468
:1032200000D69B01AC0160E070E080E89FE30E9463
:10323000C4D96C966CAF7DAF8EAF9FAF6C97AC96D8
:10324000CCACDDACEEACFFACAC97C986DA86EB86D5
:10325000FC864D865E866F86788A60910202709148
:103260000302072E000C880B990B0E94A1D5209118
:103270004B0230914C0240914D0250914E020E94FF
:1032800000D62AE037ED43E25CE30E9400D66CA74B
:103290007DA78EA79FA70E9410C59B01AC01285354
:1032A0003F4F4F4F5F4FA0962CAF3DAF4EAF5FAF3C
:1032B000A0974CAC5DAC6EAC7FAC22242394312C37
:1032C00039E12D963FAF2D9762964EAD5FAD629777
:1032D0004215530509F453C10E9404930E9410C57E
:1032E000DC01CB01A096CCACDDACEEACFFACA09782
:1032F0008C199D09AE09BF09B7FD10C00E9410C509
:103300009B01AC0128533F4F4F4F5F4FA0962CAF0E
:103310003DAF4EAF5FAFA0970E945A582D963FAD7C
:103320002D9731502D963FAF2D97332309F44BC085
:1033300024962CAD3DAD4EAD5FAD24976C966CAD33
:103340007DAD8EAD9FAD6C970E9400D66B017C0168
:103350009201A30128966CAD7DAD8EAD9FAD2897EF
:103360000E9400D6A70196010E94C5D97B018C015D
:103370009201A3016C966CAD7DAD8EAD9FAD6C9747
:103380000E9400D64B015C0124962CAD3DAD4EADA4
:103390005FAD249728966CAD7DAD8EAD9FAD28971F
:1033A0000E9400D69B01AC01C501B4010E94C4D9A2
:1033B0002B013C01C701D80124968CAF9DAFAEAF65
:1033C000BFAF249757C0B10180E090E00E949FD525
:1033D00028962CAD3DAD4EAD5FAD28970E9400D62E
:1033E0004B015C010E949EDA6B017C01C501B401B6
:1033F0000E9426DC4B015C01A70196016CAD7DADFE
:103400008EAD9FAD0E9400D62B013C012C962CADB9
:103410003DAD4EAD5FAD2C97C501B4010E9400D605
:10342000A30192010E94C5D92B013C01A501940181
:103430006CAD7DAD8EAD9FAD0E9400D64B015C01A1
:103440002C962CAD3DAD4EAD5FAD2C97C701B601AE
:103450000E9400D69B01AC01C501B4010E94C4D9F1
:1034600024966CAF7DAF8EAF9FAF249749E12D9628
:103470004FAF2D979201A30168966CAD7DAD8EADD7
:103480009FAD68970E94C5D969837A838B839C839B
:1034900024962CAD3DAD4EAD5FAD2497A4966CAD9A
:1034A0007DAD8EAD9FADA4970E94C5D96D837E83FF
:1034B0008F839887A8962CAD3DAD4EAD5FADA89794
:1034C00069857A858B859C850E94C5D969877A87AD
:1034D0008B879C87E0962CAD3DAD4EAD5FADE09700
:1034E0006D857E858F8598890E94C5D96D877E8779
:1034F0008F87988BCE0101960E943B5CE090C405BB
:103500001CAA1DAA1EAA1FAA89819A81AB81BC810F
:1035100088A399A3AAA3BBA38D819E81AF81B885FF
:103520008CA39DA3AEA3BFA389859A85AB85BC85DB
:1035300088A799A7AAA7BBA7AE01485D5F4FBE01A8
:103540006C5D7F4FCE0180960E94BDAEBE016C5C6B
:103550007F4F6B018E01045D1F4F9E01235F3F4F24
:10356000AE01485D5F4F60517109CE0180960E94A7
:10357000EE60882321F07FEF271A370AA5CEE0906E
:10358000C40518AE19AE1AAE1BAE8091E00590913D
:10359000E105A091E205B091E30588A399A3AAA350
:1035A000BBA38091E4059091E505A091E605B0915B
:1035B000E7058CA39DA3AEA3BFA38091E8059091DE
:1035C000E905A091EA05B091EB0588A799A7AAA7FC
:1035D000BBA7AE01485D5F4FBE016C5D7F4FCE0162
:1035E00080960E94BDAECE01C8966C018E01045D2E
:1035F0001F4F2CEE35E0AE01485D5F4FBE016C5DA4
:103600007F4F48970E94EE6080E1E0EEF5E0A9E28E
:10361000B4E001900D928A95E1F70C942C300E9451
:103620008551F80184918F010F5F1F4F8111F7CFF2
:10363000EDE1F2E084918F010F5F1F4F882311F4B9
:103640000C942C300E948551F801F4CF80E50E9443
:103650006951882379F080910C0490910D040097B2
:1036600049F04AE050E060E070E00E941AD46B013B
:103670007C0103C0C12CD12C760183E50E946951E5
:10368000882361F00E94E95020E030E04AE754E4EA
:103690000E9400D60E940EDB6B017C010E94127119
:1036A0000E9410C5C60ED71EE81EF91E0E9410C546
:1036B000DC01CB018C199D09AE09BF09B7FD02C021
:1036C0000C942C300E945A58F1CF809135028823F7
:1036D00011F40C942C300E948D7489E40E9469517D
:1036E000882329F00E94E9502B013C0103C0412CA2
:1036F000512C32018AE40E946951882329F00E94EA
:10370000E9504B015C0103C0812C912C540180E5F0
:103710000E946951882329F00E94E9506B017C01C5
:1037200003C0C12CD12C760181E50E946951882308
:1037300039F00E94E9506CAF7DAF8EAF9FAF04C0EF
:103740001CAE1DAE1EAE1FAE9091C405CC55DF4F12
:103750009883C45AD0406091020270910302072EF0
:10376000000C880B990B0E94A1D520914B0230913F
:103770004C0240914D0250914E020E9400D62AE028
:1037800037ED43E25CE30E9400D668AB79AB8AABCD
:103790009BAB2091290430912A0440912B04509135
:1037A0002C0424962CAF3DAF4EAF5FAF2497C301DE
:1037B000B2010E94C5D9EB966CAF7DAF8EAF9FAFC3
:1037C000EB9740902D0450902E0460902F04709041
:1037D0003004A3019201C501B4010E94C5D9EF963E
:1037E0006CAF7DAF8EAF9FAFEF972091E00530912A
:1037F000E1054091E2055091E305C701B6010E9441
:10380000C5D9C158DF4F688379838A839B83CF579B
:10381000D0402091E4053091E5054091E6055091B6
:10382000E7056CAD7DAD8EAD9FAD0E94C5D9CD577E
:10383000DF4F688379838A839B83C358D040249663
:10384000CCACDDACEEACFFAC2497C982DA82EB8263
:10385000FC824D825E826F8278860E9410C59B0139
:10386000AC0128533F4F4F4F5F4FC956DF4F28835E
:1038700039834A835B83C759D040BDEC8B2EBCECA7
:103880009B2EA92CBDE3BB2E2D961FAE2D976196C6
:103890001FAE619765961FAE6597A1961FAEA19763
:1038A0000E9404930E9410C58B019C01C956DF4FF2
:1038B000C880D980EA80FB80C759D0400C191D0907
:1038C0002E093F0937FD10C09B01AC0128533F4F23
:1038D0004F4F5F4FC956DF4F288339834A835B833D
:1038E000C759D0400E945A582D967FAD2D976196AA
:1038F0006FAD619765969FAD6597A1968FADA197C6
:10390000272F362F492F582FC501B4010E94C5D942
:103910006CAF21967FAF219729968FAF2997259677
:103920009FAF259720E030E040E85FE30E94EBDBAB
:10393000181664F41CAE21961FAE219730E8299624
:103940003FAF29974FE325964FAF25976091E0054C
:103950007091E1058091E2059091E305C957DF4F31
:10396000688379838A839B83C758D04080912904D8
:1039700090912A04A0912B04B0912C04C557DF4FDD
:1039800088839983AA83BB83CB58D04025969FAD6B
:1039900025979F932996AFAD2997AF932196BFADF9
:1039A0002197BF93ECADEF93C957DF4FA880B98043
:1039B000CA80DB80C758D040C158DF4FE880F9800B
:1039C0000A811B81CF57D040EB962CAD3DAD4EAD5B
:1039D0005FADEB97C557DF4F688179818A819B8105
:1039E000CB58D0400E947CB70F900F900F900F9053
:1039F00069966FAF69976D967FAF6D97A9968FAFF8
:103A0000A997A5969FAFA597C090E405D090E5052E
:103A1000E090E605F090E705C157DF4FC882D982F4
:103A2000EA82FB82CF58D04020912D0430912E04A1
:103A300040912F0450913004CD56DF4F28833983B5
:103A40004A835B83C359D04025963FAD25973F936A
:103A500029964FAD29974F9321965FAD21975F939C
:103A60006CAD6F93C157DF4FA880B980CA80DB80EF
:103A7000CF58D040CD57DF4FE880F9800A811B81B5
:103A8000C358D040EF962CAD3DAD4EAD5FADEF9736
:103A9000CD56DF4F688179818A819B81C359D0409F
:103AA0000E947CB70F900F900F900F90AD966FAF64
:103AB000AD97E1967FAFE197E2968FAFE297E396FD
:103AC0009FAFE39789819A81AB81BC81C556DF4F57
:103AD00088839983AA83BB83CB59D040CD80DE8075
:103AE000EF80F884C156DF4FC882D982EA82FB8218
:103AF000CF59D040E4961FAEE4972D967FAD2D9719
:103B000061966FAD619765969FAD6597A1968FADF4
:103B1000A197272F362F492F582FBCAD2196AFAD37
:103B200021972996FFAD29972596EFAD25976B2F05
:103B30007A2F8F2F9E2F0E94C4D92FE632E143E0C7
:103B40005BE30E949BD587FD3DC12D967FAD2D97F0
:103B500061966FAD619765969FAD6597A1968FADA4
:103B6000A197272F362F492F582FBCAD2196AFADE7
:103B700021972996FFAD29972596EFAD25976B2FB5
:103B80007A2F8F2F9E2F0E94C5D920E030E040E091
:103B90005FE30E9400D6662E972E882E792E9F9383
:103BA0008F937F936F93C957DF4FA880B980CA80E6
:103BB000DB80C758D040C158DF4FE880F9800A81C8
:103BC0001B81CF57D040EB962CAD3DAD4EAD5FADD8
:103BD000EB97C557DF4F688179818A819B81CB58EC
:103BE000D0400E947CB70F900F900F900F90E596F9
:103BF0006FAFE597E6967FAFE697E7968FAFE797CB
:103C0000CD55DF4F9883C35AD0407F928F929F92B9
:103C10006F92C157DF4FA880B980CA80DB80CF5830
:103C2000D040CD57DF4FE880F9800A811B81C3580F
:103C3000D040EF962CAD3DAD4EAD5FADEF97CD567C
:103C4000DF4F688179818A819B81C359D0400E946E
:103C50007CB70F900F900F900F90162F072FB82E54
:103C6000A92EAD962FADAD97E1963FADE197E296C7
:103C70004FADE297E3965FADE397C156DF4F6881A2
:103C800079818A819B81CF59D0400E94C5D920E09B
:103C900030E040E05FE30E9400D61B012C016996F2
:103CA0002FAD69976D963FAD6D97A9964FADA997CA
:103CB000A5965FADA597C556DF4F688179818A814A
:103CC0009B81CB59D0400E94C5D920E030E040E034
:103CD0005FE30E9400D69B01AC01E5966FADE597CE
:103CE000E6967FADE697E7968FADE797CD55DF4F28
:103CF0009881C35AD0400E94C4D96B017C0120E056
:103D000030E0A9010E94EBDB87FF04C0F7FAF094D2
:103D1000F7F8F094A2019101612F702F8B2D9A2D4D
:103D20000E94C4D91B012C0120E030E0A9010E94AF
:103D3000EBDB87FF04C057FA509457F85094A20168
:103D40009101C701B6010E94C5D92DEC3CEC4CECA9
:103D50005DE30E949BD51816ACF5AD961FAFAD97ED
:103D6000E1960FAFE197E296BFAEE297E396AFAE72
:103D7000E397E596DFACE5976996DFAE6997E6963F
:103D8000EFACE6976D96EFAE6D97E796FFACE797D1
:103D9000A996FFAEA997CD55DF4F2881C35AD040D1
:103DA000A5962FAFA5976CAE21969FAE2197299629
:103DB0008FAE299725967FAE259731E0E4963FAFE9
:103DC000E4979BCEE4964FADE497411158C12D96F0
:103DD0007FAD2D9761966FAD619765969FAD6597A5
:103DE000A1968FADA197272F362F492F582FBCAD05
:103DF0002196AFAD21972996FFAD29972596EFAD76
:103E000025976B2F7A2F8F2F9E2F0E94C4D96B017D
:103E10007C012DEC3CEC4CEC5DE30E94EBDB1816D6
:103E20000CF42DC1A7019601C701B6010E94C5D9A6
:103E30002D96EFAD2D976196BFAD61976596AFADAD
:103E40006597A196FFADA1972E2F3B2F4A2F5F2F8D
:103E50000E94C5D9662E972E882E792E20E030E05C
:103E600040E85FE30E94EBDB87FF09C17F928F92FE
:103E70009F926F92C957DF4FA880B980CA80DB80BC
:103E8000C758D040C158DF4FE880F9800A811B81B4
:103E9000CF57D040EB962CAD3DAD4EAD5FADEB971F
:103EA000C557DF4F688179818A819B81CB58D0408B
:103EB0000E947CB70F900F900F900F90E4966FAF19
:103EC000E497E5967FAFE597E6968FAFE697E7969E
:103ED0009FAFE7977F928F929F926F92C157DF4F6C
:103EE000A880B980CA80DB80CF58D040CD57DF4F43
:103EF000E880F9800A811B81C358D040EF962CAD31
:103F00003DAD4EAD5FADEF97CD56DF4F6881798106
:103F10008A819B81C359D0400E947CB70F900F903B
:103F20000F900F90162F072FB82EA92E262F372F60
:103F3000482F592FC156DF4F688179818A819B8133
:103F4000CF59D0400E94C5D920E030E040E05FE387
:103F50000E9400D66B017C01E4962FADE497E596B4
:103F60003FADE597E6964FADE697E7965FADE797ED
:103F7000C556DF4F688179818A819B81CB59D040BA
:103F80000E94C5D920E030E040E05FE30E9400D607
:103F90009B01AC0169966FAD69976D967FAD6D978A
:103FA000A9968FADA997A5969FADA5970E94C4D954
:103FB0001B012C0120E030E0A9010E94EBDB87FF10
:103FC00004C057FA509457F85094A7019601AD9643
:103FD0006FADAD97E1967FADE197E2968FADE29739
:103FE000E3969FADE3970E94C4D96B017C0120E06A
:103FF00030E0A9010E94EBDB87FF04C0F7FAF094E0
:10400000F7F8F094A2019101C701B6010E94C5D949
:104010002DEC3CEC4CEC5DE30E94EBDB18167CF1E4
:10402000AD961FAFAD97E1960FAFE197E296BFAEA9
:10403000E297E396AFAEE397E4965FADE4976996B7
:104040005FAF6997E5966FADE5976D966FAF6D972A
:10405000E6967FADE697A9967FAFA997E7968FADD5
:10406000E797A5968FAFA5976CAE21969FAE219747
:1040700029968FAE299725967FAE2597A8CE2D96A7
:104080007FAD2D9761966FAD619765969FAD6597F2
:10409000A1968FADA197272F362F492F582FBCAD52
:1040A0002196AFAD21972996FFAD29972596EFADC3
:1040B00025976B2F7A2F8F2F9E2F0E94C4D94B01EB
:1040C0005C0169968FAD69976D969FAD6D97A996C6
:1040D000AFADA997A596BFADA59789839A83AB830A
:1040E000BC83AD968FADAD97E1969FADE197E2961B
:1040F000AFADE297E396BFADE3978D839E83AF8329
:10410000B8877CAD21966FAD219729969FAD2997F1
:1041100025968FAD2597272F362F492F582F60E0F2
:1041200070E080E89FE30E94C4D96B017C0120917C
:1041300031043091320440913304509134040E9490
:1041400000D62B013C012091E8053091E905409112
:10415000EA055091EB05BCAD2196AFAD21972996AC
:10416000FFAD29972596EFAD25976B2F7A2F8F2FCF
:104170009E2F0E9400D69B01AC01C301B2010E9498
:10418000C5D969877A878B879C87209135043091C0
:1041900036044091370450913804C701B6010E949B
:1041A00000D66B017C012091EC053091ED0540912A
:1041B000EE055091EF05BCAD2196AFAD2197299644
:1041C000FFAD29972596EFAD25976B2F7A2F8F2F6F
:1041D0009E2F0E9400D69B01AC01C701B6010E9430
:1041E000C5D96D877E878F87988BCE0101960E94F7
:1041F0003B5C1CA61DA61EA61FA689819A81AB81C9
:10420000BC8188A399A3AAA3BBA38D819E81AF8102
:10421000B8858CA39DA3AEA3BFA389859A85AB85E2
:10422000BC8588A799A7AAA7BBA7AE01485D5F4F29
:10423000BE016C5D7F4FCE0180960E94BDAEDE0157
:104240009C966D01CC55DF4FE880C45AD0408E015A
:10425000005D1F4F9E01235F3F4FAE01485D5F4FE2
:10426000BE016C5D7F4FCE0180960E94EE60882378
:1042700069F120E030E040E85FE3BCAD2196AFADEE
:1042800021972996FFAD29972596EFAD25976B2F9E
:104290007A2F8F2F9E2F0E949BD587FF17C03CAD92
:1042A0002D963FAF2D9721964FAD219761964FAF39
:1042B000619729965FAD299765965FAF65972596BB
:1042C0006FAD2597A1966FAFA197EACA80E1E0EEA6
:1042D000F5E0A9E2B4E001900D928A95E1F70C9423
:1042E0002C3080E00E942B760C942C3083E50E94C9
:1042F0006951882321F10E94C950182F863070F02F
:10430000E5EEF2E084918F010F5F1F4F882311F4D7
:104310000C942C300E948551F801F4CF833009F4BD
:104320004AC130F4813091F1823009F43FC008C0B5
:10433000843009F49FC1853009F4ACC101C010E09C
:104340000E94DF75811103C0E5ECF2E013C080919B
:10435000FD17882319F06BE073E002C06FE073E093
:104360008DEB92E00E9461B78AE00E9485510E9425
:10437000F7AE96C184917F01BFEFEB1AFB0A882349
:1043800009F48EC10E948551F701F4CF0E94AAAFB3
:10439000109201021092000282EB92E09093FC07CF
:1043A0008093FB070E94B1510C942C308091000245
:1043B0009091010297FF0EC0E9E8F2E084918F012D
:1043C0000F5F1F4F882311F40C942C300E948551ED
:1043D000F801F4CF0097A1F48091210280931F048B
:1043E00019821A821B821C8218A219A21AA21BA26D
:1043F000BE016F5F7F4FCE0180960E947BC227C0B7
:10440000815065E00E948DDC80FF03C024E0291B01
:10441000922F25E09202F0011124E80FF11D87FD93
:10442000FA95EE0FFF1FEE0FFF1FEB54FF4E80912A
:10443000310490913204A0913304B091340480830C
:104440009183A283B38380911F0480932102809182
:10445000000290910102893191050CF067C0109221
:1044600021029C012F5F3F4F3093010220930002F5
:1044700065E00E948DDC80FF03C024E0291B922FA1
:1044800040913104509132046091330470913404AE
:1044900048A359A36AA37BA319821A821B821C8298
:1044A00044E0840290011124B9016F5B754F4B0108
:1044B000DB012D913D914D915C91B4E09B02C001D7
:1044C0001124FC01EB5AF54F5F01608171818281FB
:1044D0009381DE0111966D01E12CF12C00EA10E4CC
:1044E0000E94ABC119821A821B821C82B601CE01C6
:1044F00080960E947BC2F50180819181A281B38167
:104500008093290490932A04A0932B04B0932C0445
:10451000F40180819181A281B38180932D049093D5
:104520002E04A0932F04B0933004BCC080E090E030
:10453000A0EAB0E48093310490933204A093330452
:10454000B09334040E9417770E9412718FEF9FEF8F
:104550009093010280930002E5E7F2E084918F01DD
:104560000F5F1F4F882321F00E948551F801F6CF7D
:1045700083E992E09A83898304E610E019A308A3F3
:10458000BE016F5F7F4FCE0180960E942EC38AEBE3
:1045900092E09A83898319A308A3BE016F5F7F4FBE
:1045A000CE0180960E942EC381E00E942B7681E08E
:1045B0000E940C7677C088E50E9469518823A1F09B
:1045C0000E94B9501FEF160F1530A8F0EEE5F2E08B
:1045D00084918F010F5F1F4F882311F40C942C30AE
:1045E0000E948551F801F4CF88E50E9485510E9410
:1045F0003CCA0C942C3089E50E9469518823A1F0B3
:104600000E94B9500FEF060F0530A8F0E7E4F2E082
:1046100084918F010F5F1F4F882311F40C942C306D
:104620000E948551F801F4CF89E50E9485510E94CE
:104630003CCA0C942C308AE50E946951882399F079
:104640000E94E95025E0129FF0011124E00FF11DB6
:10465000EE0FFF1FEE0FFF1FEB54FF4E60837183C1
:104660008283938335C08AE50E9485510E943CCAAB
:104670000C942C308AE50E9469518823A1F30E9492
:10468000E9506093B1107093B2108093B31090937F
:10469000B4101EC080E00E940C760E94AAAF18C021
:1046A0001230B1F46091000270910102693171051C
:1046B00014F069E170E088E392E00E9448B769E194
:1046C00070E083E392E00E9448B78AE00E9485513F
:1046D0000E94E8710C942C3080913502882311F4EB
:1046E0000C942C3089E40E946951E82E882321F033
:1046F0000E94B950062F01C000E08AE40E9469516F
:10470000F82E882321F00E94B950162F01C010E026
:10471000EE2011F0053020F4FF2081F0153070F00C
:10472000ECEFF2E084918F010F5F1F4F882311F4AB
:104730000C942C300E948551F801F4CF0E947B51DB
:10474000EE2091F034E00302F0011124EB5AF54F12
:1047500080819181A281B3818093E0059093E105EE
:10476000A093E205B093E305FF2091F044E014022A
:10477000F0011124EF5BF54F80819181A281B3811B
:104780008093E4059093E505A093E605B093E705D3
:1047900080E50E946951882319F00E94DA5003C015
:1047A00080E50E94205186E40E9469518823D9F057
:1047B0000E94E9506B017C0120E030E0A9010E94D9
:1047C000EBDB181684F420E030E040E752E4C70148
:1047D000B6010E94A1DA60934B0270934C02809361
:1047E0004D0290934E020E94D25C0C942C30909318
:1047F0001E040C942C301FE4212E12E0312E03ED08
:10480000E02E05E0F02E69E274E07DAF6CAF8EE043
:10481000C82E84E0D82E00E010E0D1018D911D015A
:104820000E946951882309F44BC00E94E9502B0172
:104830003C01133049F0F6012081318142815381DE
:104840000E94C4D92B013C01ACADBDAD2D913D9171
:104850004D915C91C301B2010E94C4D94B015C012E
:104860002DEB37E346E855EB0E94EBDB87FD0AC0F2
:104870002DEB37E346E855E3C501B4010E949BD513
:104880001816F4F4133051F4409235045092360463
:10489000609237047092380401E012C0A5019401BF
:1048A000F70160817181828193810E94C5D9D7010E
:1048B0006D937D938D939C931397812F0E946E77B8
:1048C0001F5FB4E0EB0EF11CECADFDAD3496FDAF17
:1048D000ECAFF4E0CF0ED11C143009F09ECF0023D2
:1048E00009F4F6CEC0903504D0903604E090370439
:1048F000F090380420E030E0A901C701B6010E9421
:10490000C5D920916A1130916B1140916C11509171
:104910006D110E9400D60E94F6DB60933D0A7093F1
:104920003E0A80933F0A9093400AC0922D0AD0928B
:104930002E0AE0922F0AF092300A90910B0A809191
:104940000C0A981719F00E94B470C2CE0E9412711E
:1049500080916F00982F927081FF05C080916F0049
:104960008D7F80936F0040913D0A50913E0A609187
:104970003F0A7091400A4093311050933210609377
:10498000331070933410992309F4A2CE80916F00F4
:10499000826080936F009CCE0E9462C30C942C3086
:1049A00080913418909135188637910509F4F8C62E
:1049B0000CF0C9C08D34910509F42AC40CF055C01F
:1049C0008A31910509F430C224F58531910509F445
:1049D000E9C184F48231910509F483C584319105DC
:1049E00009F4A0C1419711F00C94DB2F0E94145CD4
:1049F0000C942C308731910509F4DEC10CF4D6C13A
:104A00008831910509F4EEC1499709F4F6C10C9477
:104A1000DB2F8F31910509F403C39CF48C31910590
:104A200009F4A8C20CF40EC28D31910511F40C9456
:104A30002C304E9711F00C94DB2F0E94AC790C9423
:104A40002C308A32910509F49DC32CF4809709F427
:104A50009BC20C94DB2F8B34910509F4C3C38C34B7
:104A6000910509F4C2C30C94DB2F8B36910509F430
:104A70000AC50CF042C08535910509F461C5FCF406
:104A80008235910509F426C584F48135910511F02C
:104A90000C94DB2F0E9444900E949FA910923A042C
:104AA0001092390400E010E0FEC48335910509F44A
:104AB00014C58435910509F414C50C94DB2F883690
:104AC000910509F4A8C37CF48C35910511F00C9480
:104AD000DB2FEFE4CE2EE2E0DE2EFEE5EF2EF1E15D
:104AE000FF2E10E046C58936910509F451C48A3677
:104AF000910509F4ACC40C94DB2F8037910509F4BF
:104B000016C484F48D36910509F481C40CF40CC4E8
:104B10008E36910509F4A4C38F36910509F4B1C30B
:104B20000C94DB2F8237910509F4A2C50CF406C45E
:104B30008337910509F4F3C08537910511F40C947E
:104B40002C300C94DB2F8E3221E0920711F40C9460
:104B5000172E0CF067C08B3C910509F4E1C68CF56B
:104B60008C38910509F456C48CF48837910509F402
:104B700067C60CF462C68937910511F00C94DB2FDF
:104B800010926806109267060C942C308E3B9105AB
:104B900009F45AC434F48B39910509F413C40C9404
:104BA000DB2F883C910509F451C6893C910511F031
:104BB0000C94DB2F7FE4E72E72E0F72E0EE311E179
:104BC00095C68C3D910509F465C79CF48D3C910513
:104BD00009F437C70CF4C0C68E3C910509F434C7FC
:104BE000833D910511F00C94DB2F0E94DCA00C9406
:104BF0002C30823E910509F4C7C734F48D3D9105F0
:104C000009F455C70C94DB2F8C3241E0940709F46A
:104C1000E5C78D32914011F00C94DB2F0E9439A032
:104C20000C942C30853F61E0960711F40C94042F0E
:104C3000DCF58A39A1E09A0709F47DC3BCF480331E
:104C4000E1E09E0711F40C946E2E14F40C946B2E7C
:104C5000833621E0920709F45EC08039914011F05B
:104C60000C94DB2F0E9412710C942C30853A41E099
:104C7000940711F40C94012F4CF4843A914011F0F4
:104C80000C94DB2F0E94D4980C942C308C3A71E059
:104C9000970709F4FCC6843F914011F00C94DB2F78
:104CA0000E9489800C942C308A39B2E09B0711F461
:104CB0000C94432FB4F4873FF1E09F0711F40C9458
:104CC0000A2F14F40C94072F883F31E0930711F456
:104CD0000C94162F8C30924011F40C943A2F0C94B3
:104CE000DB2F8B3853E0950711F40C942C303CF4F7
:104CF0008438934011F40C94702F0C94DB2F803A7D
:104D0000A3E09A0709F47FC1873E934011F40C9405
:104D1000C82F0C94DB2FE7E6FBE10C94EE2EEDECB4
:104D2000F4E0E3C4EAE2F3E084918F010F5F1F4FE8
:104D3000882321F00E948551F801F6CF1092070DCB
:104D40008AEB9AE00E941CA48BE1EAEBFAE0DE0118
:104D5000159601900D928A95E1F78091B80A90918D
:104D6000B90A9C838B8385EE92E09A83898340E025
:104D700050E0BE016F5F7F4F80E090E00E94BE89EF
:104D8000CE0101960E94F357EBE1F3E084918F018D
:104D90000F5F1F4F882311F40C942C300E94855113
:104DA000F801F4CF0E948D870C942C301092890A60
:104DB00010928A0A0C942C30E0913218F09133183A
:104DC0008081882329F0803209F410823196F8CF4F
:104DD00040E061E080913218909133180E9478C5CC
:104DE0000C942C3080918A0A882319F081E08093FA
:104DF000890A0E940D900C942C301092890A80919F
:104E00003910813011F00C942C3082E080933910ED
:104E10000E9410C560933510709336108093371040
:104E2000909338100C942C3080918A0A882311F4C6
:104E30000C942C3083E50E94695181110C9436301A
:104E40000C942C3083E40E942051882309F450C034
:104E5000E8E6F3E084918F010F5F1F4F882321F074
:104E60000E948551F801F6CF8091550C811103C045
:104E7000EBE3F3E012C0BE016F5F7F4F82E59CE081
:104E80000E94E4A28E010F5F1F4FF80181918F01F4
:104E9000882349F10E948551F8CF84918F010F5FDB
:104EA0001F4F882301F10E948551F801F6CFA0EC35
:104EB000CA2EA3E0DA2EE12CF12C20E080914B06E3
:104EC00090E00E2C02C0959587950A94E2F780FD3C
:104ED00008C2AFEFEA1AFA0AB2E0CB0ED11CE5E045
:104EE000EE16F10459F78AE00E9485510C942C309B
:104EF00080918A0A882339F08091890A882319F0E1
:104F0000E5E4F3E003C0E7E5F3E028C084918F0116
:104F10000F5F1F4F882321F00E948551F801F6CFC3
:104F20006091030D7091040D8091050D9091060D17
:104F30004AE00E94A7548FE20E9485516091FF0CC5
:104F40007091000D8091010D9091020D4AE00E9438
:104F5000A7548AE00E9485510C942C3084918F01D3
:104F60000F5F1F4F882311F40C942C300E94855141
:104F7000F801F4CF40E060E080913218909133184E
:104F80000E9478C50C942C308091890A81110E946E
:104F9000127180918A0A882311F40C942C3080E5D8
:104FA0000E946951882319F00E94DA5003C080E5FD
:104FB0000E942051182F482F61E080913218909163
:104FC00033180E9478C583E50E946951882381F0D7
:104FD0000E94B950AB01BC014093030D5093040DE6
:104FE0006093050D7093060D82E59CE00E94D5A1AB
:104FF00080918A0A882319F081E08093890A11112F
:105000000C942C30F6CE809132189091331821E018
:105010002093880A40E060E00E9478C50C942C3010
:105020000E94BE8F7B018C0120E831E541E050E019
:105030000E9489D9C9016DE671E00E949ADC4B019A
:105040005C01C801B70120E13EE040E050E00E9471
:1050500089D9CA01B90128E130E040E050E00E945E
:1050600089D9762E672EC62ED72EBCE32B2E312C57
:10507000412C512CC801B701A20191010E9489D98C
:10508000F62EE72ECA01B901A20191010E9489D929
:10509000CB018E010F5F1F4F81149104D1F0EF926D
:1050A000FF927F936F936F927F92BF92AF929F9286
:1050B0008F928FE993E09F938F931F930F930E949A
:1050C0006DD50FB6F894DEBF0FBECDBFECE7FBE1A8
:1050D00045C0A114B10489F0EF92FF927F936F93C2
:1050E0006F927F92BF92AF928FE893E09F938F93DE
:1050F0001F930F930E946DD5E4CFCD2879F0EF92E6
:10510000FF927F936F936F927F9283E893E09F93D8
:105110008F931F930F930E946DD5D3CF892B69F086
:10512000EF92FF927F936F938BE793E09F938F9320
:105130001F930F930E946DD5C4CFEF92FF9287E724
:1051400093E09F938F931F930F930E946DD50F90C1
:105150000F900F900F900F900F90B8CF84917F0118
:105160009FEFE91AF90A882321F00E948551F7017F
:10517000F5CFB80183EB93E00E9461B78AE00E940B
:1051800085516AC783E50E946951882309F464C781
:105190000E94C950E82E80E50E946951882331F0B1
:1051A0000E94C950182F87FF02C056C71DE089E42E
:1051B0000E946951882349F00E94DA508111C4C7C6
:1051C000E5EBF5E085EE95E009C089E40E94205109
:1051D000F5CF31968E179F0709F4B6C724911213A5
:1051E000F8CF87C70E940D9037C780913910813062
:1051F00009F032C782E0809339100E9410C5609395
:10520000351070933610809337109093381024C760
:105210000E942F9021C788E690E00E9412558111CC
:105220001BC780914B0683FD17C783E50E94695118
:10523000882399F00E94E9500E9409DBCB010E946B
:1052400026860E94E95020E030E044EB52E40E94C0
:105250009BD5181614F00E942F900E948BB9FCC6A3
:105260008EE40E946951882309F4F6C60E94B95061
:10527000609310187093111880931218909313185C
:10528000EBC683E50E942051882359F083E50E94F4
:105290006951882319F00E94C95001C080E08093B1
:1052A0004B06ECE7FBE184918F010F5F1F4F8111EB
:1052B00003C0EEECF3E004C00E948551F801F3CF87
:1052C00084918F010F5F1F4F882321F00E94855129
:1052D000F801F6CF80914B068111E9CDEAECF3E0BD
:1052E00018C0BB24B394B20E222319F08CE20E94A2
:1052F0008551F60185919491FC0184918F010F5F96
:105300001F4F882321F00E948551F801F6CF2B2DE5
:10531000E0CD84918F010F5F1F4F882309F4E3CD07
:105320000E948551F801F5CF1092340295C685EDA3
:1053300093E00E9415580E949B9A8EC683E50E94B6
:105340006951811103C0ECE7FBE10BC00E94C95019
:105350008D3318F4809322027FC68CE3809322025F
:105360007BC684918F010F5F1F4F882321F00E941D
:105370008551F801F6CF4091220250E060E070E0E4
:105380008EED93E00E940EB78AE00E94855164C6BC
:1053900089E690E00E941255811111C0E5EEF3E01C
:1053A00084918F010F5F1F4F882321F00E94855148
:1053B000F801F6CF0E94468D8AE00E948551109236
:1053C000C505D7C683E50E946951882309F444C600
:1053D0000E94C950182F8D3308F01CE31093D2059A
:1053E0000E9410C56B017C01212F30E0A8EEB3E0D4
:1053F0000E94B5D9C60ED71EE81EF91EC092CE0572
:10540000D092CF05E092D005F092D10525C60E943A
:10541000AE7722C680914B0683FD1EC683E50E94AF
:105420006951882309F418C60E94E9500E9409DBDB
:105430006E36710514F06EE670E070933C04609374
:105440003B040E94008E08C60E94B27205C680E529
:105450000E946951811106C083E50E946951882329
:1054600059F005C00E94C9508111F6C5F5CF0E94C0
:10547000B9506F3F710510F06FEF70E070933A0410
:1054800060933904E9C580E50E946951811105C026
:1054900010923A0410923904DFC50E94B950672B6C
:1054A00009F0DAC5F5CF62E370E080E090E00E9499
:1054B000D8C40E9404930F5F1F4F0331110599F761
:1054C00062E370E080E090E00E94D8C40E94049300
:1054D0006AD6C2C510921D04BFC581E080931D0429
:1054E000BBC583E50E946951882399F00E94E95069
:1054F00020E030E04AE754E40E9400D60E940EDB30
:1055000060932302709324028093250290932602D5
:10551000A3C588E50E9420518111B9C589E50E9483
:1055200020518111B4C58AE50E9420518111AFC577
:1055300085E40E9420518111AAC50E949FA98CC5B3
:1055400083E50E942051882309F486C50E94E95012
:1055500020E030E04AE754E40E9400D60E940EDBCF
:105560006093CA057093CB058093CC059093CD05CD
:1055700073C5D6018D916D010E942051882309F4D5
:105580006DC0133009F063C00E94E9504B015C010B
:1055900020E030E040EA51E40E949BD587FF4EC0F6
:1055A000A501940160916A1170916B1180916C1149
:1055B00090916D110E94A1DA2B013C019B01AC017D
:1055C00060911A0670911B0680911C0690911D0631
:1055D0000E9400D660931A0670931B0680931C06E7
:1055E00090931D06A301920160913A0670913B06CB
:1055F00080913C0690913D060E9400D660933A0649
:1056000070933B0680933C0690933D0660913A115F
:1056100070913B1180913C1190913D110E949FD55A
:10562000A30192010E9400D60E940EDB60933A1102
:1056300070933B1180933C1190933D1180926A11BD
:1056400090926B11A0926C11B0926D1107C00E94E4
:10565000E950F70160837183828393831F5FF4E0D5
:10566000EF0EF11C143009F084CF0E942CBBF4C45F
:105670000E94127183E50E946951882309F428C8A9
:105680000E94B9506230710509F022C80E941F5C67
:105690008BE50E9485516091B8057091B9058091A4
:1056A000BA059091BB0542E00E9468554091BC0547
:1056B0005091BD056091BE057091BF058BEE93E0E2
:1056C0000E942BB74091C0055091C1056091C20561
:1056D0007091C30588EE93E00E942BB78DE50E9480
:1056E00085518AE00E948551B7C484918F010F5F74
:1056F0001F4F882321F00E948551F801F6CF60E00A
:105700008DEB94E00E94B17161E086EB94E00E9421
:10571000B17161E08BEA94E00E94B17161E08BE9C4
:1057200094E00E94B17160E082E994E00E94B1715E
:1057300061E088E894E00E94B17160E08EE794E057
:105740000E94B17160E086E794E00E94B17161E06F
:1057500088E694E00E94B17160E08AE594E00E94DE
:10576000B17160E08BE494E00E94B17160E08DE380
:1057700094E00E94B17160E087E294E00E94B17110
:1057800060E086E194E00E94B17160E081E094E025
:105790000E94B17161E08EEE93E00E94B1715CC431
:1057A000009132181091331883E0D12C40E08150E1
:1057B000E9F0D8019C91292F2B7F2134C1F7119654
:1057C0002C912133A1F7913421F0953421F441E05B
:1057D00002C0DD24D39498012E5F3F4F89012F5FD3
:1057E0003F4FF80190819032C9F3E1CF442369F033
:1057F000ECE7FBE184917F012FEFE21AF20A8823A4
:1058000021F00E948551F701F5CFDD2069F0E3E931
:10581000F5E084917F013FEFE31AF30A882321F03A
:105820000E948551F701F5CFD8018D918D01882314
:1058300009F459CB0E948551F7CF0E9442B00CC4A5
:1058400081E0809368068093670606C488EC90E048
:105850000E941255811100C484E40E9420518823C3
:1058600009F441C00E94E9506B017C0111E020E085
:1058700030E0A9010E949BD5811101C010E0109376
:10588000191120E030E0A901C701B6010E949BD5A3
:10589000882349F10E94E950E0915C10B4E0EB9F4D
:1058A000F0011124E25EFE4E608371838283938354
:1058B00020E030E0A90160911E1170911F118091CC
:1058C0002011909121110E949BD581110CC080E084
:1058D00090E0A0EEBFE380931E1190931F11A09360
:1058E0002011B09321110E94DDA9B6C3F701819167
:1058F0007F010E942051882351F00E94E9500E94AC
:105900000EDBD8016D937D938D939C9313970C5F61
:105910001F4FB1E10E341B0749F70E94BBB99CC36E
:105920006FE4E62E62E0F62E0EE216E0F7018191BA
:105930007F010E942051882341F00E94E950D80144
:105940006D937D938D939C9313970C5F1F4FB6E0DF
:105950000E331B0759F780C383E50E9469518823E2
:10596000A1F00E94E9506093260670932706809369
:10597000280690932906609322067093230680934D
:1059800024069093250610E001C011E080E50E94F6
:105990006951882359F00E94E9506093260670935C
:1059A0002706809328069093290610E082E50E943E
:1059B0006951882359F00E94E95060932A06709338
:1059C0002B0680932C0690932D0610E084E50E9410
:1059D0006951882359F00E94E95060932206709320
:1059E0002306809324069093250636C3112309F4D9
:1059F00033C3409126065091270660912806709186
:105A000029068DE995E00E942BB740912A06509116
:105A10002B0660912C0670912D068AE995E00E9474
:105A20002BB7409122065091230660912406709175
:105A3000250687E995E00E942BB78AE00E948551F0
:105A40000BC30E94227108C34FE4C42E42E0D42E3F
:105A500059E6E52E56E0F52E10E0F60181916F0132
:105A60000E942051882359F00E94E950D7016D937C
:105A70007D938D939C931397812F0E946E771F5F68
:105A8000B4E0EB0EF11C133041F70C9468230E9434
:105A90009096E2C283E50E946951882309F4DCC232
:105AA0000E94B9507093030260930202D5C28DED3B
:105AB00090E00E9412558111CFC283E50E94695186
:105AC000811103C0ECE7FBE139C000915C1010E0EC
:105AD0000E94B950000F111FF801E35CFD4F718364
:105AE000608380915C1090E07C01EE0CFF1CEE0C5A
:105AF000FF1C8701095D1D4F880F991FFC01E35CA6
:105B0000FD4F60817181072E000C880B990B0E945C
:105B1000A1D52AE037ED43E25CE30E9400D6F7010D
:105B2000E65EFE4E20813181428153810E9400D683
:105B3000F80160837183828393838EC284918F0185
:105B40000F5F1F4F882321F00E948551F801F6CF87
:105B500085E40E94855180915C10805D0E94855192
:105B6000E0915C10F0E0EE0FFF1FE35CFD4F608101
:105B700071818DEA95E00E9448B785E20E948551C7
:105B80008AE00E94855168C280E50E9420518823E6
:105B900009F462C20E94B9506B017C0183E50E9446
:105BA0006951882321F00E94B9508B0102C00FEF88
:105BB0001FEFC8010196039708F04EC2D7FC4CC2F4
:105BC0002C2DE5EBF5E085EE95E03491231709F4F3
:105BD00090C231968E179F07C1F78EC283E50E944F
:105BE0006951882319F00E94B95002C064E071E045
:105BF00079A368A380E50E946951882339F00E9447
:105C0000B9506938F3E17F0730F402C068EE73E001
:105C10007A83698304C088E893E19A838983BE010B
:105C2000605E7F4FCE0101960E942EC315C283E5B0
:105C30000E942051182F882371F00E94E9500E9481
:105C400009DB70932C0260932B0221E0672B09F093
:105C500020E020934A0680E50E942051882359F0D5
:105C600020912B0230912C02232B11F00E94DA504C
:105C700080934A06F1C11111EFC1ECE7FBE1849179
:105C80008F010F5F1F4F882321F00E948551F8017B
:105C9000F6CF80914A06882319F063E173E002C0D1
:105CA00066E173E08AEF95E00E9461B760912B0294
:105CB00070912C0289EE95E00E9448B7E5EEF5E080
:105CC00084918F010F5F1F4F882309F4C5C10E9483
:105CD0008551F801F5CF0E94D89ABEC180E50E9497
:105CE0002051882351F00E94E95060934210709334
:105CF0004310809344109093451089E40E942051F2
:105D0000882381F00E94E9502CEA35EC47E25EE3FB
:105D10000E9400D660933E1070933F108093401015
:105D20009093411084E40E942051882381F00E94C6
:105D3000E9502CEA35EC47E25EE30E94A1DA609379
:105D40003A1070933B1080933C1090933D10ECE719
:105D5000FBE184918F010F5F1F4F882321F00E9488
:105D60008551F801F6CF4091421050914310609157
:105D700044107091451085E196E00E942BB72CEA03
:105D800035EC47E25EE360913E1070913F108091E8
:105D90004010909141100E94A1DAAB01BC0181E159
:105DA00096E00E942BB72CEA35EC47E25EE3609167
:105DB0003A1070913B1080913C1090913D100E94E0
:105DC00000D6AB01BC018DE096E00E942BB78AE0C3
:105DD0000E94855141C10E948551F80184918F0133
:105DE0000F5F1F4F8111F7CFE9E1F6E084918F013A
:105DF0000F5F1F4F882309F42FC10E948551F801BE
:105E0000F5CF0E94E99728C10E947D8025C10E949C
:105E1000E6B422C183E50E942051882321F00E942C
:105E2000DA5091E089270E9477B016C181E0809313
:105E300058060E94737A10925806882309F40CC100
:105E4000ECE7FBE184918F010F5F1F4F811103C0CD
:105E5000E8E2F6E004C00E948551F801F3CF849196
:105E60008F010F5F1F4F882309F4F6C00E948551F0
:105E7000F801F5CF8091890A882309F4EDC081E00B
:105E800080938C0AE9C08AE50E946951811103C0A0
:105E9000E6E3F6E00BC00E94E95060932611709390
:105EA00027118093281190932911D6C084918F01D6
:105EB0000F5F1F4F882321F00E948551F801F6CF14
:105EC000409126115091271160912811709129114C
:105ED00083E396E00E942BB78AE00E948551BCC004
:105EE0008BE40E946951811103C0ECE7FBE136C0ED
:105EF0008BE40E9469518823C1F00E94E9506B0134
:105F00007C0120E030E0A9010E94EBDB87FD0AC0A4
:105F100020E030E040E251E4C701B6010E949BD589
:105F2000181634F4E5E5F6E00EC0C12CD12C76014C
:105F30000E941271C0921E06D0921F06E0922006A7
:105F4000F092210689C084918F010F5F1F4F882333
:105F500009F482C00E948551F801F5CF84918F0128
:105F60000F5F1F4F882321F00E948551F801F6CF63
:105F700040911E0650911F066091200670912106E7
:105F800084E796E00E942BB78AE00E94855164C0A6
:105F900081E08093350283E50E946951882339F0BE
:105FA0000E94DA50811158C00E94C76055C083E535
:105FB0000E942051F7CF0E9462C34EC0F090341867
:105FC0000E9412711091FD1780E00E940C76FF2054
:105FD00029F1ECE7FBE184918F010F5F1F4F8823CC
:105FE00021F00E948551F801F6CF84E50E94855189
:105FF0006F2D70E080E090E04AE00E94A75480E2BC
:106000000E948551E1E9F6E084918F010F5F1F4FF7
:10601000882311F10E948551F801F6CF1092C40532
:10602000812F0E940C76ECE7FBE184918F010F5FDA
:106030001F4F882321F00E948551F801F6CF60910F
:10604000C40570E08FE796E00E9448B78AE00E949E
:10605000855102C00E9462C31092C5050E94AA60C9
:1060600088C00E948D740E94D25CF6CF0E94B95005
:10607000AB01BC014093030D5093040D6093050DDB
:106080007093060D82E59CE00E94D5A1E5CF0E94A9
:10609000127188E50E942051882331F05F9A809127
:1060A00028048E7F8093280489E50E94205188234C
:1060B00039F08A9A479A809128048D7F809328042A
:1060C0008AE50E942051882361F080910801809523
:1060D000817080930601479A809128048B7F80937A
:1060E000280485E40E942051882309F4B5CF129A30
:1060F000B3CF0E9421CAB0CF0E941271BC2C60E0C5
:106100008C2D0E94D5C30F3F2FEF120759F48C2D11
:106110000E947FC331E020E0892B09F030E0032F9B
:10612000122F05C00130110561F401E010E08B2D44
:106130000E947FC38017910709F48ECF0E945A589E
:10614000F6CF00E010E0F3CF61E0812F0E94D5C3CD
:106150006E2D812F0E94A7C3F12CB701812F0E94C1
:1061600011C4193009F078CFF0923A04E092390462
:1061700073CFCC55DF4F0FB6F894DEBF0FBECDBF47
:10618000DF91CF911F910F91FF90EF90DF90CF9013
:10619000BF90AF909F908F907F906F905F904F9047
:1061A0003F902F9008952F923F924F925F926F925F
:1061B0007F928F929F92AF92BF92CF92DF92EF9297
:1061C000FF920F931F93CF93DF93CDB7DEB76F97F7
:1061D0000FB6F894DEBF0FBECDBFC0904304D09081
:1061E0004404E0904504F090460420E030E040EAAA
:1061F00050E4C701B6010E949BD587FD19C120E07C
:1062000030E041E953E4C701B6010E94EBDB181608
:106210000CF40EC11092A60E1092A50E80910901E9
:106220004091A40E042E000C550B817021E08227B2
:1062300090E04817590709F433C080910901817033
:1062400028272093A40E81111BC00E948D87E1EAAC
:10625000FCE084918F01882351F0082E000C990BEB
:106260000E9488870F5F1F4FF8018491F4CF8DE063
:1062700090E00E9488878AE090E00E94888710C0A2
:10628000E5EAFCE084918F01882389F3082E000C55
:10629000990B0E9488870F5F1F4FF8018491F4CFFC
:1062A0008091970E833009F44CC02CF4882351F070
:1062B0008130D9F072C0843009F43EC0853009F4D1
:1062C0004DC06BC08091890A882309F466C081E0C3
:1062D0008093970E0E9410C560939B0E70939C0E46
:1062E00080939D0E90939E0E58C08091890A8111D3
:1062F00054C08091550C882321F082E08093970E42
:106300004CC01092970EEDE9FCE084918F01882338
:1063100051F0082E000C990B0E9488870F5F1F4FC9
:10632000F8018491F4CF8DE090E00E9488878AE0A4
:1063300090E00E94888731C08091E40E8823E9F2C2
:106340002CC08091890A811128C080910B0A9091FC
:106350000C0A891B8F7009F496C01FC08091890AAE
:1063600081111BC080910B0A90910C0A891B8F70C0
:1063700009F4ABC012C08DE090E00E9488878AE0EB
:1063800090E00E9488871092970E8DE79CE0909392
:10639000FC078093FB070E94B15180918C0E909175
:1063A0008D0E03974CF571EB272E78E0372EE0E643
:1063B0008E2EEAEE9E2EA12CB12C82EF9FE00E9441
:1063C000924C18161906C4F480918C0E90918D0E83
:1063D000049794F482EF9FE00E94564C8093920EB3
:1063E000E091930EF091940E8A3019F08D3009F0FF
:1063F0007DC0309709F083C080918C0E90918D0EF6
:10640000009711F40C945F40019790938D0E809348
:106410008C0E80918E0E90918F0E019664E070E04C
:106420000E94AEDC90938F0E80938E0E0C945F4092
:106430008091A50E9091A60E8136FAEE9F07E8F0A6
:106440001092A60E1092A50EE9EAFCE084918F014D
:10645000882351F0082E000C990B0E9488870F5F4B
:106460001F4FF8018491F4CF8DE090E00E9488875F
:106470008AE090E00E948887D1CE01969093A60E84
:106480008093A50ECBCE89E89CE09093FC07809387
:10649000FB070E94B1518091E40E882311F082E045
:1064A00001C084E08093970EE5E8FCE084918F01C1
:1064B000882309F438CF082E000C990B0E94888796
:1064C0000F5F1F4FF8018491F3CFE1E8FCE0849166
:1064D0008F01882309F44FCF082E000C990B0E94DE
:1064E00088870F5F1F4FF8018491F3CF8A3309F437
:1064F00080CFEF35F10514F40C94F33D7ACF809101
:10650000900E9091910E20E6289F7001299FF00C2B
:1065100011248701045F124FE00FF11F108261E424
:1065200070E0C8010E9431DD009711F40C94D73D52
:106530009093960E8093950E801B910B8E0D9F1D50
:1065400060E070E0835F924F0E949CD10E9409DB63
:10655000CB01770FAA0BBB0B8232910510F00C9484
:10656000D73DFC018827EE58FF4F8F4F0C94DDDCA0
:10657000E8E7FCE084918F01882351F0082E000C9D
:10658000990B0E9488870F5F1F4FF8018491F4CF09
:1065900020E030E040E05FE3609143047091440408
:1065A00080914504909146041EC0E3E7FCE084918D
:1065B0008F01882351F0082E000C990B0E948887C8
:1065C0000F5F1F4FF8018491F4CF609141047091E7
:1065D0004204072E000C880B990B0E94A1D520E0E5
:1065E00030E040E05FE30E94C5D90E9409DBCB01A7
:1065F0000E9403560E94B0C78DE090E00E948887F9
:106600008AE090E00E9488870C94D73DEEE6FCE09B
:1066100084918F01882351F0082E000C990B0E9461
:1066200088870F5F1F4FF8018491F4CF20E030E09E
:1066300040E05FE360913D0470913E0480913F042F
:1066400090914004D0CFE9E6FCE084918F0188234B
:1066500051F0082E000C990B0E9488870F5F1F4F86
:10666000F8018491F4CF60913B0470913C04B1CF68
:106670002091390430913A0444E6429FC001439F7F
:10668000900D11246FEF70E00E94AEDC8B01653637
:10669000710510F004E610E0E4E6FCE084917F016F
:1066A000882359F0082E000C990B0E948887FFEF71
:1066B000EF1AFF0AF7018491F3CFB80180E090E070
:1066C00041C7E0E6FCE084918F01882351F0082E59
:1066D000000C990B0E9488870F5F1F4FF80184916F
:1066E000F4CF80E290E00E948887ECE5FCE08491A2
:1066F0008F01882351F0082E000C990B0E94888787
:106700000F5F1F4FF8018491F4CF609129047091BD
:106710002A0480912B0490912C040E94B1C780E23E
:1067200090E00E948887E8E5FCE084918F0188234F
:1067300051F0082E000C990B0E9488870F5F1F4FA5
:10674000F8018491F4CF60912D0470912E04809112
:106750002F04909130040E94B1C780E290E00E9423
:106760008887E4E5FCE084918F01882351F0082EAE
:10677000000C990B0E9488870F5F1F4FF8018491CE
:10678000F4CF609131047091320480913304909180
:1067900034040E94B1C780E290E0A0C58091890ACC
:1067A000882309F450C0EFE4FCE084918F01882332
:1067B00051F0082E000C990B0E9488870F5F1F4F25
:1067C000F8018491F4CF80918A0A882359F180914D
:1067D000550C882329F18091FF0C9091000DA09118
:1067E000010DB091020D0097A105B105C1F0BC01EA
:1067F000CD016D597F4F8F4F9F4F24E630E040E031
:1068000050E00E9489D96091030D7091040D809130
:10681000050D9091060D0E9489D9822F01C080E05C
:1068200090E0E6CEEBE4FCE084918F01882309F44C
:10683000E3CE082E000C990B0E9488870F5F1F4F34
:10684000F8018491F3CFE3E4FCE084918F01882385
:1068500009F4D2CE082E000C990B0E9488870F5F96
:106860001F4FF8018491F3CFEEE3FCE084918F0198
:10687000882351F0082E000C990B0E9488870F5F27
:106880001F4FF8018491F4CF80919B0E90919C0E44
:10689000A0919D0EB0919E0E892B8A2B8B2B09F413
:1068A00077C00E9410C5A50194010E9489D9690191
:1068B0007A0160919B0E70919C0E80919D0E90913B
:1068C0009E0EA50194010E9489D98601021B130B1B
:1068D000C8016CE370E00E949ADCCB019927EAE0E2
:1068E000F0E0BF010E94AEDC282FCB01BF010E9467
:1068F000AEDC805D80932004205D20932104109203
:10690000220480E294E00E94B0C780E290E00E94FE
:106910008887ECE3FCE084917F01882359F0082EFE
:10692000000C990B0E948887FFEFEF1AFF0AF7010E
:106930008491F3CF80E290E00E948887C8016CE3E5
:1069400070E00E949ADC6AE070E00E94AEDC605D5C
:1069500060932004805D809321041092220480E2E1
:1069600094E00E94B0C780E290E00E948887EAE34A
:10697000FCE084918F01882309F43ECE082E000CA0
:10698000990B0E9488870F5F1F4FF8018491F3CF06
:1069900080E290E00E948887E2E3FCE084918F012E
:1069A000882309F429CE082E000C990B0E948887B1
:1069B0000F5F1F4FF8018491F3CF1092C50E8091A5
:1069C000090180FF11C0EEE2FCE084918F01882371
:1069D00009F412CE082E000C990B0E9488870F5FD5
:1069E0001F4FF8018491F3CF83E50E944CC78823A1
:1069F00041F00E9467C70E940EDB70939A0E60936D
:106A0000990EEAE2FCE084918F01882351F0082E70
:106A1000000C990B0E9488870F5F1F4FF80184912B
:106A2000F4CF8DE090E00E9488878AE090E00E9499
:106A300088878091E30E882309F442C28091990EE1
:106A400090919A0E8430910509F4C8C08830910560
:106A500009F47DC1892B09F0E7C3EEE4FAE08491E3
:106A60008F01882351F0082E000C990B0E94888713
:106A70000F5F1F4FF8018491F4CF8DE090E00E94EA
:106A800088878AE090E00E948887E3E4FAE08491B6
:106A90008F01882351F0082E000C990B0E948887E3
:106AA0000F5F1F4FF8018491F4CF8DE090E00E94BA
:106AB00088878AE090E00E948887E7E3FAE0849183
:106AC0008F01882351F0082E000C990B0E948887B3
:106AD0000F5F1F4FF8018491F4CF8DE090E00E948A
:106AE00088878AE090E00E948887EBE2FAE0849150
:106AF0008F01882351F0082E000C990B0E94888783
:106B00000F5F1F4FF8018491F4CF8DE090E00E9459
:106B100088878AE090E00E948887EDE1FAE084911E
:106B20008F01882351F0082E000C990B0E94888752
:106B30000F5F1F4FF8018491F4CF8DE090E00E9429
:106B400088878AE090E00E948887EFE0FAE08491ED
:106B50008F01882351F0082E000C990B0E94888722
:106B60000F5F1F4FF8018491F4CF8DE090E00E94F9
:106B700088878AE090E00E948887E2E0FAE08491CA
:106B80008F01882351F0082E000C990B0E948887F2
:106B90000F5F1F4FF8018491F4CF8DE090E00E94C9
:106BA00088878AE090E00E948887E5EFF9E0849189
:106BB0008F01882351F0082E000C990B0E948887C2
:106BC0000F5F1F4FF8018491F4CF8DE090E00E9499
:106BD00088878AE090E00E94888726C3E7EEF9E084
:106BE00084918F01882351F0082E000C990B0E948C
:106BF00088870F5F1F4FF8018491F4CF8DE090E0FC
:106C00000E9488878AE090E00E948887E9EDF9E099
:106C100084918F01882351F0082E000C990B0E945B
:106C200088870F5F1F4FF8018491F4CF8DE090E0CB
:106C30000E9488878AE090E00E948887E3ECF9E070
:106C400084918F01882351F0082E000C990B0E942B
:106C500088870F5F1F4FF8018491F4CF8DE090E09B
:106C60000E9488878AE090E00E948887EDEAF9E038
:106C700084918F01882351F0082E000C990B0E94FB
:106C800088870F5F1F4FF8018491F4CF8DE090E06B
:106C90000E9488878AE090E00E948887EBE9F9E00B
:106CA00084918F01882351F0082E000C990B0E94CB
:106CB00088870F5F1F4FF8018491F4CF8DE090E03B
:106CC0000E9488878AE090E00E948887E9E8F9E0DE
:106CD00084918F01882351F0082E000C990B0E949B
:106CE00088870F5F1F4FF8018491F4CF8DE090E00B
:106CF0000E9488878AE090E00E948887EBE7F9E0AD
:106D000084918F01882351F0082E000C990B0E946A
:106D100088870F5F1F4FF8018491F4CF8DE090E0DA
:106D20000E9488878AE090E00E948887EDE6F9E07B
:106D300084918F01882309F448CF082E000C990B09
:106D40000E9488870F5F1F4FF8018491F3CFE6E61A
:106D5000F9E084918F01882351F0082E000C990BE3
:106D60000E9488870F5F1F4FF8018491F4CF8DE058
:106D700090E00E9488878AE090E00E948887EFE593
:106D8000F9E084918F01882351F0082E000C990BB3
:106D90000E9488870F5F1F4FF8018491F4CF8DE028
:106DA00090E00E9488878AE090E00E948887E8E46B
:106DB000F9E084918F01882351F0082E000C990B83
:106DC0000E9488870F5F1F4FF8018491F4CF8DE0F8
:106DD00090E00E9488878AE090E00E948887E1E343
:106DE000F9E084918F01882351F0082E000C990B53
:106DF0000E9488870F5F1F4FF8018491F4CF8DE0C8
:106E000090E00E9488878AE090E00E948887EAE10B
:106E1000F9E084918F01882351F0082E000C990B22
:106E20000E9488870F5F1F4FF8018491F4CF8DE097
:106E300090E00E9488878AE090E00E948887E3E0E3
:106E4000F9E084918F01882351F0082E000C990BF2
:106E50000E9488870F5F1F4FF8018491F4CF8DE067
:106E600090E00E9488878AE090E00E948887E5EFA2
:106E7000F8E084918F01882351F0082E000C990BC3
:106E80000E9488870F5F1F4FF8018491F4CF8DE037
:106E900090E00E9488878AE090E00E948887E7EE71
:106EA000F8E084918F01882309F48FCE082E000C1E
:106EB000990B0E9488870F5F1F4FF8018491F3CFD1
:106EC00080918A0A882309F486C181E08093070DA6
:106ED0001092090D1092080D89ED9AE00E941CA4F1
:106EE0008BE1E9EDFAE0DE01159601900D928A95AD
:106EF000E1F78091D70A9091D80A9C838B8385EE25
:106F000092E09A83898340E050E0BE016F5F7F4F3B
:106F100080E090E00E94BE89CE0101960E94F35766
:106F2000C090080DD090090D0091990E10919A0E05
:106F3000C601801B910B049720F06801F3E0CF0E8F
:106F4000D11C58ED452E58E0552E69EC662E68E0B0
:106F5000762EC016D10608F467C10115110509F097
:106F6000A1C06DE87AE089ED9AE00E94E4A26AE1AE
:106F700073E08DE89AE00E943CDD892B09F04AC05D
:106F8000F201849148EDE42E48E0F42E882359F074
:106F9000082E000C990B0E948887FFEFEF1AFF0A5A
:106FA000F7018491F3CF8DE090E00E9488878AE01A
:106FB00090E00E948887F301849139ECE32E38E059
:106FC000F32E882359F0082E000C990B0E94888715
:106FD000FFEFEF1AFF0AF7018491F3CF8DE090E005
:106FE0000E9488878AE090E00E9488874AE060E0FB
:106FF00070E0CB010E94A754E9EBF8E084917F0197
:107000002FEFE21AF20A882309F4E2C00E948551A8
:10701000F701F4CFE5EBF8E084917F01882359F084
:10702000082E000C990B0E948887FFEFEF1AFF0AC9
:10703000F7018491F3CF8DE090E00E9488878AE089
:1070400090E00E948887F101849121EBE22E28E0F4
:10705000F22E882359F0082E000C990B0E94888785
:10706000FFEFEF1AFF0AF7018491F3CF8DE090E074
:107070000E9488878AE090E00E9488874AE060E06A
:1070800070E0CB010E94A754ECEAF8E084917F0104
:107090002FEFE21AF20A882309F49AC00E94855160
:1070A000F701F4CF60E070E0C80101970E94848B83
:1070B00080918B0A882309F45FC0EAEAF8E08491A2
:1070C0007F01882359F0082E000C990B0E948887B5
:1070D000FFEFEF1AFF0AF7018491F3CF8DE89AE0F2
:1070E0000E94B0C78DE090E00E9488878AE090E01F
:1070F0000E948887E8EAF8E084917F01882359F0AC
:10710000082E000C990B0E948887FFEFEF1AFF0AE8
:10711000F7018491F3CF8AE99AE00E94B0C78DE02D
:1071200090E00E9488878AE090E00E948887C801EA
:10713000A0E0B0E04AE0BC01CD010E94A754E6EA1D
:10714000F8E084917F012FEFE21AF20A882321F000
:107150000E948551F701F5CF9AE9E92E9AE0F92EC0
:10716000F70181917F01882319F00E948551F8CFA2
:107170008AE00E9485512CC08DE89AE00E94B0C739
:107180008DE090E00E9488878AE090E00E948887E6
:107190008AE99AE00E94B0C78DE090E00E9488875B
:1071A0008AE090E00E948887C801A0E0B0E04AE051
:1071B000BC01CD010E94A7548AE9E82E8AE0F82E8E
:1071C000F70181917F01882399F20E948551F8CFC0
:1071D0000F5F1F4FBECEE7E9F8E084918F0188234F
:1071E00051F0082E000C990B0E9488870F5F1F4FEB
:1071F000F8018491F4CF8DE090E00E9488878AE0C6
:1072000090E00E948887E8E8F8E084918F01882365
:1072100009F4DBCC082E000C990B0E9488870F5FC5
:107220001F4FF8018491F3CFE6E2FCE084918F01D7
:10723000882309F4E1C9082E000C990B0E94888765
:107240000F5F1F4FF8018491F3CF8091890A882343
:1072500039F00E94F088ABC48091890A8823E9F054
:107260000E9495C1A4C48091970E823019F0833694
:1072700009F09DC40E94CF88E2E2FCE084918F0176
:10728000882309F4B9C9082E000C990B0E9488873D
:107290000F5F1F4FF8018491F3CF8091970E8336D3
:1072A00009F085C4DDCF89E19CE00E9415588091EA
:1072B0000B0A90910C0A891B8F7009F078C4809199
:1072C000970E823009F473C4833609F0A4C46FC4E6
:1072D0008DE090E00E9488878AE090E00E94888795
:1072E0008BC980910B0A90910C0A891B8F7009F051
:1072F0005EC48091970E823009F459C4833609F434
:1073000056C48091550C8111DAC451C483E50E94A2
:107310004CC7811126C083E40E944CC7882309F41E
:1073200046C480910B0A90910C0A891B8F7009F05A
:107330003EC420E030E040E251E4609131047091BD
:10734000320480913304909134040E949BD587FFCE
:1073500008C086E09CE09093FC078093FB070E94A6
:10736000B1510E9467C720E030E0A9010E949BD57F
:1073700087FD10C00E9467C720E030E849E853E469
:107380000E94EBDB18164CF00E9467C70E940EDBD0
:10739000CB0105C080E090E002C083E191E00E9453
:1073A000268605C483E50E944CC7882309F4FFC3E1
:1073B0000E9467C720E030E0A9010E949BD587FDAD
:1073C00011C00E9467C720E030E046E153E40E940C
:1073D000EBDB18164CF00E9467C70E940EDB362FBD
:1073E000272F04C030E001C036E920E0832F922F20
:1073F0008E36910514F08EE690E090933C048093D5
:107400003B040E94008ED3C383E50E944CC78823AF
:10741000D9F00E9467C720E030E04FE753E40E94B4
:1074200000D620E030E048EC52E40E94A1DA0E944D
:107430000EDB6F3F710519F010F06FEF70E0709385
:107440003A0460933904D8C88FEF90E090933A04DF
:1074500080933904D1C880910B0A90910C0A891B42
:107460008F7009F0C9C88091890A8111C5C80E942E
:107470009B9A5F9A809128048E7F809328048A9A31
:10748000479A809128048D7F809328048091080179
:107490008095817080930601479A809128048B7FA4
:1074A00080932804129AA8C883E50E944CC78823B9
:1074B00019F10E9467C720E030E040E252E40E94E8
:1074C0009BD587FD0FC00E9467C720E030EC49E7DD
:1074D00054E40E94EBDB181644F00E9467C70E9438
:1074E00009DB05C068E270E002C067EE73E07093EC
:1074F0000302609302025BC3E0E0FCE084918F0131
:10750000882351F0082E000C990B0E9488870F5F8A
:107510001F4FF8018491F4CFC0900202D090030273
:107520000D2C000CEE08FF08F7FE0EC06DE282EF96
:107530009FE00E94094C66277727CB016C197D09D3
:107540008E099F094AE003C04AE0C701B6010E94C4
:1075500070C752C880910B0A90910C0A891B8F70DA
:1075600009F025C38091970E823009F420C3833639
:1075700009F0EBC21CC380910B0A90910C0A891B85
:107580008F7009F039C88091970E823009F434C8A1
:10759000833609F0B6C330C880910B0A90910C0A6B
:1075A000891B8F7009F003C38091970E823009F414
:1075B000FEC2833609F0FBC4FAC280910B0A909197
:1075C0000C0A891B8F7009F0F2C28091970E8230ED
:1075D00009F4EDC2833609F020C5E9C280910B0A97
:1075E00090910C0A891B8F7009F0E1C28091970E6F
:1075F000823009F4DCC2833609F045C5D8C28091D7
:10760000C50E811103C00E948D87C4C18E3271F5F1
:107610008091C60E8E3209F046C180912A0C8823D3
:1076200009F4B8C1815080932A0C882361F090E05E
:1076300001974FE1489F9001499F300D1124C901E6
:107640008C50954F02C086EB9AE02BE1FC013496FA
:10765000A9EDBAE001900D922A95E1F7FC01828133
:1076600093819093D80A8093D70A94C18C3309F000
:107670001AC16CE173E085EC9EE00E943CDD892B31
:1076800021F481E08093E30E85C16BE273E085EC29
:107690009EE00E943CDD892B79F4E4E6F8E08491D9
:1076A0008F010F5F1F4F882321F00E948551F80141
:1076B000F6CF81E598E0E4C062E473E085EC9EE0FB
:1076C0000E943CDD892B79F4EDE2F8E084918F0192
:1076D0000F5F1F4F882321F00E948551F801F6CFDC
:1076E0008AE198E0CDC069E573E085EC9EE00E94F8
:1076F0003CDD892B79F4EFEFF7E084918F010F5F88
:107700001F4F882321F00E948551F801F6CF8AEFA0
:1077100097E0B6C067E673E085EC9EE00E943CDD32
:10772000892B79F4EFEDF7E084918F010F5F1F4F04
:10773000882321F00E948551F801F6CF8AED97E069
:107740009FC065E773E085EC9EE00E943CDD892BDD
:1077500079F4EFEBF7E084918F010F5F1F4F8823DF
:1077600021F00E948551F801F6CF86EB97E088C0A2
:1077700063E873E085EC9EE00E943CDD892B71F4A8
:1077800003E917E0F8018491882329F00F5F1F4F68
:107790000E948551F7CF8CE897E072C069E973E0E9
:1077A00085EC9EE00E943CDD892B79F4EDE6F7E064
:1077B00084918F010F5F1F4F882321F00E94855114
:1077C000F801F6CF86E697E05BC06BEA73E085ECE4
:1077D0009EE00E943CDD892B79F4EEE4F7E0849191
:1077E0008F010F5F1F4F882321F00E948551F80100
:1077F000F6CF8DE397E044C066EB73E085EC9EE046
:107800000E943CDD892B79F4E4E2F7E084918F015A
:107810000F5F1F4F882321F00E948551F801F6CF9A
:1078200082E197E02DC062EC73E085EC9EE00E945F
:107830003CDD892B79F4E7EFF6E084918F010F5F4F
:107840001F4F882321F00E948551F801F6CF85EE65
:1078500096E016C060ED73E085EC9EE00E943CDD92
:10786000892BA9F4EBECF6E084918F010F5F1F4F99
:10787000882321F00E948551F801F6CF89EB96E02C
:107880009093FC078093FB070E94B15183C06DED7C
:1078900073E085EC9EE00E943CDD892B09F07AC004
:1078A0001092E30E77C01D8218861C821B8285EE23
:1078B00092E09A8389838091DC0A811103C066EB90
:1078C0007AE002C065ED7AE06115710519F06C5F30
:1078D0007F4F02C060E070E021E045EC5EE0CE0149
:1078E00005960E9452A8882361F18BE1FE0135962E
:1078F000A9EDBAE001900D928A95E1F72B813C81C8
:107900003093D80A2093D70A80912A0C8A3008F045
:107910003DC091E0980F90932A0CFFE18F9FC0012A
:107920001124DC01A850B54F4BE1E9EDFAE00190DC
:107930000D924A95E1F7FC01EC50F54F3383228319
:1079400025C0ECE7FBE184918F010F5F1F4F882377
:1079500021F00E948551F801F6CFE3EAF6E0849128
:107960008F010F5F1F4F882321F00E948551F8017E
:10797000F6CF05EC1EE0F80181918F01882319F004
:107980000E948551F8CF8AE00E948551CE01019670
:107990000E94F3571092C50E8091090180FF07C124
:1079A000E4E4FBE084918F01882311F40C94FC3211
:1079B000082E000C990B0E9488870F5F1F4FF8015B
:1079C0008491F2CF8FE40E944CC781110C94FC3259
:1079D00083E40E944CC70C94FC3283E50E944CC7A0
:1079E000811159C08FE40E944CC7882319F08CE0A4
:1079F0009BE007C084E50E944CC7882349F084EED1
:107A00009AE09093FC078093FB070E94B15143C01A
:107A100083E40E944CC7882319F08BEB9AE0F1CFE6
:107A200081E50E944CC7882319F083E99AE0E9CFE9
:107A300088E40E944CC78823C9F0EFE8FAE08491FB
:107A40008F01882351F0082E000C990B0E94888723
:107A50000F5F1F4FF8018491F4CF8DE090E00E94FA
:107A600088878AE090E00E94888715C08CE40E9495
:107A70004CC7882381F0EBE8FAE084918F018823DA
:107A800061F3082E000C990B0E9488870F5F1F4F2F
:107A9000F8018491F4CFE3E5FBE084918F01882322
:107AA00011F40C94FC32082E000C990B0E9488876C
:107AB0000F5F1F4FF8018491F2CF80910B0A8091E4
:107AC0000C0A0C94FC3283E50E944CC7882309F40D
:107AD0006EC083E69AE09093FC078093FB070E94B8
:107AE000B151E3E5FBE084918F01882311F40C94FC
:107AF000FC32082E000C990B0E9488870F5F1F4FE5
:107B0000F8018491F2CFEEE5FAE084918F018823A9
:107B100051F0082E000C990B0E9488870F5F1F4FB1
:107B2000F8018491F4CFE9E5FAE084918F0188238C
:107B300011F40C94FC32082E000C990B0E948887DB
:107B40000F5F1F4FF8018491F2CF88E50E944CC768
:107B5000811106C089E50E944CC7882309F4C3C07F
:107B600088E50E944CC7882341F08AEF9BE0909300
:107B7000FC078093FB070E94B15189E50E944CC726
:107B8000882341F084EF9BE09093FC078093FB07F0
:107B90000E94B1518AE50E944CC7882341F08EEEC5
:107BA0009BE09093FC078093FB070E94B15180916A
:107BB000900E9091910E019664E070E00E94AEDC10
:107BC0009093910E8093900E80918C0E90918D0EDB
:107BD000019690938D0E80938C0E1092940E1092BD
:107BE000930E0C94DD314091900E5091910E9F01B7
:107BF0002F5F3F4F3093940E2093930E90E6949F07
:107C00009001959F300D1124245F324FE20FF31F36
:107C100080830C94DD310091950E1091960E7801C1
:107C200024E0E20EF11C6AE270E0C7010E9431DD3F
:107C3000F80124812F3221F4B8016B5F7F4F03C01C
:107C40002C3339F4B70185EC9EE00E9445DD0C949D
:107C5000FC321092C50E009719F0FC01319710828A
:107C60008091950E9091960E40E061E004960E94FE
:107C700078C58091550C882389F0E5E1FCE084917A
:107C80008F01882309F424CB082E000C990B0E9445
:107C900088870F5F1F4FF8018491F3CFE1E1FCE08B
:107CA00084918F01882309F413CB082E000C990BC3
:107CB0000E9488870F5F1F4FF8018491F3CF0E94C5
:107CC000CF88EDE0FCE084918F01882311F40C94BF
:107CD000FC32082E000C990B0E9488870F5F1F4F03
:107CE000F8018491F2CF8AE50E944CC7811138CF08
:107CF00083E40E944CC7882309F459CF8AEE9BE0A5
:107D000050CF86E40E944CC7882309F44DC10E94DD
:107D100067C70E940EDB8B0186EE9BE09093FC0709
:107D20008093FB070E94B15188E50E944CC78823CD
:107D300009F451C00E9467C72B013C012DEC3CECBB
:107D40004CE45EE30E949BD59E012F5F3F4F79017B
:107D5000181674F020E030E0A901C301B2010E94BE
:107D6000EBDB18162CF41F930F938BED9BE005C1F2
:107D70002DEC3CEC4CEC5DEBC301B2010E949BD5B9
:107D800018167CF020E030E040E85FEBC301B20160
:107D90000E94EBDB18162CF41F930F938FEC9BE0E3
:107DA000ECC01F930F93C301B2010E9409DB7F93C4
:107DB0006F9385EC9BE09F938F93FF92EF920E94CD
:107DC0006DD50FB6F894DEBF0FBECDBFCE010196C4
:107DD0000E948C51DFC089E50E944CC7882309F4BA
:107DE00041C00E9467C72B013C012DEC3CEC4CE4E8
:107DF0005EE30E949BD5FE0131967F01181674F058
:107E000020E030E0A901C301B2010E94EBDB1816AB
:107E10002CF41F930F938AEB9BE0AFC02DEC3CEC4E
:107E20004CEC5DEBC301B2010E949BD518167CF0AF
:107E300020E030E040E85FEBC301B2010E94EBDBE1
:107E400018162CF41F930F938EEA9BE096C01F9395
:107E50000F93C301B2010E9409DB7F936F9384EA01
:107E60009BE0A9CF8AE50E944CC7882309F441C052
:107E70000E9467C72B013C012DEC3CEC4CE45EE317
:107E80000E949BD5FE0131967F01181674F020E008
:107E900030E0A901C301B2010E94EBDB18162CF4FB
:107EA0001F930F9389E99BE068C02DEC3CEC4CECF0
:107EB0005DEBC301B2010E949BD518167CF020E057
:107EC00030E040E85FEBC301B2010E94EBDB181623
:107ED0002CF41F930F938DE89BE04FC01F930F93DB
:107EE000C301B2010E9409DB7F936F9383E89BE09B
:107EF00062CF85E40E944CC7882309F44BC00E94DE
:107F000067C72B013C012DEC3CEC4CE45EE30E9486
:107F10009BD5FE0131967F01181674F020E030E009
:107F2000A901C301B2010E94EBDB18162CF41F93C8
:107F30000F9388E79BE021C02DEC3CEC4CEC5DEB13
:107F4000C301B2010E949BD518167CF020E030E0FE
:107F500040E85FEBC301B2010E94EBDB18162CF482
:107F60001F930F938CE69BE008C0C301B2010E94EF
:107F700009DB7F936F9381E69BE09F938F93FF9242
:107F8000EF920E946DD50F900F900F900F900F9071
:107F90000F901CCF8DE59BE09093FC078093FB072F
:107FA0000E94B1510C94FC3200E010E0B5CE20E00C
:107FB00030E040E251E460913104709132048091EC
:107FC0003304909134040E949BD587FF08C086E556
:107FD0009BE09093FC078093FB070E94B15182E3E2
:107FE00090E090933C0480933B040E94008E88ECC8
:107FF00090E00E942686E3E5FBE084918F018823D0
:1080000011F40C94FC32082E000C990B0E94888706
:108010000F5F1F4FF8018491F2CF20E030E040E283
:1080200051E4609131047091320480913304909155
:1080300034040E949BD587FF08C08CE49BE090939A
:10804000FC078093FB070E94B15180E590E090937C
:108050003C0480933B040E94008E80EF90E00E94DD
:108060002686E3E5FBE084918F01882311F40C94CC
:10807000FC32082E000C990B0E9488870F5F1F4F5F
:10808000F8018491F2CF80E090E00E942686109261
:108090003C0410923B040E94008EE8E4FBE08491D3
:1080A0008F01882311F40C94FC32082E000C990BDC
:1080B0000E9488870F5F1F4FF8018491F2CF6F965F
:1080C0000FB6F894DEBF0FBECDBFDF91CF911F91E9
:1080D0000F91FF90EF90DF90CF90BF90AF909F9067
:1080E0008F907F906F905F904F903F902F9008956A
:1080F0002F923F924F925F926F927F928F929F92B8
:10810000AF92BF92CF92DF92EF92FF920F931F93A5
:10811000CF93DF93CDB7DEB762970FB6F894DEBF8B
:108120000FBECDBFF8948FEF9FEF9093890080939F
:1081300088002AE02A8B212C312C78948091990494
:1081400090919A04A0919B04B0919C04892B8A2B56
:108150008B2B09F016C2809118108823E1F0109241
:1081600018108091161090911710892B09F409C2EC
:1081700010925104109217101092161090910B0A41
:1081800080910C0A981709F4FCC180910C0A8F5F4A
:108190008F7080930C0A8091161090911710892B84
:1081A00009F4EFC1409195045091960460919704B1
:1081B000709198048091910490919204A0919304FD
:1081C000B09194040091880410E020E030E0841B1A
:1081D000950BA60BB70B081719072A073B0710F4D6
:1081E000D901C801E82F840F951FA61FB71F8093E0
:1081F000950490939604A0939704B09398042091CB
:10820000840030918500225E3F4F40916D04509173
:108210006E0460916F047091700480915D04909180
:108220005E04A0915F04B0916004840F951FA61FA7
:10823000B71F80936D0490936E04A0936F04B09366
:108240007004B7FD1CC0889A80912510909126106B
:10825000A0912710B091281040910402042E000C28
:10826000550B660B770B840F951FA61FB71F8093C6
:10827000251090932610A0932710B09328104091BA
:108280007104509172046091730470917404809130
:10829000610490916204A0916304B0916404840F1E
:1082A000951FA61FB71F8093710490937204A0932B
:1082B0007304B0937404B7FD1CC08E9A809129108A
:1082C00090912A10A0912B10B0912C104091050292
:1082D000042E000C550B660B770B840F951FA61F01
:1082E000B71F8093291090932A10A0932B10B0935E
:1082F0002C10409175045091760460917704709130
:1083000078048091650490916604A0916704B0910F
:108310006804840F951FA61FB71F80937504909360
:108320007604A0937704B0937804B7FD3FC08091A2
:108330004B04F09106028823C9F08091490482FF22
:1083400002C0F7FD06C080914804882311F40C9404
:10835000304A8091490490914A0493FF02C0F7FD8E
:108360000CC080914704811108C006C080910B01A8
:108370008095887080930901419A40912D10509109
:108380002E1060912F10709130108F2FFF0F990BCE
:10839000AA0BBB0B840F951FA61FB71F80932D1030
:1083A00090932E10A0932F10B09330104091790429
:1083B00050917A0460917B0470917C0480916904EF
:1083C00090916A04A0916B04B0916C04840F951F86
:1083D000A61FB71F8093790490937A04A0937B041F
:1083E000B0937C04B7FD3AC04091311050913210E7
:1083F0006091331070913410C09007020C2C000C67
:10840000DD08EE08FF084C0D5D1D6E1D7F1D4093BD
:1084100031105093321060933310709334104091A8
:10842000590450915A0460915B0470915C04841B60
:10843000950BA60BB70B8093790490937A04A093C5
:108440007B04B0937C0490914C048091860493FF4C
:1084500002C0815001C08F5F8093860480918400A8
:108460009091850082179307C8F380916D049091D5
:108470006E04A0916F04B0917004B7FD15C04091D7
:10848000590450915A0460915B0470915C04841B00
:10849000950BA60BB70B80936D0490936E04A0937D
:1084A0006F04B09370048898809171049091720465
:1084B000A0917304B0917404B7FD15C040915904A4
:1084C00050915A0460915B0470915C04841B950B7D
:1084D000A60BB70B8093710490937204A09373045E
:1084E000B09374048E988091750490917604A09155
:1084F0007704B0917804B7FD3AC040915904509187
:108500005A0460915B0470915C04841B950BA60B6C
:10851000B70B8093750490937604A0937704B0937F
:10852000780480914B048823E1F08091490482FF14
:1085300004C08091060287FD05C08091480488230D
:1085400009F496C78091490490914A0493FF04C0AE
:108550008091060287FD0BC080914704811107C0FE
:1085600005C080910B018870809309014198E1500A
:1085700041F0809184009091850082179307C8F3A1
:1085800042CE8091110290911202A0911302B091FB
:108590001402892B8A2B8B2B09F091C080918704C0
:1085A000882309F453C08090950490909604A0907D
:1085B0009704B0909804C0908204D0908304E09017
:1085C0008404F090850440918604C814D904EA0418
:1085D000FB0480F48091520490915304209156043E
:1085E000309157042817390728F4415040938604E6
:1085F000019714C08C149D04AE04BF04E0F4809174
:1086000052049091530420915404309155048217E0
:10861000930788F44F5F4093860401969093530428
:108620008093520440910D0250910E0260910F020E
:10863000709110020EC08FEF9FEFDC0180930D024E
:1086400090930E02A0930F02B09310024FEF5FEFD2
:10865000BA018091860487FD02C0169A01C016985F
:1086600080918400909185004E962091860422236B
:10867000F1F0149A20918400309185002817390771
:10868000C8F32091860427FF02C02F5F01C021504C
:1086900020938604149820918604222331F320919C
:1086A00084003091850028173907C8F3DDCF409347
:1086B000110250931202609313027093140280917E
:1086C000990490919A04A0919B04B0919C04892BE9
:1086D0008A2B8B2B09F049C6A0911610B091171068
:1086E000109711F40C94D94B8090950490909604B7
:1086F000A0909704B09098044091910450919204F6
:10870000609193047091940484169506A606B706AA
:10871000D8F01092510410921710109216109091E8
:108720000B0A80910C0A981711F40C94D94B809184
:108730000C0A8F5F8F7080930C0A40EDC42E47E0C7
:10874000D42EE12CF12C1AC440918D0450918E044A
:1087500060918F0470919004481559056A057B0556
:1087600008F4AAC14091890450918A0460918B0455
:1087700070918C04D6960D911D912D913C91D997B5
:10878000401751076207730708F077C1411551057B
:108790006105710549F480904D0490904E04A090BD
:1087A0004F04B090500464C1E12CF980842E952FC1
:1087B000862F0A811B81FD81EE813F8128859C8067
:1087C000E091EE17E89D912CFF273091EF17389D2F
:1087D000900CF11D1090F017189CF00DE99F900C73
:1087E000F11D399FF00DE89FF00D092D1F2F099DF8
:1087F000E12D332722270F9FE00D311D2E1D199DDE
:10880000E00D311D2E1D1F9F300D211D032F122F36
:10881000099DF12C332722270F9FF00C311D2E1DAF
:10882000199DF00C311D2E1D1F9F300D211D032F92
:10883000122FEE2780904D0490914E0480914F04AA
:108840000090A9040E2809F483C03091A504309F3C
:10885000E1198E089E098E092091A604209FE01937
:1088600081089E098E09F090A704F09E8018910956
:108870008E09319FE01981089E098E09219F801879
:1088800091098E09F19E90198109099DF12C3327D8
:1088900022270F9FF00C311D2E1D199DF00C311D4C
:1088A0002E1D1F9F300D211D032F122F3091A1046B
:1088B000309FE10D8E1C9E1D8E1D2091A204209FD5
:1088C000E00D811C9E1D8E1DF090A304F09E800C77
:1088D000911D8E1D319FE00D811C9E1D8E1D219FBF
:1088E000800C911D8E1DF19E900D811D099DF12C16
:1088F000332722270F9FF00C311D2E1D199DF00CE0
:10890000311D2E1D1F9F300D211D032F122F309161
:108910009D04309FE1198E089E098E0920919E04C6
:10892000209FE01981089E098E09F0909F04F09E17
:10893000801891098E09319FE01981089E098E09DE
:10894000219F801891098E09F19E9019810982C09A
:108950003091A504309FE10D8E1C9E1D8E1D20912F
:10896000A604209FE00D811C9E1D8E1DF090A70483
:10897000F09E800C911D8E1D319FE00D811C9E1D6F
:108980008E1D219F800C911D8E1DF19E900D811DCD
:10899000099DF12C332722270F9FF00C311D2E1D2E
:1089A000199DF00C311D2E1D1F9F300D211D032F11
:1089B000122F3091A104309FE1198E089E098E0973
:1089C0002091A204209FE01981089E098E09F09051
:1089D000A304F09E801891098E09319FE019810847
:1089E0009E098E09219F801891098E09F19E901988
:1089F0008109099DF12C332722270F9FF00C311D8F
:108A00002E1D199DF00C311D2E1D1F9F300D211D97
:108A1000032F122F30919D04309FE10D8E1C9E1D5F
:108A20008E1D20919E04209FE00D811C9E1D8E1D99
:108A3000F0909F04F09E800C911D8E1D319FE00DE3
:108A4000811C9E1D8E1D219F800C911D8E1DF19EEF
:108A5000900D811D11249C82F9820A831B83FD8362
:108A6000EE833F832887912C992AA12CB12CA82A28
:108A70008DEA94E121E0298B14C0D2968D909D90CF
:108A8000AD90BC90D597F4CFB694A7949794879463
:108A9000D988DD0CD98A049624E1893C920709F42F
:108AA000EDC4FC0105911591259134910815190526
:108AB0002A053B0548F3E2C44090820450908304A9
:108AC0006090840470908504481459046A047B04FF
:108AD00008F0C3C180918104811121C0FD01EE5BCA
:108AE000FF4FE080F18002811381789620813181EF
:108AF00042815381D2966D917D918D919C91D597B4
:108B00000E9457B6DD24D394D0928104E0911610D0
:108B1000F091171082A993A9A4A9B5A98EC140917B
:108B20007D0450917E0460917F0470918004DA96F8
:108B30000D911D912D913C91DD97401751076207D2
:108B4000730708F073C1411551056105710549F4BA
:108B500080914D0490914E04A0914F04B091500427
:108B60006CC1F0E0E985842F352F262FAA857B85FF
:108B70006C855D85BE854F859889B091EE17B89F4D
:108B8000612D55274091EF17489F600D511D1090A2
:108B9000F017189E500DB39F600D511D439F500D4F
:108BA000B29F500DA62F752FA69FB12D4427992750
:108BB000A59FB00D411D9F1F769FB00D411D9F1FAA
:108BC000759F400D911DA42F792FA69FE12D44275D
:108BD0009927A59FE00D411D9F1F769FE00D411D28
:108BE0009F1F759F400D911DA42F792FBB2780914A
:108BF0004D0430914E0420914F040090A9040F2A97
:108C000009F483C04091A5044A9FB1198F0B3F0B13
:108C10002F0B9091A6049A9FB01981093F0B2F0B3F
:108C2000E091A704EA9F801931092F0B479FB019E3
:108C300081093F0B2F0B979F801931092F0BE79F5D
:108C400030192109A69FE12D44279927A59FE00D02
:108C5000411D9F1F769FE00D411D9F1F759F400D79
:108C6000911DA42F792F4091A1044A9FB10D8F1F10
:108C70003F1F2F1F9091A2049A9FB00D811D3F1F8F
:108C80002F1FE091A304EA9F800D311D2F1F479FE6
:108C9000B00D811D3F1F2F1F979F800D311D2F1F6E
:108CA000E79F300D211DA69FE12D44279927A59F01
:108CB000E00D411D9F1F769FE00D411D9F1F759F79
:108CC000400D911DA42F792F40919D044A9FB11909
:108CD0008F0B3F0B2F0B90919E049A9FB019810927
:108CE0003F0B2F0BE0919F04EA9F801931092F0B56
:108CF000479FB01981093F0B2F0B979F80193109AE
:108D00002F0BE79F3019210982C04091A5044A9F8B
:108D1000B10D8F1F3F1F2F1F9091A6049A9FB00D7A
:108D2000811D3F1F2F1FE091A704EA9F800D311D79
:108D30002F1F479FB00D811D3F1F2F1F979F800D35
:108D4000311D2F1FE79F300D211DA69FE12D4427C8
:108D50009927A59FE00D411D9F1F769FE00D411DA6
:108D60009F1F759F400D911DA42F792F4091A10445
:108D70004A9FB1198F0B3F0B2F0B9091A2049A9F22
:108D8000B01981093F0B2F0BE091A304EA9F8019D2
:108D900031092F0B479FB01981093F0B2F0B979F6C
:108DA000801931092F0BE79F30192109A69FE12D6A
:108DB00044279927A59FE00D411D9F1F769FE00D39
:108DC000411D9F1F759F400D911DA42F792F40912C
:108DD0009D044A9FB10D8F1F3F1F2F1F90919E042E
:108DE0009A9FB00D811D3F1F2F1FE0919F04EA9FA6
:108DF000800D311D2F1F479FB00D811D3F1F2F1F5D
:108E0000979F800D311D2F1FE79F300D211D1124CD
:108E1000E987AA877B876C875D87BE874F87988B9A
:108E200090E0932BA0E0B0E0A22B07C0A65ABF4F62
:108E30008D919D910D90BC91A02D2DEA34E141E0E2
:108E4000498BF901459155916591749148175907DE
:108E50006A077B0708F49CC3A9C380918604882312
:108E6000E1F0FD01E85BFF4F4081518160E070E07F
:108E700000910D0210910E0220910F02309110020C
:108E8000401751076207730741F0109211021092C8
:108E90001202109213021092140240910902509192
:108EA0000A0260910B0270910C0277FF5FC0AE5A0C
:108EB000BF4FCD90DD90ED90FC908DEA94E121E0E4
:108EC000FC0145915591659174914C155D056E05B8
:108ED0007F0550F4F694E794D794C794220F049634
:108EE00074E1893C970761F72093880480E2C816F3
:108EF000D104E104F10428F470E2C72ED12CE12C56
:108F0000F12C90E2C91AD108E108F108C114A8E0D7
:108F1000DA06E104F10408F405C4B4E0DB9EC00104
:108F2000112483559F4EFC01329625913491EC2DEE
:108F30006627E39FA001E29F410D561F0694461F3E
:108F4000561F112460E070E0FC0125913491C901A5
:108F5000A0E0B0E0841B950BA60BB70B8093090231
:108F600090930A02A0930B02B0930C02C0900902E6
:108F7000D0900A02E0900B02F0900C028091161043
:108F800090911710892B09F0E8C10E94D9B69093EF
:108F9000171080931610892B09F4DFC1E091161089
:108FA000F0911710808183FF3EC085899689A7893B
:108FB000B08D8093251090932610A0932710B09326
:108FC0002810818D928DA38DB48D8093291090935C
:108FD0002A10A0932B10B0932C10858D968DA78D01
:108FE000B0A180932D1090932E10A0932F10B093CA
:108FF000301081A192A1A3A1B4A1809331109093CC
:109000003210A0933310B093341090910B0A8091DA
:109010000C0A981709F4B9CF80910C0A8F5F8F70F2
:1090200080930C0AB2CFC588D688E788F08C81E09F
:10903000C114D104E104F10409F480E0018D128D22
:10904000238D348D011511052105310509F082604C
:10905000458D568D678D70A14115510561057105CE
:1090600009F084608093510410927D0410927E0474
:1090700010927F04109280041092890410928A0446
:1090800010928B0410928C0485A196A1A7A1B0A583
:109090008093910490939204A0939304B0939404CA
:1090A000882499245401881A990AAA0ABB0A809232
:1090B000790490927A04A0927B04B0927C0480920E
:1090C000750490927604A0927704B092780480920E
:1090D000710490927204A0927304B092740480920E
:1090E0006D0490926E04A0926F04B0927004CC0C48
:1090F000DD1CEE1CFF1CC0925D04D0925E04E09269
:109100005F04F0926004000F111F221F331F0093B1
:109110006104109362042093630430936404440F49
:10912000551F661F771F4093650450936604609334
:1091300067047093680441A152A163A174A1440F14
:10914000551F661F771F4093690450936A0460930C
:109150006B0470936C04880F991FAA1FBB1F809328
:10916000590490935A04A0935B04B0935C0410924A
:10917000950410929604109297041092980482A578
:1091800093A5A4A5B5A580938D0490938E04A09378
:109190008F04B093900486A597A5A0A9B1A9809348
:1091A000820490938304A0938404B093850481A5E2
:1091B00080935804DF01A95BBF4F9C919093870473
:1091C000992339F115962D913C91119730935704BD
:1091D0002093560412972D913C911197309355048A
:1091E0002093540410921102109212021092130252
:1091F0001092140212972D913C91A90160E070E049
:1092000040930D0250930E0260930F027093100270
:109210000CC088248A94982C540180920D0290925C
:109220000E02A0920F02B0921002EA5BFF4F9081F3
:1092300020914C0492130AC02091080230E0482F7C
:10924000082E000C550B4217530731F090934C0435
:10925000809308020E94A9B68091680681110E943D
:10926000BAAF2FEF3FEFA9012093090230930A0212
:1092700040930B0250930C02E0911610F0911710DE
:10928000DF01DE96ED90FD900D911C9122A933A98E
:1092900044A955A9EA5AFF4F608171818281938167
:1092A0000E9457B610928104E0911610F0911710A9
:1092B000EA5AFF4F80809180A280B3808DEA94E1CA
:1092C00021E0FC014591559165917491481559052E
:1092D0006A057B0558F4B694A79497948794220F57
:1092E0000496A9ECB4E1A817B90759F720938804AC
:1092F000B0E28B169104A104B10428F4B0E28B2EE5
:10930000912CA12CB12C30E2831A9108A108B1084C
:10931000811448E09406A104B10408F427C254E083
:10932000959EC001112483559F4EFC0132962591D4
:109330003491782D6627739FA001729F410D561FAF
:109340000694461F561F1124FC01C590D490E12CB1
:10935000F12CC41AD50AE108F108C0929904D09200
:109360009A04E0929B04F0929C040091990410915D
:109370009A0420919B0430919C04409111025091D9
:1093800012026091130270911402F02E198BF22FC9
:10939000E32F401751076207730720F4F42E598B0F
:1093A000F62FE72F8F2D9989AF2FBE2F0097E1E081
:1093B000AE07B10520F08FEF9FEFA0E0B0E0081BF3
:1093C000190B2A0B3B0B0093990410939A042093DA
:1093D0009B0430939C044F3FFFEF5F076F077F07AD
:1093E00061F0481B590B6A0B7B0B409311025093A1
:1093F00012026093130270931402F8942091840077
:1094000030918500205F3F4F4A8941504A8B442369
:1094100041F0280E391E2216330610F40C949D409C
:1094200001C01901309289002092880078946296D8
:109430000FB6F894DEBF0FBECDBFDF91CF911F9165
:109440000F91FF90EF90DF90CF90BF90AF909F90E3
:109450008F907F906F905F904F903F902F900895E6
:1094600080910B0180958870809309010C94A9412B
:1094700080910B0188708093090164C83989309309
:10948000880480E288169104A104B10428F430E233
:10949000832E912CA12CB12C30E2831A9108A108C3
:1094A000B108811488E09806A104B10420F1E4E039
:1094B0009E9EC001112483559F4EFC01329625913A
:1094C0003491F82DEE27F39F7001F29FE10CFE1E00
:1094D0000694EE1EFE1E1124FC01C590D490860158
:1094E00020E030E0480159018E189F08A108B1081A
:1094F0007501640122C09501840136952795179561
:109500000795F801EC7FCF018355934FFC01C5907F
:10951000D490FC01329625913491E82DE770E29FBA
:10952000C001E39F900D112423E0969587952A951D
:10953000E1F7C81AD90AE12CF12C4C0D5D1D6E1D06
:109540007F1D4093890450938A0460938B04709329
:109550008C049091870480918604992309F473C048
:10956000882309F40BCDA85BBF4F8D919C91A0E09F
:10957000B0E040910D0250910E0260910F02709187
:10958000100284179507A607B70709F05FC0F6CC4D
:10959000B695A79597958795D988DD0CD98A2C5FC4
:1095A0003F4F44E1293C340709F04BCC5989509393
:1095B000880480329105A105B10520F480E290E095
:1095C000A0E0B0E08097A109B109811558E09507A6
:1095D000A105B10508F443C074E0979F90011124E0
:1095E00023553F4EF901329645915491EE27859FC0
:1095F000B001849F610D7E1F06946E1F7E1F112493
:10960000F901C590D490E12CF12CC61AD70AE108D3
:10961000F10880917D0490917E04A0917F04B09127
:1096200080048C0D9D1DAE1DBF1D80937D04909305
:109630007E04A0937F04B0938004809187048111FD
:1096400030C080918604882309F498CC10921102CE
:109650001092120210921302109214028FCCAC01DD
:10966000BD017695679557954795FA01EC7F9F0167
:109670002355334FF901C590D490F90132964591A5
:1096800054918770849F9001859F300D1124F3E0E1
:1096900036952795FA95E1F7C21AD30AE12CF12CF9
:1096A000B8CF8989480E511C611C711C809116101D
:1096B00090911710481459046A047B04D8F420913F
:1096C0008604222309F45ACCFC01E85BFF4F208179
:1096D0003181A90160E070E000910D0210910E024D
:1096E00020910F0230911002401751076207730753
:1096F00009F444CC1092110210921202109213023B
:1097000010921402FC01E85BFF4F80819181A0E080
:10971000B0E080930D0290930E02A0930F02B093DD
:1097200010022CCCD701C601B695A79597958795C1
:10973000FC01EC7FCF018355934FFC0125913491BF
:10974000FC013296459154916C2D6770649FC00165
:10975000659F900D112463E0969587956A95E1F7D2
:10976000281B390BC901A0E0B0E0F8CBD501C4013A
:10977000B695A79597958795FC01EC7FCF0183550A
:10978000934FFC01C590D490FC0132962591349101
:10979000482D4770429FC001439F900D1124A3E0C4
:1097A00096958795AA95E1F7C81AD90AE12CF12C6C
:1097B000D4CD80EDC82E87E0D82EE12CF12CE5CB5E
:1097C00090910318E92FF0E0EB58F94F80839F5FE9
:1097D000943018F49093031802C0109203188091EB
:1097E00004188F5F8093041808958091AA059091C2
:1097F000AB05981759F0E92FF0E0E65DFA4F80814C
:109800009F5F9F779093AB0590E008958FEF9FEF58
:1098100008950F931F93CF93DF93FC01A685B7851F
:109820008D0100581F4FE8018881998101968F773B
:109830009927AD014E575F4FEA01288139812817DA
:109840003907D1F3E80128813981A20FB31F6C9346
:10985000A685B785A058BF4F11969C938E93A68975
:10986000B7892C9181E090E0078C02C0880F991F86
:109870000A94E2F7822B8C9381E081A30488F58916
:10988000E02D80818064808381E090E0DF91CF9142
:109890001F910F910895FC0181A1882329F0A489CB
:1098A000B5898C9186FFFBCF11A20895FC01A48598
:1098B000B585FD01E058FF4F2081318132968081CE
:1098C00091812817390779F080819181A80FB91FFC
:1098D0008C91208131812F5F3F4F2F773327318348
:1098E000208390E008958FEF9FEF0895DC011C9690
:1098F000ED91FC911D97DF01A058BF4F2D913C9138
:10990000119712968D919C9111972817390739F06C
:109910008D919C91E80FF91F808190E008958FEF61
:109920009FEF0895FC0124853585F901E058FF4F2C
:109930008081918132962081318180589F4F821B96
:10994000930B60E870E00C94AEDC0895089580E01D
:1099500090E00895CF93FC0120812B33A1F020915A
:109960000418243080F4C62FBC0180910318F0E65F
:109970008F9FC00111248658994F0E9445DD8C2F7E
:109980001FDF81E001C080E0CF9108952F923F92C8
:109990004F925F926F927F928F929F92AF92BF92FF
:1099A000CF92DF92EF92FF920F931F93CF93DF93AB
:1099B00000D000D0CDB7DEB79A8389830E9410C54E
:1099C000E981FA81C680D780E084F184C114D10492
:1099D000E104F10409F0ACC22485222309F469C32F
:1099E00032852150248721E0230F228745852413C7
:1099F00001C01286E981FA8124E0329FE00DF11D59
:109A00001124C684D784E088F188E981FA81C28272
:109A1000D382E482F582DC01CB018C0D9D1DA11D5A
:109A2000B11D86839783A087B18784819581892B17
:109A300009F43FC3FFB7FD83F894E981FA812280DE
:109A400033802101612C712C0481158180912D02BC
:109A50008F3121F08F3F09F068C205C0ECE9F9E1D0
:109A600024912E83DAC08FE180932D02ECE9F9E195
:109A700084918E838F3F09F458C2823009F469C003
:109A800030F5882309F44CC0813009F0C6C010922B
:109A90008000109281008091810088608093810015
:109AA00080918100816080938100E6EAF7E2E49191
:109AB000F0E0EE0FFF1FED5AF84D85919491ECEE1A
:109AC000F7E2E491E093AD04E1E0EE8330C19E81E2
:109AD000943009F482C008F460C0953009F09DC04C
:109AE00010922001109221018091210188608093C1
:109AF000210180912101816080932101E6EAF7E252
:109B0000E491F0E0EE0FFF1FED5AF84D859194912E
:109B1000ECEEF7E2E491E093AA0495E09E8307C19E
:109B200014BC15BC84B5826084BD85B5816085BDDB
:109B3000E6EAF7E2E491F0E0EE0FFF1FED5AF84D90
:109B400085919491ECEEF7E2E491E093AE041E82ED
:109B5000ABC21092B0001092B1008091B000826050
:109B60008093B0008091B10081608093B100E6EAFB
:109B7000F7E2E491F0E0EE0FFF1FED5AF84D85910A
:109B8000949190935A0680935906ECEEF7E2E49193
:109B9000E0935B06F2E0FE8387C210929000109281
:109BA0009100809191008860809391008091910054
:109BB000816080939100E6EAF7E2E491F0E0EE0F35
:109BC000FF1FED5AF84D85919491ECEEF7E2E49188
:109BD000E093AC0423E02E83AAC01092A000109260
:109BE000A1008091A10088608093A1008091A100D4
:109BF00081608093A100E6EAF7E2E491F0E0EE0FE5
:109C0000FF1FED5AF84D85919491ECEEF7E2E49147
:109C1000E093AB0484E08E838AC0EE81E7FD85C1CA
:109C200061E08FE10E94D5C38E818D7F09F083C0F2
:109C30004801A12CB12C60E072E18AE790E0A50117
:109C400094010E94C1DC29833A834B835C836901C0
:109C50007A01F1E0CF1AD108E108F1082FEFC2161E
:109C6000D104E104F10409F008F44EC060E472E4A8
:109C70008FE090E0A50194010E94C1DC69017A01A6
:109C800081E0C81AD108E108F1089E81923009F5F7
:109C9000EFEFCE16D104E104F10409F008F4CBC1D2
:109CA00060E970ED83E090E0A50194010E94C1DCC1
:109CB00069017A01F1E0CF1AD108E108F1082FEF2C
:109CC000C216D104E104F10411F008F041C183E0AF
:109CD00027C08FEFC816D104E104F104B9F0B0F049
:109CE00068E478EE81E090E0A50194010E94C1DC77
:109CF00069017A0191E0C91AD108E108F108EE8101
:109D0000EE2309F49AC163C181E001C082E09E8123
:109D1000911106C095B5987F892B85BD7AC085E0E5
:109D20009091B100987F892B8093B10072C061E05F
:109D30008FE10E94D5C34801A12CB12C60E072E1F3
:109D40008AE790E0A50194010E94C1DC69017A01D3
:109D5000E1E0CE1AD108E108F108C114D104F1E024
:109D6000EF06F10488F068E478EE81E090E0A50168
:109D700094010E94C1DC69017A0181E0C81AD1080E
:109D8000E108F10883E001C081E09E81913071F427
:109D900090918100987F892B8093810045284628E7
:109DA0004728D9F52FEF3FEFA90168C0EE81E330D6
:109DB00071F490919100987F892B809391004528B0
:109DC0004628472851F52FEF3FEFA90179C0FE81C2
:109DD000F43071F49091A100987F892B8093A100B9
:109DE000452846284728C9F42FEF3FEFA9017AC03C
:109DF0002E81253071F490912101987F892B8093D9
:109E0000210145284628472841F42FEF3FEFA901BB
:109E10007BC045284628472869F0D801AA0FBB1FF8
:109E200091010E94B5D928EE33E040E050E00E9455
:109E300089D903C02FEF3FEFA9018E81823081F1D4
:109E40002CF4882361F08130C9F06FC09E8194307A
:109E500009F448C0ACF1953009F456C066C0C7BCDF
:109E60002093BF043093C0044093C1045093C204B4
:109E700080916E00826080936E0057C0D0928900FE
:109E8000C09288002093BB043093BC044093BD046F
:109E90005093BE0480916F00826080936F0045C034
:109EA000C092B30020935C0630935D0640935E063B
:109EB00050935F068091700082608093700035C07F
:109EC000D0929900C09298002093B7043093B804C0
:109ED0004093B9045093BA048091710082608093DA
:109EE000710023C0D092A900C092A8002093B304AF
:109EF0003093B4044093B5045093B604809172003B
:109F000082608093720011C0D0922901C092280112
:109F10002093AF043093B0044093B1045093B20443
:109F200080917300826080937300ED81EFBFC1C0A8
:109F3000DC01CB018C199D09AE09BF09B7FDB9C081
:109F40004698E981FA811682178210861186B1C07F
:109F500068E478EE81E090E0A50194010E94C1DC04
:109F600069017A01F1E0CF1AD108E108F1082FEF79
:109F7000C216D104E104F10441F138F164E274EF56
:109F800080E090E0A50194010E94C1DC69017A01A2
:109F9000F1E0CF1AD108E108F1082FEFC216D10481
:109FA000E104F10409F008F4BACE62E17AE780E056
:109FB00090E0A50194010E94C1DC69017A0181E071
:109FC000C81AD108E108F10819C084E0A9CE2FEF22
:109FD000C216D104E104F10409F008F463C062E19F
:109FE0007AE780E090E0A50194010E94C1DC69015C
:109FF0007A01F1E0CF1AD108E108F1082FEFC2167B
:10A00000D104E104F104A9F0A0F089819A81AB8127
:10A01000BC812AE0B595A795979587952A95D1F7A4
:10A020006C017D01F1E0CF1AD108E108F10887E069
:10A0300077CE86E075CE82E073CEEFEFCE16D104F8
:10A04000E104F10469F160F162E17AE780E090E017
:10A05000A50194010E94C1DC69017A0181E0C81A5E
:10A06000D108E108F1089FEFC916D104E104F10419
:10A07000A9F0A0F089819A81AB81BC813AE0B595C5
:10A08000A795979587953A95D1F76C017D01E1E009
:10A09000CE1AD108E108F10885E03CCE84E03ACE42
:10A0A00083E038CE84E033CE61E08FE10E94D5C3F7
:10A0B000BFCD26960FB6F894DEBF0FBECDBFDF91A1
:10A0C000CF911F910F91FF90EF90DF90CF90BF90B5
:10A0D000AF909F908F907F906F905F904F903F9048
:10A0E0002F9008950F931F93CF93DF93CDB7DEB7D3
:10A0F0002C970FB6F894DEBF0FBECDBFE9E2F4E0B7
:10A1000080859185A285B38544815581668177815B
:10A11000008111812281338109831A832B833C833F
:10A120004D835E836F83788789879A87AB87BC87E7
:10A13000AE01475F5F4FBE016B5F7F4FCE0101965F
:10A140000E94BDAE25E334E0AE01475F5F4FBE0124
:10A150006B5F7F4FCE0101960E9416BA2C960FB608
:10A16000F894DEBF0FBECDBFDF91CF911F910F914D
:10A17000089580910C0490910D04009731F04AE00D
:10A1800050E060E070E00C94EFD260E070E0CB0152
:10A190000895EFDF97FD0AC0ECDF6F3F7105810581
:10A1A000910509F02CF4E5DF862F089580E00895ED
:10A1B0008FEF089580910C0490910D04892B31F05C
:10A1C000E8DF91E0811103C090E001C091E0892FA8
:10A1D00008950F931F93CF9380910C0490910D04D9
:10A1E000009711F1FC018F01C1912C2F2F7DA9F057
:10A1F000C53411F0C536B9F7F801108260E070E09F
:10A2000080910C0490910D040E949CD1F801C083B0
:10A21000562F472F382F292F0BC060E070E0CF91C9
:10A220001F910F910C949CD150E040E030E020E071
:10A23000652F742F832F922FCF911F910F91089527
:10A2400081548A3108F042C0E82FF0E040912E1886
:10A2500050912F18609130187091311804C0769584
:10A260006795579547958A95D2F7842F817040FF5F
:10A270002FC0EC5EF74E9081992309F1E091F3171E
:10A28000F091F417E90FF11D908120ED290F2A308C
:10A2900098F09E3211F491810CC09D3211F09B32E6
:10A2A00071F4918120ED290F2A3030F09E3239F47B
:10A2B000928190539A3018F42E2F9F2F02C020E0E5
:10A2C00090E020930C0490930D04089580E008958D
:10A2D0000895B6DF882341F081E020910C0430918D
:10A2E0000D04232B09F480E00895FC012381211142
:10A2F0000C94BFA2089580E1E9E2F4E0A0EEB5E09D
:10A3000001900D928A95E1F708959091C00095FF14
:10A31000FCCF8093C6000895EF92FF921F93CF93D6
:10A32000DF937C0160E016DB182F882399F0ECE7BF
:10A33000FBE18491EF012196882319F0E6DFFE010D
:10A34000F8CFB7018DEC94E10E9461B782E2DDDFC6
:10A350008AE0DBDF812FDF91CF911F91FF90EF909B
:10A360000895DF92EF92FF920F931F93CF93DF93A5
:10A37000CDB7DEB76E970FB6F894DEBF0FBECDBF78
:10A380006091FB077091FC076115710541F14DE18A
:10A3900050E0CE0101967C010E9444D51E8EF7014B
:10A3A0008F010E191F09D190DD2019F09AE0D91202
:10A3B000F7CFF701E00FF11F1082C701ADDF88234F
:10A3C00071F0DD20A9F00F5F1F4F8091FB07909186
:10A3D000FC07080F191F1093FC070093FB0781E08F
:10A3E0002091FB073091FC07232B29F480E003C068
:10A3F00000E010E0F0CF6E960FB6F894DEBF0FBE0F
:10A40000CDBFDF91CF911F910F91FF90EF90DF9023
:10A4100008953F924F925F926F927F928F929F9298
:10A42000AF92BF92CF92DF92EF92FF920F931F9362
:10A43000CF93DF931F92CDB7DEB793DF811174C244
:10A4400080910418843008F047C0CFD9AC0197FF41
:10A450007CC142C08E3409F0D9C10115110509F43F
:10A46000D5C160E076E1C8010E9453D57C01892BFB
:10A4700009F48EC16EE470E0C80104960E9431DDDB
:10A48000009709F485C14AE050E060E070E0019671
:10A490000E94EFD26093C3047093C4048093C504F8
:10A4A0009093C6048090101890901118A0901218E4
:10A4B000B09013182FEF821A920AA20AB20A6815F6
:10A4C00079058A059B0509F465C1EF2809F062C189
:10A4D0008DEC95E10E941AC78091890A882309F4BE
:10A4E00023C280910418811102C010922905EE2424
:10A4F000E3944091030D5091040D6091050D70910E
:10A50000060D8091FF0C9091000DA091010DB0916E
:10A51000020D481759076A077B0708F4E12C00E091
:10A5200010E09924939480E6882E95E0A92E96E178
:10A53000B92E2DE8322E80910418843008F0F4C131
:10A54000E110F2C1809129058111EEC180915A0C70
:10A5500090915B0CA0915C0CB0915D0C8093030D0D
:10A560009093040DA093050DB093060D41E050E0CB
:10A57000BE016F5F7F4F82E59CE00E9446A5019778
:10A5800019F4898190E002C08FEF9FEFF82E409080
:10A59000030D5090040D6090050D7090060D4091D4
:10A5A000FF0C5091000D6091010D7091020DEE2491
:10A5B000E394441655066606770608F4E12C441623
:10A5C000550666067706B0F4019609F46AC08AE07B
:10A5D000F81609F489C09DE0F91609F485C023E254
:10A5E000F21619F08AE3F81296C0809128058111BD
:10A5F00092C06FC00E94127182E59CE00E94BFA2CF
:10A6000080916D0C882359F1815080936D0C389E98
:10A61000C001112441E061E08E58934F0E9478C53B
:10A62000E0916D0C94E0E99FF0011124E259F34FA1
:10A6300040815181628173814093030D5093040DD9
:10A640006093050D7093060D82E59CE00E94D5A1F4
:10A6500080918A0A8823A9F09092890A12C01092E8
:10A66000890A0E949FA90E942F900E94BE8F6D337D
:10A6700071058105910528F0B092FC07A092FB07B7
:10A6800070DE8091890A811128C0E8E1F6E18491A9
:10A690006F012FEFC21AD20A8823D9F036DEF601F5
:10A6A000F6CFE7E6FBE184916F019FEFC91AD90A63
:10A6B000882319F02ADEF601F6CFE9E0F6E184916D
:10A6C0006F012FEFC21AD20A882319F01EDEF6019D
:10A6D000F6CF83E2F81208C005C023E2F21221C1CE
:10A6E00000E010E09092290510922805011511054F
:10A6F00019F40E9404930CC080910318889E000DE9
:10A70000111D1124F801E658F94F108280E058D845
:10A7100000E010E010CF0F35110508F00CCF9BE3DF
:10A72000F91202C09092280580912805811103CF6B
:10A7300080910318F801889EE00DF11D1124E65860
:10A74000F94FF0820F5F1F4FF6CE982F20910E1811
:10A7500030910F188A3019F09D3009F0B0C0109276
:10A7600027052115310519F40E94049369CEF901DA
:10A77000E953FB4F108210920F1810920E1807EC3D
:10A7800014E0F8018191803209F064CE8F01F9CF95
:10A79000C80179CE6AE270E0C8010E9469DD9C01BF
:10A7A000009701F1982F901BF12C992339F09150CB
:10A7B000F801E90FF11D8081F826F7CF4AE050E05B
:10A7C00060E070E0C90101960E94EFD2CF2CD12C3D
:10A7D000E12CF12C6C157D058E059F0531F08EEA7C
:10A7E00095E178CE84E895E175CE8091C30490918F
:10A7F000C404A091C504B091C6048093101890932E
:10A800001118A0931218B09313180EC08091870AE4
:10A81000882351F064EE73E0C8010E943CDD892B6F
:10A8200019F08AE595E156CE80913502811126C056
:10A8300067E470E0C8010E9431DD0097F9F04AE05A
:10A8400050E060E070E001960E94EFD297FD16C0E4
:10A8500064307105810591052CF065307105810525
:10A86000910561F4E3EEF4E184917F019FEFE91A31
:10A87000F90A882319F049DDF701F6CF68EE73E095
:10A88000C8010E943CDD892B11F4109234026DEE58
:10A8900073E0C8010E943CDD892B19F48AED94E134
:10A8A000C4D362EF73E0C8010E943CDD892B11F430
:10A8B0000E949B9A61E087EC94E04CD8C1CD2F3583
:10A8C00031050CF0BDCD9C35C1F40E94F54B97FDD0
:10A8D000B7CD209127052111B3CD20910E183091CD
:10A8E0000F18A9014F5F5F4F50930F1840930E1838
:10A8F000F901E953FB4F8083A3CD9B3319F481E029
:10A90000809327058091270581119ACDC901019671
:10A9100090930F1880930E18F901E953FB4F408371
:10A920008FCD10922805E5CE0F90DF91CF911F912A
:10A930000F91FF90EF90DF90CF90BF90AF909F90DE
:10A940008F907F906F905F904F903F9008958F927F
:10A950009F92AF92BF92EF92FF920F931F93CF936C
:10A96000DF93CDB7DEB7A0970FB6F894DEBF0FBE6A
:10A97000CDBF611571058105910589F100E0842E37
:10A98000912CA12CB12C102FEE24E394F12CEC0E81
:10A99000FD1EE00EF11C07FDFA94A50194010E9432
:10A9A00089D9F7016083B901CA010F5F611571058B
:10A9B0008105910541F71F3F21F1E1E0F0E0EC0F47
:10A9C000FD1FE10FF11D17FDFA9580818A3010F00F
:10A9D00097E301C090E3890F98DC1150ECCF80E33E
:10A9E000A0960FB6F894DEBF0FBECDBFDF91CF911A
:10A9F0001F910F91FF90EF90BF90AF909F908F901D
:10AA000084CCA0960FB6F894DEBF0FBECDBFDF9109
:10AA1000CF911F910F91FF90EF90BF90AF909F90BB
:10AA20008F900895EF92FF920F931F93CF93DF9330
:10AA30007C0184E54EDCD82F882321F1AADBC82FC6
:10AA40001816E4F4ECE7FBE184918F010F5F1F4FD0
:10AA5000882319F05ADCF801F7CF8DE456DCB701F2
:10AA600080E090E04AE073DF6C2FCC0F770B8CE234
:10AA700096E10E9448B78AE048DC08C080935C10E9
:10AA8000D0E004C08091C40580935C108D2FDF91CD
:10AA9000CF911F910F91FF90EF900895CF92DF9289
:10AAA000EF92FF926B017C0197FF0AC08DE22DDCD3
:10AAB000F094E094D094C094C11CD11CE11CF11C12
:10AAC0004AE0C701B601FF90EF90DF90CF903FCFF3
:10AAD0008F929F92AF92BF92CF92DF92EF92FF92AE
:10AAE000CF936B017C01B42E20E030E0A9010E94DD
:10AAF0009BD587FF06C08DE208DCF7FAF094F7F8E3
:10AB0000F094C0E060E070E080E09FE3CB1541F09E
:10AB10002DEC3CEC4CEC5DE30E9400D6CF5FF6CF11
:10AB20009B01AC01C701B6010E94C5D96B017C0134
:10AB30000E940EDB4B015C014AE009DFCC2379F176
:10AB4000C501B4010E949FD59B01AC01C701B601AC
:10AB50000E94C4D96B017C018EE2D7DB20E030E09B
:10AB600040E251E4C701B6010E9400D64B015C01EE
:10AB70000E9409DB6B01770FEE08FF08C701B601E1
:10AB80008DDFC701B6010E94A1D59B01AC01C501B3
:10AB9000B4010E94C4D96B017C01C150F9F6CF9178
:10ABA000FF90EF90DF90CF90BF90AF909F908F90ED
:10ABB00008951F920F920FB60F9211240BB60F92A9
:10ABC0002F938F939F93EF93FF932091AB05E09189
:10ABD000AA0581E08E0F8F779091C600281729F083
:10ABE000F0E0E65DFA4F9083E82FE093AA05FF912D
:10ABF000EF919F918F912F910F900BBE0F900FBEF1
:10AC00000F901F9018959C0197FD0EC084369105FA
:10AC100084F064E670E00E94AEDCCB016AE070E094
:10AC20000E94AEDC805D06C03195219531098DE230
:10AC300001C080E2809324042A30310564F0EAE008
:10AC4000F0E0C901BF010E94AEDCCB01BF010E9450
:10AC5000AEDC805D01C080E280932504C9016AE01A
:10AC600070E00E94AEDC805D8093260484E294E074
:10AC700008951F920F920FB60F9211240BB60F92E8
:10AC80002F933F938F939F93EF93FF9320916A0F9E
:10AC900030916B0F80916C0F90916D0F28173907D1
:10ACA00031F4809131018F7D8093310114C0E091A6
:10ACB0006C0FF0916D0FE651F14F208180916C0F78
:10ACC00090916D0F01968F77992790936D0F8093D8
:10ACD0006C0F20933601FF91EF919F918F913F91DF
:10ACE0002F910F900BBE0F900FBE0F901F901895D5
:10ACF0001F920F920FB60F9211240BB60F922F9343
:10AD00004F935F938F939F93EF93FF9380913001C5
:10AD100082FD1CC0209136018091EE0F9091EF0FC3
:10AD20004091F00F5091F10F01968F7799274817B6
:10AD3000590771F0E091EE0FF091EF0FE259F04FEB
:10AD400020839093EF0F8093EE0F02C08091360125
:10AD5000FF91EF919F918F915F914F912F910F9064
:10AD60000BBE0F900FBE0F901F9018958FEF8EBDEA
:10AD70000DB407FEFDCF8EB508954F925F926F928E
:10AD80007F928F929F92AF92BF92CF92DF92EF927B
:10AD9000FF920F931F93CF93DF93D82EC82FD0E04D
:10ADA000FE01ED55F84EC49082E0D81203C081E058
:10ADB00080934B047E01EE0CFF1CEE0CFF1CF70190
:10ADC000E956F84E45905590659074906C2D0C2C7A
:10ADD000000C770B880B990B0E94A1D54B015C01ED
:10ADE00020E030E040EC5FE3C301B2010E9400D6F6
:10ADF000A50194010E9400D6AB01BC0100E010E067
:10AE000098018D2D0E941175F701E557F84E259197
:10AE1000359145915491C501B4010E9400D64B0172
:10AE20005C0120E030E0A9010E949BD5882309F451
:10AE300046C000E010E09801B501A40170588D2DC6
:10AE40000E941175FE01E857F84EC491C11115C05A
:10AE5000ECE7FBE18491EF012196882319F055DAA4
:10AE6000FE01F8CFE6E6F7E18491EF012196882311
:10AE700019F04BDAFE01F8CFCAE0F701E459F74DBB
:10AE800045905590659074906C2F70E080E090E054
:10AE90000E94A1D59B01AC01C301B2010E94A1DABD
:10AEA0002B013C01A5019401C501B4010E94C5D943
:10AEB000AB01BC01930182018D2D0E94117582E0CE
:10AEC000D81249C040902611509027116090281147
:10AED0007090291120E030E0A901C301B2010E9465
:10AEE000EBDB5301420187FF04C0B7FAB094B7F817
:10AEF000B09420E030E0A901C501B4010E949BD5C7
:10AF0000882349F120E030E0A901C301B2011C14FB
:10AF10002CF40E94EBDB18162CF008C00E949BD585
:10AF200087FF04C081E08093480403C081E08093E0
:10AF300047041C1424F4B7FAB094B7F8B09400E0B6
:10AF400010E09801B501A40182E00E9411751092F1
:10AF500048041092470410924B0481E090E00D2CBD
:10AF600001C0880F0A94EAF790912804982B9093D7
:10AF700028049091DF05892B8093DF05F701ED52BE
:10AF8000FA4F10821182128213828D2D0E946E77E9
:10AF9000F701E65AF84E85919591A591B491E70194
:10AFA000C75DDB4F88839983AA83BB839BD8F70156
:10AFB000E052FA4F88819981AA81BB818083918375
:10AFC000A283B383DF91CF911F910F91FF90EF90F8
:10AFD000DF90CF90BF90AF909F908F907F906F90B9
:10AFE0005F904F90089525EE32E0FC01318320837D
:10AFF00004967BC95F9A809128048E7F80932804F1
:10B000008A9A479A809128048D7F809328048091A2
:10B0100008018095817080930601479A80912804E9
:10B020008B7F80932804129A0895E7E6FBE18491D0
:10B03000EF012196882319F068D9FE01F8CFEAE3E1
:10B04000F7E18491EF012196882319F05ED9FE0182
:10B05000F8CF0E944490CEDFE6E3F7E18491EF0160
:10B06000882349F0082E000C990B0E9488872196AE
:10B07000FE018491F5CF8DE090E00E9488878AE000
:10B0800090E00E948887FFEF2BE48DE1F150204093
:10B090008040E1F700C00000F8949FEFE4E3FCE09B
:10B0A0009150E040F040E1F700C000000E94449061
:10B0B000A895FECF2F923F924F925F926F927F9210
:10B0C0008F929F92AF92BF92CF92DF92EF92FF92B8
:10B0D0000F931F93CF93DF9300D01F92CDB7DEB7AE
:10B0E0000E94D3300E9410C56B017C011091220296
:10B0F000112309F475C08091C505882309F470C037
:10B100004091FC055091FD056091FE057091FF0591
:10B1100046015701841A950AA60AB70AB7FC72C0FD
:10B12000833041F134F481300CF45AC0ECE7FBE198
:10B1300006C0843009F054C0ECE7FBE137C08491CD
:10B140009F012F5F3F4F3B832A83882321F0DDD867
:10B15000EA81FB81F4CFE4EBF6E184919F012F5F5C
:10B160003F4F3B832A83882309F43AC0CED8EA8133
:10B17000FB81F3CFECE7FBE184919F012F5F3F4F11
:10B180003B832A83882321F0C0D8EA81FB81F4CF56
:10B19000EDE9F6E184919F012F5F3F4F3B832A83C6
:10B1A0008823F1F0B2D8EA81FB81F4CF84919F012A
:10B1B0002F5F3F4F3B832A83882321F0A6D8EA8163
:10B1C000FB81F4CFE5E8F6E184919F012F5F3F4FCB
:10B1D0003B832A83882321F098D8EA81FB81F4CF2E
:10B1E000212F30E0A8EEB3E00E94B5D9C60ED71EDD
:10B1F000E81EF91EC092FC05D092FD05E092FE0506
:10B20000F092FF0589B182FB882780F98093E40ED4
:10B210009091E50E98170CF049C08091E60E909140
:10B22000E70EA091E80EB091E90E0196A11DB11DA7
:10B23000883B3DE39307A105B1054CF48093E60EEE
:10B240009093E70EA093E80EB093E90E3BC01092E6
:10B25000E60E1092E70E1092E80E1092E90E809121
:10B26000890A882319F00E94F0881DC0E6ECF6E1F7
:10B270008491FB83EA83882371F0082E000C990BDC
:10B280000E9488872A813B812F5F3F4F3B832A831F
:10B29000F9018491F0CF8DE090E00E9488878AE0E8
:10B2A00090E00E9488878091E40E0AC0891751F0CF
:10B2B0001092E60E1092E70E1092E80E1092E90E30
:10B2C0008093E50E80910418843008F4A2D80E947F
:10B2D00010C5C090CA05D090CB05E090CC05F09089
:10B2E000CD05C114D104E104F10489F10091C60532
:10B2F0001091C7052091C8053091C9050C0D1D1D81
:10B300002E1D3F1D4B015C01801A910AA20AB30A4F
:10B31000B7FC1DC0E7E6FBE184919F012F5F3F4F23
:10B320003B832A83882329F00E948551EA81FB818F
:10B33000F3CF6091F3177091F4178CEF96E10E94B0
:10B3400061B78AE00E94855183EF96E181C0C09089
:10B350002302D0902402E0902502F0902602C1142E
:10B36000D104E104F104E9F130910B0A20910C0AB7
:10B37000321749F06093C6057093C7058093C805DE
:10B380009093C9052EC00091C6051091C705209164
:10B39000C8053091C9050C0D1D1D2E1D3F1DDC017A
:10B3A000CB01801B910BA20BB30BB7FD1AC05F9AA8
:10B3B000809128048E7F809328048A9A479A8091EE
:10B3C00028048D7F809328048091080180958170E6
:10B3D00080930601479A809128048B7F80932804EC
:10B3E000129A80910C0690910D06909902C00196D8
:10B3F00004C0181619062CF4019790930D0680933B
:10B400000C0680910C0690910D068E3E92400CF138
:10B41000E7E6FBE184919F012F5F3F4F3B832A8347
:10B42000882329F00E948551EA81FB81F3CFE3ED67
:10B43000F6E184919F012F5F3F4F3B832A8388234E
:10B4400029F00E948551EA81FB81F3CF8AEC96E1D5
:10B45000ECDD0E9410C500910806109109062091AC
:10B460000A0630910B064B015C01801A910AA20A70
:10B47000B30AB7FC4EC08B019C010C53164F2F4FE3
:10B480003F4F009308061093090620930A06309355
:10B490000B064F9BA9C17A9BA7C12091060120FFF3
:10B4A000A3C120915B1021119FC1379B9DC1379B88
:10B4B0009BC1029B99C10091040610910506209141
:10B4C000060630910706011511052105310599F091
:10B4D000DC01CB01801B910BA20BB30B80569A4E63
:10B4E000A109B1098827B7FD83959927AA27BB270A
:10B4F000682F619501C060E0262F30E08091020145
:10B5000061118095807180930001B90187E00E94EC
:10B5100011C490910B0A80910C0A981791F0E09158
:10B520000C0A28E6E29FF0011124E053FE4E6081F0
:10B5300080910C0A90910B0A981729F08F5F8F70F9
:10B54000F9CF6091390470E089E00E9411C48091C4
:10B550005610882309F4F8C0009143021091440268
:10B56000809045028C82909046029A8260914104BC
:10B57000709142046E5F7F4F072E000C880B990B71
:10B580000E94A1D59801A4010E949BD587FDDCC033
:10B59000F0900C0A212C312CE12C198280910B0A9D
:10B5A0008F1509F462C08F2D90E038E6A32EA89E77
:10B5B000F001A99EF00D1124E259FE4E45895689ED
:10B5C0006789708D452B462B472B81F4418D528D19
:10B5D000638D748D452B462B472B41F4458D568D3D
:10B5E000678D70A1452B462B472BD1F128E6B22E53
:10B5F000B89E9001B99E300D1124C90182599E4E0A
:10B600006C01FC0161817281838194810E9430DC34
:10B610004B015C01F60161A172A183A194A10E947A
:10B620009FD52B013C01F60165A176A187A190A5CC
:10B630000E949FD59B01AC01C301B2010E94A1DA17
:10B64000A50194010E9400D65B016C0191014E2D71
:10B6500059810E94EBDB18161CF41501EC2CD982E1
:10B6600081E08F0D8F70F82E99CF20914702309195
:10B6700048024091490250914A02B1018E2D9981B0
:10B680000E9400D698014C815A810E94C5D96B0155
:10B690007C019B01AC01B8018C819A810E94EBDB9B
:10B6A0001816ACF000913F021091400280904102C8
:10B6B0008C82909042029A829801A401B601C7013F
:10B6C0000E94EBDB18161CF08601EC82FA82C09017
:10B6D0000006D0900106E0900206F0900306980163
:10B6E0004C815A81C701B6010E94EBDB1816D4F4D5
:10B6F00020E037ED43EA5CE3B8018C819A810E9437
:10B7000000D64B015C0128E431EE4AE75FE3C70154
:10B71000B6010E9400D6A50194010E94C5D98B01F3
:10B720008C839A83C801AC81BA8180930006909380
:10B730000106A0930206B0930306B801CD010E9452
:10B7400009DBCB010E9426860E94049389E69AE0D9
:10B750000E94C64CA090D205A982AA2009F44DC02F
:10B760000E9410C50091CE051091CF052091D00503
:10B770003091D105DC01CB01801B910BA20BB30BE7
:10B78000B7FD3BC00E9410C56B017C01B9802B2D19
:10B7900030E0A8EEB3E00E94B5D9C60ED71EE81E71
:10B7A000F91EC092CE05D092CF05E092D005F0925E
:10B7B000D1050E94468D8AE00F900F900F900F9058
:10B7C000DF91CF911F910F91FF90EF90DF90CF907D
:10B7D000BF90AF909F908F907F906F905F904F90B1
:10B7E0003F902F900C94855160930406709305064A
:10B7F00080930606909307065ECE0F900F900F90F1
:10B800000F90DF91CF911F910F91FF90EF90DF90FC
:10B81000CF90BF90AF909F908F907F906F905F90F0
:10B820004F903F902F9008955F988A984798809105
:10B830000801817080930601479812980895CF936C
:10B84000DF9380E00E9472A9C8EBD5E0688379831A
:10B850008A839B8381E00E9472A96C837D838E839F
:10B860009F8382E00E9472A9688779878A879B8775
:10B87000DF91CF910895CF92DF92EF92FF92CF9315
:10B88000DF9320912102222309F485C0EC01C090AE
:10B89000AC05D090AD05E090AE05F090AF05A701E6
:10B8A0009601688179818A819B810E949BD587FF5F
:10B8B00004C0C882D982EA82FB82C090B005D090D1
:10B8C000B105E090B205F090B305A70196016C8137
:10B8D0007D818E819F810E949BD587FF04C0CC8291
:10B8E000DD82EE82FF82C0901502D0901602E090B9
:10B8F0001702F0901802A7019601688179818A8168
:10B900009B810E94EBDB181624F4C882D982EA825C
:10B91000FB82C0901902D0901A02E0901B02F090B6
:10B920001C02A70196016C817D818E819F810E94FE
:10B93000EBDB181624F4CC82DD82EE82FF82C0900D
:10B94000B405D090B505E090B605F090B705A70115
:10B950009601688579858A859B850E949BD587FF9E
:10B9600004C0C886D986EA86FB86C0901D02D090A6
:10B970001E02E0901F02F0902002A7019601688548
:10B9800079858A859B850E94EBDB181624F4C8868E
:10B99000D986EA86FB86DF91CF91FF90EF90DF900A
:10B9A000CF9008952F923F924F925F926F927F9225
:10B9B0008F929F92AF92BF92CF92DF92EF92FF92BF
:10B9C0000F931F93CF93DF93CDB7DEB7CC54D1093C
:10B9D0000FB6F894DEBF0FBECDBF80EE95E04BDF13
:10B9E00080914B0683FDA9C0C090EC05D090ED0579
:10B9F000E090EE05F090EF0520913504309136048B
:10BA00004091370450913804C701B6010E949BD57C
:10BA1000882309F492C080914A06811133C0609155
:10BA200043047091440480914504909146040E941F
:10BA300009DB20912B0230912C026217730714F559
:10BA4000C0923504D0923604E0923704F092380464
:10BA5000ECE7FBE184917F019FEFE91AF90A882363
:10BA600021F00E948551F701F5CFEAE6F6E18491D5
:10BA70007F01AFEFEA1AFA0A882321F00E9485516C
:10BA8000F701F5CF8090EC059090ED05A090EE05C4
:10BA9000B090EF0520913504309136044091370481
:10BAA00050913804C501B4010E94C4D96B017C01D6
:10BAB00020E030E0A9010E94EBDB87FF04C0F7FA29
:10BAC000F094F7F8F094E091C405B4E0EB9FF00136
:10BAD0001124E95DFD4F2081318142815381C701ED
:10BAE000B6010E9400D620E030E048E453E40E9412
:10BAF000EBDB181614F58092350490923604A09270
:10BB00003704B0923804ECE7FBE184917F019FEFAA
:10BB1000E91AF90A882321F00E948551F701F5CF2F
:10BB2000EBE4F6E184917F01AFEFEA1AFA0A882389
:10BB300021F00E948551F701F5CF8091FD176090AB
:10BB4000020270900302C090E005D090E105E09001
:10BB5000E205F090E3058090E4059090E505A09063
:10BB6000E605B090E705882309F481C22090FE170E
:10BB70003090FF17409000185090011820E030E0FE
:10BB8000A901C201B1010E949BD5882379F02091BF
:10BB9000E8053091E9054091EA055091EB05C201B5
:10BBA000B1010E94EBDB18160CF061C2B301770CF7
:10BBB000880B990B0E94A1D520914B0230914C0229
:10BBC00040914D0250914E020E9400D62AE037ED7E
:10BBD00043E25CE30E9400D66DA77EA78FA798ABD7
:10BBE0002091290430912A0440912B0450912C0477
:10BBF000C701B6010E94C4D92B013C0120912D043C
:10BC000030912E0440912F0450913004C501B401AD
:10BC10000E94C4D925966CAF7DAF8EAF9FAF25979C
:10BC200020E030E0A901C301B2010E949BD581113F
:10BC300041C020E030E0A90125966CAD7DAD8EAD10
:10BC40009FAD25970E949BD5811134C07090C4058B
:10BC500019AA1AAA1BAA1CAAC982DA82EB82FC8240
:10BC60008D829E82AF82B8868091E8059091E90529
:10BC7000A091EA05B091EB0589879A87AB87BC87CD
:10BC8000AE01475F5F4FBE016B5F7F4FCE010196F4
:10BC90000E94BDAEFE01F1966F01E72C8E01035D9F
:10BCA0001F4F2CEE35E0AE01475F5F4FBE016B5F6B
:10BCB0007F4F2AC2209131043091320440913304E5
:10BCC000509134046091E8057091E9058091EA058E
:10BCD0009091EB050E94C4D929966CAF7DAF8EAFD1
:10BCE0009FAF299720913504309136044091370455
:10BCF000509138046091EC057091ED058091EE054E
:10BD00009091EF050E94C4D921966CAF7DAF8EAFA4
:10BD10009FAF2197A3019201C301B2010E9400D6F7
:10BD20006B017C0125962CAD3DAD4EAD5FAD2597E9
:10BD3000CA01B9010E9400D69B01AC01C701B6013E
:10BD40000E94C5D96B017C0129962CAD3DAD4EAD4D
:10BD50005FAD2997CA01B9010E9400D69B01AC01D1
:10BD6000C701B6010E94C5D90E9430DC6B017C017D
:10BD70002DEB37E346E855E30E949BD587FF17C0BC
:10BD800020E030E0A90121966CAD7DAD8EAD9FAD78
:10BD900021970E94EBDB2196CCACDDACEEACFFAC86
:10BDA000219787FF04C0F7FAF094F7F8F0942DEB91
:10BDB00037E346E855E3C701B6010E949BD587FDEE
:10BDC000A6C120E030E040EA50E4C701B6010E947D
:10BDD000A1DA0E940EDB1B01672B19F422242394A5
:10BDE000312CB10180E090E00E949FD59B01AC0115
:10BDF00060E070E080E89FE30E94A1DA4B015C0103
:10BE00009B01AC01C701B6010E9400D62D966CAF14
:10BE10007DAF8EAF9FAF2D97A5019401C301B201F5
:10BE20000E9400D6698B7A8B8B8B9C8BA501940129
:10BE300025966CAD7DAD8EAD9FAD25970E9400D649
:10BE40006D8B7E8B8F8B988FA501940129966CAD9D
:10BE50007DAD8EAD9FAD29970E9400D6698F7A8FF8
:10BE60008B8F9C8FA501940121966CAD7DAD8EAD1D
:10BE70009FAD21970E9400D66D8F7E8F8F8F98A3E4
:10BE800080E1E9E2F4E0DE01119601900D928A95DD
:10BE9000E1F799249394F1E02F1A310809F04BC08F
:10BEA000E090C4052D968CAD9DADAEADBFAD2D9788
:10BEB00089AF9AAFABAFBCAF8091E0059091E1053F
:10BEC000A091E205B091E30589A39AA3ABA3BCA31B
:10BED0008091E4059091E505A091E605B091E70514
:10BEE0008DA39EA3AFA3B8A78091E8059091E90523
:10BEF000A091EA05B091EB0589A79AA7ABA7BCA7CB
:10BF0000AE01475D5F4FBE016B5D7F4FCE018196F5
:10BF10000E94BDAEDE01D9966D018E01035D1F4FFB
:10BF20002CEE35E0AE01475D5F4FBE016B5D7F4F8C
:10BF3000CE018196EBC08091F405811112C00E9460
:10BF400010C5DC01CB0188539F4FAF4FBF4F80938B
:10BF5000F0059093F105A093F205B093F30590924C
:10BF6000F4050E9404930E9410C5C090F005D09083
:10BF7000F105E090F205F090F305DC01CB018C199E
:10BF80009D09AE09BF09B7FD11C00E9410C5DC01B3
:10BF9000CB0188539F4FAF4FBF4F8093F0059093D5
:10BFA000F105A093F205B093F30584D86E01B1E1D9
:10BFB000CB0ED11CFE0131967F015601D6012D9189
:10BFC0003D914D915D916D01F7016081718182819B
:10BFD00093810E94C5D9D7016D937D938D939D93D5
:10BFE0007D01AA16BB0651F7E090C4052D968CADD5
:10BFF0009DADAEADBFAD2D978DAB9EABAFABB8AF2A
:10C0000089819A81AB81BC8189A39AA3ABA3BCA38C
:10C010008D819E81AF81B8858DA39EA3AFA3B8A764
:10C0200089859A85AB85BC8589A79AA7ABA7BCA74C
:10C03000AE01475D5F4FBE016B5D7F4FCE018196C4
:10C040000E94BDAEDE01D5966D018E01035D1F4FCE
:10C050009E01235F3F4FAE01475D5F4FBE016B5DA9
:10C060007F4FCE018196BAD0811115CF19CFB30180
:10C07000770C880B990B0E94A1D520914B0230912F
:10C080004C0240914D0250914E020E9400D62AE08F
:10C0900037ED43E25CE30E9400D669AB7AAB8BAB31
:10C0A0009CAB7090C4058091E8059091E905A09142
:10C0B000EA05B091EB05C982DA82EB82FC82898ABB
:10C0C0009A8AAB8ABC8A89A39AA3ABA3BCA31DA6F8
:10C0D0001EA61FA618AAAE014F5D5F4FBE016F5E80
:10C0E0007F4FCE0101960E94BDAEFE01BD966F014D
:10C0F000E72C8E010F5C1F4F2CEE35E0AE014F5D3B
:10C100005F4FBE016F5E7F4FCE01019667D080E129
:10C11000E0EEF5E0A9E2B4E001900D928A95E1F736
:10C12000C45BDF4F0FB6F894DEBF0FBECDBFDF910B
:10C13000CF911F910F91FF90EF90DF90CF90BF9024
:10C14000AF909F908F907F906F905F904F903F90B7
:10C150002F900895CF93DF93E0910218F0E0EB5811
:10C16000F94F8081882381F0E8E4F6E18491EF01C2
:10C170002196882321F00E948551FE01F7CF8AE0A5
:10C18000DF91CF910C948551DF91CF910895CF939A
:10C19000DF938091AA058093AB05EFE3F6E18491EC
:10C1A000EF012196882321F00E948551FE01F7CFEF
:10C1B0008091101890911118A0911218B091131835
:10C1C000BC01CD016F5F7F4F8F4F9F4F0E944E5537
:10C1D0008AE00E948551DF91CF91BCCF2F923F9290
:10C1E0004F925F926F927F928F929F92AF92BF9287
:10C1F000CF92DF92EF92FF920F931F93CF93DF9333
:10C20000CDB7DEB7C857D1090FB6F894DEBF0FBE61
:10C21000CDBFE0915810F0915910EF2B11F00C9414
:10C22000AE692896DFAECEAE28976E2C79016A01F2
:10C230005B01FC0120813181428153816C962CAFDE
:10C240003DAF4EAF5FAF6C9720915E1130915F11A3
:10C2500040916011509161116C966CAD7DAD8EADC9
:10C260009FAD6C970E9400D60E94F6DBE0966CAF03
:10C270007DAF8EAF9FAFE097D5018D919D910D90D1
:10C28000BC91A02DA0968CAF9DAFAEAFBFAFA097D5
:10C2900020916211309163114091641150916511A8
:10C2A000BC01CD010E9400D60E94F6DBE4966CAF83
:10C2B0007DAF8EAF9FAFE497D6012D913D914D910B
:10C2C0005C91A4962CAF3DAF4EAF5FAFA497209189
:10C2D0006611309167114091681150916911A496CF
:10C2E0006CAD7DAD8EAD9FADA4970E9400D60E942F
:10C2F000F6DBE8966CAF7DAF8EAF9FAFE897D701C6
:10C300002D913D914D915C9122962CAF3DAF4EAF5A
:10C310005FAF229720916A1130916B1140916C119F
:10C3200050916D1122966CAD7DAD8EAD9FAD229773
:10C330000E9400D60E94F6DB60966CAF7DAF8EAF98
:10C340009FAF609780914B0683FF1CC060962CAD19
:10C350003DAD4EAD5FAD609720933D0A30933E0AF0
:10C3600040933F0A5093400A22968CAD9DADAEADEE
:10C37000BFAD229780932D0A90932E0AA0932F0A87
:10C38000B093300AD801BC91B9A7F801F181F9AB9B
:10C39000D8011296BC91BEABF801F381FAAF80913F
:10C3A0000B0A90910C0A891B8F708F3019F40E9430
:10C3B0005A58F5CF00910B0AE9960FAFE997809193
:10C3C0000B0A082F10E01CA30BA38091310A909157
:10C3D000320AA091330AB091340AE0968CAC9DAC3D
:10C3E000AEACBFACE097881A990AAA0ABB0A809142
:10C3F000350A9091360AA091370AB091380AE4962E
:10C400002CAC3DAC4EAC5FACE497281A390A4A0A12
:10C410005B0A8091390A90913A0AA0913B0AB09147
:10C420003C0AE8962CAD3DAD4EAD5FADE897281BBC
:10C43000390B4A0B5B0B2DA33EA34FA358A780914A
:10C440003D0A90913E0AA0913F0AB091400A609641
:10C450000CAD1DAD2EAD3FAD6097081B190B2A0B1F
:10C460003B0B0DA71EA72FA738AB012B022B032BCD
:10C4700009F4BCC080914A0681114BC0609143040D
:10C480007091440480914504909146040E9409DB18
:10C4900020912B0230912C02621773070CF039C0E7
:10C4A00060962CAD3DAD4EAD5FAD609720933D0ADB
:10C4B00030933E0A40933F0A5093400A22968CAD37
:10C4C0009DADAEADBFAD229780932D0A90932E0AFD
:10C4D000A0932F0AB093300AECE7FBE184918F011F
:10C4E0000F5F1F4F811103C0E5ECF7E104C00E940C
:10C4F0008551F801F3CF84918F010F5F1F4F88237F
:10C5000021F00E948551F801F6CF1DA61EA61FA698
:10C5100018AA94E0699E80011124095D1D4F6DA544
:10C520007EA58FA598A90E94A1D5D8012D913D91F6
:10C530004D915C910E9400D66B017C0120E030E0BF
:10C54000A9010E94EBDB87FF04C0F7FAF094F7F82B
:10C55000F09460916A1170916B1180916C119091BF
:10C560006D110E9409DB9B01AC01A8ECB0E00E94B8
:10C57000ABD90E94A1D5A70196010E949BD587FF48
:10C5800039C060960CAD1DAD2EAD3FAD60970093E8
:10C590003D0A10933E0A20933F0A3093400A2296A8
:10C5A0002CAD3DAD4EAD5FAD229720932D0A30935B
:10C5B0002E0A40932F0A5093300AECE7FBE1849156
:10C5C0008F010F5F1F4F811103C0E6EAF7E104C03E
:10C5D0000E948551F801F3CF84918F010F5F1F4FA7
:10C5E000882321F00E948551F801F6CF1DA61EA6D2
:10C5F0001FA618AAD501C4018827B7FD83959927DE
:10C60000AA27BB27782E57FE03C0382F3260732E1F
:10C610008DA19EA1AFA1B8A5B7FF03C0972D9460CF
:10C62000792E0DA51EA52FA538A937FF03C0172DFC
:10C630001860712E24E0629E80011124095D1D4F57
:10C640006DA57EA58FA598A90E94A1D5D8012D9191
:10C650003D914D915C910E9400D66B017C0120E0E0
:10C6600030E0A9010E94EBDB87FF04C0C701B601DF
:10C67000905802C0C701B60120E030E040E05FE31F
:10C680000E94C5D90E940EDB6AAB7BAB8CAB9DAB25
:10C6900088E60BA11CA1809FF001819FF00D112461
:10C6A000E259FE4E1082EA5BFF4F7082B501A40191
:10C6B000B7FE07C044275527BA01481959096A0926
:10C6C0007B0988E60BA11CA1809FF001819FF00DE2
:10C6D0001124E259FE4E458B568B678B708F2C963A
:10C6E0002CAE3DAE4EAE5FAE2C9757FE0DC08827E8
:10C6F0009927DC0182199309A409B5092C968CAFFE
:10C700009DAFAEAFBFAF2C9728E60BA11CA1209F19
:10C71000F001219FF00D1124E259FE4E2C968CADB4
:10C720009DADAEADBFAD2C97818F928FA38FB48F8F
:10C730000DA11EA12FA138A537FF07C03095209568
:10C74000109501951F4F2F4F3F4FE8E67E2EABA16E
:10C75000BCA17A9EF0017B9EF00D1124E259FE4EA1
:10C76000058F168F278F30A38AA99BA9ACA9BDA9D5
:10C7700081A392A3A3A3B4A323964FAF2397752EAF
:10C78000F62FE72F2C968CAD9DADAEADBFAD2C979F
:10C79000481759076A077B0778F429969FAD2997B0
:10C7A00023969FAF23972A967FAC2A972B96FFADAF
:10C7B0002B972C96EFAD2C9723968FAD2397972D23
:10C7C000AF2FBE2F80179107A207B30710F4D9012E
:10C7D000C8010AA91BA92CA93DA980179107A20786
:10C7E000B30710F4D901C80128E60BA11CA1209FB2
:10C7F000F001219FF00D1124E259FE4E85A396A36E
:10C80000A7A3B0A70697A105B10508F4A0C5DF014D
:10C81000AE59BF4F8091390490913A048D939C9307
:10C8200061A6452B462B472B09F05F9888E60BA1A4
:10C830001CA1809FF001819FF00D1124E259FE4E52
:10C84000818D928DA38DB48D892B8A2B8B2B11F02A
:10C850008A98479888E60BA11CA1809FF001819FD0
:10C86000F00D1124E259FE4E858D968DA78DB0A155
:10C87000892B8A2B8B2B31F080910801817080935A
:10C88000060147982AA93BA94CA95DA9232B242B73
:10C89000252B09F465C580915006882319F0815035
:10C8A00080935006611004C0129880E28093500675
:10C8B0006090460670904706009148061091490620
:10C8C0009301A80169A579A98EA99AAD0E949BD56B
:10C8D00087FF04C069A679AA0EAB1AAFC501B401DF
:10C8E0000E94A1D520914E1130914F1140915011CD
:10C8F000509151110E9400D626966CAF7DAF8EAF3D
:10C900009FAF2697698B7A8B8B8B9C8BC201B10171
:10C910000E94A1D520915211309153114091541190
:10C92000509155110E9400D62B013C016D8B7E8BDE
:10C930008F8B988F6DA17EA18FA198A50E94A1D504
:10C940002091561130915711409158115091591121
:10C950000E9400D64B015C01698F7A8F8B8F9C8F70
:10C9600020915A1130915B1140915C1150915D11F1
:10C97000C701B6010E9400D66B017C016D8F7E8FCE
:10C980008F8F98A388E60BA11CA1809FF001819F47
:10C99000F00D1124E259FE4E258936894789508DC4
:10C9A0002DA33EA34FA358A72630310541055105BD
:10C9B00008F4DFC42896AEADBFAD2897CD90DD90CA
:10C9C000ED90FC9020E030E0A901C701B6010E9483
:10C9D0009BD58111EDC426962CAD3DAD4EAD5FAD1E
:10C9E0002697CA01B9010E9400D66B017C01A30100
:10C9F0009201C301B2010E9400D69B01AC01C701A4
:10CA0000B6010E94C5D96B017C01A5019401C50145
:10CA1000B4010E9400D69B01AC01C701B6010E947F
:10CA2000C5D90E9430DC28E60BA11CA1209FF00193
:10CA3000219FF00D1124E259FE4E65877687878786
:10CA4000908B88E60BA11CA1809FF001819FF00DC7
:10CA50001124E259FE4E4584568467847088A301F0
:10CA6000920160E070E080E89FE30E94A1DA6496A2
:10CA70006CAF7DAF8EAF9FAF649729A539A94EA942
:10CA80005AAD0E9400D64B015C0180910B0A909137
:10CA9000090A891B8F7027968FAF2797A5019401EC
:10CAA00060E074E284E799E40E94A1DA0E94F6DB78
:10CAB0006B017C0127968FAD27978250863008F452
:10CAC00086C4A5019401C301B2010E9400D69B0156
:10CAD000AC010E9400D668966CAF7DAF8EAF9FAF61
:10CAE000689788E6ABA1BCA18A9F80018B9F100D3F
:10CAF000112402591E4E68962CAD3DAD4EAD5FAD72
:10CB00006897D80111962D933D934D935C9314979C
:10CB100095962D913D914D915C9198972EAB3FABA1
:10CB200048AF59AFCA01B9010E949FD56AAF7BAF28
:10CB30008CAF9DAF9B01AC01C501B4010E9400D632
:10CB40000E948BDA0E940EDBA8966CAF7DAF8EAF91
:10CB50009FAFA897F801EE5AFF4F608371838283DD
:10CB600093838E010F5E1F4F2A961FAF0EAF2A9739
:10CB70000051110924961FAF0EAF24970EE216E064
:10CB8000AC961FAF0EAFAC978E010F5D1F4F1AA36F
:10CB900009A324960EAD1FAD2497AA961FAF0EAF22
:10CBA000AA97312C212C10E819A70FE309AB2A967C
:10CBB000AEADBFAD2A972D913D914D915D912A96D5
:10CBC000BFAFAEAF2A97C501B4010E9400D66B017A
:10CBD0007C01AA96EEADFFADAA9761937193819304
:10CBE0009193AA96FFAFEEAFAA9720E030E0A9019B
:10CBF0000E94EBDB87FF04C0F7FAF094F7F8F0949B
:10CC0000AC96AEADBFADAC974D905D906D907D9004
:10CC1000AC96BFAFAEAFAC97A7019601C301B2010E
:10CC20000E949BD587FD0DC409A11AA12A962EAD9D
:10CC30003FAD2A970217130709F0B9CF20E030E083
:10CC400040E85FE3632D722D89A599A90E949BD5C9
:10CC500087FF58C07E0131E1E30EF11C24960EAD32
:10CC60001FAD2497232D322D49A559A9D8016D91C7
:10CC70007D918D919C910E9400D6F80161937193F2
:10CC8000819391938F01EE16FF0661F728E60BA1C1
:10CC90001CA1209FC001219F900D11249C012259AD
:10CCA0003E4E790189010E5A1F4FA8966CAD7DAD9D
:10CCB0008EAD9FADA8970E949FD5232D322D49A5FB
:10CCC00059A90E9400D60E940EDBD8016D937D9376
:10CCD0008D939C931397232D322D49A559A9632D2C
:10CCE000722D89A599A90E9400D668962CAD3DADFC
:10CCF0004EAD5FAD68970E9400D6F70161837283E5
:10CD0000838394832AAD3BAD4CAD5DAD64966CAD31
:10CD10007DAD8EAD9FAD64970E9400D669A77AA7BE
:10CD20008BA79CA70DA11EA12FA138A5012B022B1B
:10CD3000032B09F09EC388E62BA13CA1829F8001B2
:10CD4000839F100D112402591E4EF801818D928D82
:10CD5000A38DB48D892B8A2B8B2B09F08AC3858DEB
:10CD6000968DA78DB0A1892B8A2B8B2B09F081C3BF
:10CD700020912A0630912B0640912C0650912D06C9
:10CD800069A57AA58BA59CA50E9400D60E948BDA86
:10CD90000E940EDB2B013C01F801E95BFF4F108282
:10CDA00088E62BA13CA1829F8001839F100D112456
:10CDB00002591E4EF801E25AFF4F408251826282B0
:10CDC0007382C301B2010E949FD529A53AA54BA544
:10CDD0005CA50E94A1DA6AAF7BAF8CAF9DAFD80192
:10CDE00051966D937D938D939C935497F801E95BD5
:10CDF000FF4F8081882381F17801B8E4EB0EF11CAC
:10CE0000379620911E0630911F06409120065091C2
:10CE1000210660817181828193810E9400D62AADB2
:10CE20003BAD4CAD5DAD0E9400D620916A113091B2
:10CE30006B1140916C1150916D110E9400D69B01B5
:10CE4000AC0160E074E284EF99E40E94A1DA0E94F0
:10CE50000EDBF7017183608388E60BA11CA1809F24
:10CE6000F001819FF00D1124E259FE4E21813281A3
:10CE7000438154812C962CAF3DAF4EAF5FAF2C97C2
:10CE8000CA01B9010E9430DC362E272E8C014EE0FB
:10CE900056E062965FAF4EAF62973E0151E1650E7C
:10CEA000711C8EE096E09FAB8EAB24964EAC5FACCF
:10CEB00024973DA62DA209A719AB1AAAD201CD909D
:10CEC000DD90ED90FD902D0120E030E0A901C7013B
:10CED000B6010E94EBDB87FF04C0F7FAF094F7F885
:10CEE000F094EEA9FFA981909190A190B190FFAB31
:10CEF000EEABA7019601C501B4010E949BD587FD49
:10CF0000D8C564147504D1F627965FAD27975523CD
:10CF100009F448C6C0900D0AD0900E0AE0900F0A9E
:10CF2000F090100A2DEB37E346E855E3C701B60150
:10CF30000E949BD587FD36C6C701B6010E9430DC32
:10CF40006B017C019B01AC01632D722DC8010E9415
:10CF50009BD587FD03C03C2C2D2C87019601A70192
:10CF6000632D722DC8010E94A1DA68966CAF7DAF67
:10CF70008EAF9FAF689781E19AE028969FAF8EAF02
:10CF8000289720E030E040E85FE32AAB3BAB4CABB6
:10CF90005DAB1EAA2896AEADBFAD28972D913D91F1
:10CFA0004D915D912896BFAFAEAF289768966CAD56
:10CFB0007DAD8EAD9FAD68970E9400D64B015C01A0
:10CFC0002496EEADFFAD2497C190D190E190F19001
:10CFD0002496FFAFEEAF2497FEA9FF2391F02AA974
:10CFE0003BA94CA95DA90E9400D64B015C012AA96E
:10CFF0003BA94CA95DA9C701B6010E9400D66B01EF
:10D000007C01A7019601C501B4010E94EBDB20E081
:10D0100030E0A90118160CF092C5C701B6010E94B4
:10D02000EBDB18160CF486C520E030E0A901C50141
:10D03000B4010E949BD587FD7DC52601370177FA93
:10D04000709477F87094A3019201C501B4010E9415
:10D05000EBDB181614F4240135016296AEADBFADBA
:10D060006297CD90DD90ED90FD906296BFAFAEAF30
:10D070006297A3019201C701B6010E949BD587FF69
:10D0800015C0A3019201C701B6010E94A1DA9B015C
:10D09000AC016AA97BA98CA99DA90E9400D66AABA4
:10D0A0007BAB8CAB9DABBEA9BF5FBEABE1E2FAE050
:10D0B00028962EAD3FAD2897E217F30709F06ACF07
:10D0C0003EA9332361F02AA93BA94CA95DA9632D90
:10D0D000722DC8010E9400D6362E272E8C0124EA1C
:10D0E00030E74DE75FE3632D722DC8010E9400D643
:10D0F0006B017C0120914C0630914D0640914E060B
:10D1000050914F060E949BD587FD42C58DA59DA1DC
:10D11000A9A5B9A980934C0690934D06A0934E06FD
:10D12000B0934F0628E64BA15CA1249FC001259F28
:10D13000900D1124DC01A259BE4E7D01232D322D0C
:10D14000A801632D722DC8010E9400D6F7016187E6
:10D150007287838794876AAD7BAD8CAD9DAD905807
:10D160009B01AC010E94C5D9D7011D962D913D911F
:10D170004D915C9150970E9400D69B01AC016BE0F1
:10D1800077ED83E29BE30E94C4D99B01AC018BE065
:10D1900097EDA3E2BBE3F70185839683A783B0876E
:10D1A00010812C966CAD7DAD8EAD9FAD2C970E94FD
:10D1B0009BD518160CF4FBC483E0182B88E62BA132
:10D1C0003CA1829FF001839FF00D1124E259FE4E95
:10D1D000108380E1FE013196A1E1BAE001900D9249
:10D1E0008A95E1F72C968CAD9DADAEADBFAD2C9779
:10D1F00080930D0A90930E0AA0930F0AB093100A21
:10D20000E0960CAD1DAD2EAD3FADE0970093310A19
:10D210001093320A2093330A3093340AE4962CADEB
:10D220003DAD4EAD5FADE4972093350A3093360A9D
:10D230004093370A5093380AE8968CAD9DADAEAD59
:10D24000BFADE8978093390A90933A0AA0933B0ABE
:10D25000B0933C0A60960CAD1DAD2EAD3FAD60970E
:10D2600000933D0A10933E0A20933F0A3093400AF0
:10D270006C962CAD3DAD4EAD5FAD6C972093210A01
:10D280003093220A4093230A5093240AA0968CAD2F
:10D290009DADAEADBFADA0978093250A9093260AB1
:10D2A000A093270AB093280AA4960CAD1DAD2EAD0D
:10D2B0003FADA4970093290A10932A0A20932B0AC2
:10D2C00030932C0A22962CAD3DAD4EAD5FAD22972A
:10D2D00020932D0A30932E0A40932F0A5093300A40
:10D2E00090910B0A80910C0A981303C084E68093F6
:10D2F000080AE9968FADE9978F5F8F7080930B0ACC
:10D3000080910B0A90910A0A81508F70891351C441
:10D3100010910C0A1BA300910B0A0DA728E61BA174
:10D320000DA51013D1C4812C912CA12CB12C1DA2C0
:10D3300019A619AA1EAE212C312C00E010E02DA553
:10D340003BA12313CEC42114310409F07FC5809181
:10D350006F00826080936F0081E0ECC680E0EAC6D7
:10D360006090420670904306009144061091450675
:10D37000A7CA818D928DA38DB48D0697A105B105A5
:10D3800008F018CB858D968DA78DB0A10697A105C5
:10D39000B10508F00FCB20E030E0A901C701B601CC
:10D3A0000E94EBDB87FF04C0F7FAF094F7F8F094E3
:10D3B00088E60BA11CA1809FF001819FF00D112434
:10D3C000E259FE4EC586D686E786F08A3ACB809132
:10D3D0003E0690913F06A0914006B0914106C816C6
:10D3E000D906EA06FB0608F06CCB8C199D09AE093C
:10D3F000BF09BC01CD01660F771F881F991F2796B3
:10D400004FAD2797042F10E020E030E0A9019801EC
:10D410000E9489D9CA01B9010E949FD50E94F6DBFA
:10D420006C0D7D1D8E1D9F1D0E949FD59B01AC0123
:10D4300060E074E284E799E40E94A1DA4B015C01A8
:10D4400040CBA7019601C301B2010E94A1DA7B0182
:10D450008C019B01AC01632D722D89A599A90E94B5
:10D46000EBDB18160CF0E0CB3E2C2F2C09A719ABE8
:10D47000DBCB0AA91BA92CA93DA9012B022B032B4D
:10D4800049F02091260630912706409128065091B8
:10D49000290608C0209122063091230640912406D7
:10D4A0005091250669A57AA58BA59CA50E9400D65A
:10D4B0000E948BDA0E940EDB2B013C012AA93BA9BA
:10D4C0004CA95DA9232B242B252BC9F020E030E0AB
:10D4D000A90160911E0670911F068091200690910F
:10D4E00021060E949BD5882351F081E00DA51EA541
:10D4F0002FA538A910161106120613060CF080E0AD
:10D5000098E62BA13CA1929F8001939F100D1124BE
:10D5100002591E4E180137E4230E311CD1018C93A1
:10D52000882309F4B3C02091210A3091220A409146
:10D53000230A5091240A6C966CAD7DAD8EAD9FADE3
:10D540006C970E94C4D96DA77EA78FA798AB209136
:10D55000250A3091260A4091270A5091280AA09660
:10D560006CAD7DAD8EAD9FADA0970E94C4D94B012F
:10D570005C012091290A30912A0A40912B0A50918E
:10D580002C0AA4966CAD7DAD8EAD9FADA4970E9484
:10D59000C4D96B017C012DA53EA54FA558A9CA0190
:10D5A000B9010E9400D66DA77EA78FA798ABA501F1
:10D5B0009401C501B4010E9400D69B01AC016DA588
:10D5C0007EA58FA598A90E94C5D94B015C01A70132
:10D5D0009601C701B6010E9400D69B01AC01C501AE
:10D5E000B4010E94C5D90E9430DC6B017C012091FE
:10D5F0002D0A30912E0A40912F0A5091300A22961E
:10D600006CAD7DAD8EAD9FAD22970E94C4D9A701B0
:10D6100096010E94A1DA6B017C01F801E25BFF4FE9
:10D62000608371838283938320E030E040E450E4A0
:10D630000E94EBDB18161CF4F101108227C0209128
:10D640001E0630911F064091200650912106C70109
:10D65000B6010E9400D69B01AC0160911A06709140
:10D660001B0680911C0690911D060E94A1DA29A537
:10D670003AA54BA55CA50E9400D60E940EDB64155E
:10D6800075058605970510F42B013C0180912A1140
:10D6900090912B11A0912C11B0912D110EA91FA9C1
:10D6A00028AD39AD80179107A207B30708F4DFC092
:10D6B0002DA13EA14FA158A5232B242B252B41F1B1
:10D6C00060912E1170912F11809130119091311134
:10D6D0006415750586059705D8F42EA93FA948ADB0
:10D6E00059AD0E947AD96B017C012DA13EA14FA1B9
:10D6F00058A5C301B2010E947AD9C616D706E8061A
:10D70000F90630F4C701B6010E9489D929013A010E
:10D7100088E60BA11CA1809FF001819FF00D1124D0
:10D72000E259FE4EC18CD28CE38CF48CC114D1042E
:10D73000E104F10431F16091321170913311809163
:10D740003411909135116415750586059705C8F457
:10D750002EA93FA948AD59AD0E947AD94B015C0171
:10D76000A7019601C301B2010E947AD986169706D5
:10D77000A806B90630F4C501B4010E9489D929016F
:10D780003A0188E60BA11CA1809FF001819FF00D5A
:10D790001124E259FE4EC58CD68CE78CF0A0C11442
:10D7A000D104E104F10431F1609136117091371127
:10D7B000809138119091391164157505860597058A
:10D7C000C8F42EA93FA948AD59AD0E947AD94B01A2
:10D7D0005C01A7019601C301B2010E947AD98616A5
:10D7E0009706A806B90630F4C501B4010E9489D98C
:10D7F00029013A0188E60BA11CA1809FF001819FBD
:10D80000F00D1124E259FE4EC1A0D2A0E3A0F4A075
:10D81000C114D104E104F10409F4C2CA60913A11BF
:10D8200070913B1180913C1190913D1164157505EB
:10D830008605970508F0B4CA2EA93FA948AD59AD91
:10D840000E947AD94B015C01A7019601C301B20184
:10D850000E947AD986169706A806B90608F0A0CACB
:10D86000C501B4010E9489D929013A0199CA2DA1A3
:10D870003EA14FA158A5232B242B252BC9F1609144
:10D880002E1170912F1180913011909131116415EA
:10D8900075058605970560F50E949FD52AAD3BADBD
:10D8A0004CAD5DAD0E9400D66B017C016DA17EA1E7
:10D8B0008FA198A50E949FD54B015C01C301B201C5
:10D8C0000E949FD5A50194010E9400D69B01AC0146
:10D8D000C701B6010E949BD587FF0AC0A50194012C
:10D8E000C701B6010E94A1DA0E940EDB2B013C01A8
:10D8F00088E60BA11CA1809FF001819FF00D1124EF
:10D90000E259FE4E818C928CA38CB48C81149104CC
:10D91000A104B104B9F16091321170913311809179
:10D92000341190913511641575058605970550F5EC
:10D930000E949FD52AAD3BAD4CAD5DAD0E9400D697
:10D940006B017C01C501B4010E949FD54B015C01B4
:10D95000C301B2010E949FD5A50194010E9400D687
:10D960009B01AC01C701B6010E949BD587FF0AC08D
:10D97000A5019401C701B6010E94A1DA0E940EDB45
:10D980002B013C0188E60BA11CA1809FF001819F27
:10D99000F00D1124E259FE4E858C968CA78CB0A018
:10D9A00081149104A104B104B9F160913611709110
:10D9B00037118091381190913911641575058605DC
:10D9C000970550F50E949FD52AAD3BAD4CAD5DAD9E
:10D9D0000E9400D66B017C01C501B4010E949FD555
:10D9E0004B015C01C301B2010E949FD5A5019401C6
:10D9F0000E9400D69B01AC01C701B6010E949BD5D5
:10DA000087FF0AC0A5019401C701B6010E94A1DAEF
:10DA10000E940EDB2B013C0188E60BA11CA1809F1C
:10DA2000F001819FF00D1124E259FE4EC1A0D2A059
:10DA3000E3A0F4A0C114D104E104F10409F4B0C9D5
:10DA400060913A1170913B1180913C1190913D1180
:10DA5000641575058605970508F0A2C90E949FD533
:10DA60002AAD3BAD4CAD5DAD0E9400D64B015C01D3
:10DA7000C701B6010E949FD56B017C01C301B201B1
:10DA80000E949FD5A70196010E9400D69B01AC0180
:10DA9000C501B4010E949BD587FF82C9A7019601E9
:10DAA000C501B4010E94A1DA0E940EDB2B013C01EA
:10DAB00077C9FAA9FF2331F1A5019401632D722DD5
:10DAC000C8010E9400D64B015C012DA53DA149A5CE
:10DAD00059A9C701B6010E9400D69B01AC01C5013E
:10DAE000B4010E949BD587FF22C0A7019601C50102
:10DAF000B4010E94A1DA6DA77DA389A799AB21E0AB
:10DB00002AABFFC9A7019601C501B4010E94A1DAA1
:10DB10009B01AC016DA57DA189A599A90E9400D6A4
:10DB20006DA77DA389A799AB31E03AABEAC941E083
:10DB30004AABE7C9A7019601C501B40113C0C701EB
:10DB4000B6010E949BD587FD09C020E030E0A90105
:10DB5000C501B4010E94EBDB18164CF4A501940139
:10DB6000C701B6010E94C4D92B013C0176CA240129
:10DB7000350177FA709477F87094A3019201C70188
:10DB8000B6010E949BD587FD68CA2601370165CA88
:10DB90002DA53DA149A559A9C701B6010E949BD554
:10DBA00087FFB4CA3DA42DA009A519A9AFCA81E079
:10DBB00004CBF0900B0A8FEF8F0D8F708BA3B0907A
:10DBC0000A0A80910B0AB81609F454C0C12CD12C52
:10DBD0000BA10B1509F44EC0602E712C28E6269D72
:10DBE0008001279D100D112402591E4ED8018C91E1
:10DBF00083FD2BC00EAF1AAB0115110541F119962B
:10DC0000BC91BDA7F801F285FDA3D8011B96BC917C
:10DC1000B9A7F801F485F9ABD80115962D903D9080
:10DC20004D905C901897A20191016DA57DA189A5E9
:10DC30009F2F0E949BD5811186C1C114D10439F058
:10DC4000F601808180FD7FC102C0CEAEDAAA8BA131
:10DC500081508F708BA380910A0A8B1103C0CEACC8
:10DC6000DAA8B6CF0BA10B1529F081E08B0D8F70D0
:10DC7000B82EF1CF10910A0A1BA3C12CD12C809190
:10DC80000B0A0BA1801709F443CB802E912C28E6B8
:10DC9000289D8001299D100D112402591E4ED80186
:10DCA0008C9183FD0AC05801C114D10439F0C6011A
:10DCB0000E947C96811102C0C5C156018BA18F5F65
:10DCC0008F708BA36501DBCF802F81508F70289FD1
:10DCD000F0011124E259FE4E908193FF24CB8DA7D1
:10DCE0001ECB48E6439FC0011124DC01A259BE4E61
:10DCF0001D018C9183FD19C015966D917D918D91BB
:10DD00009C9118970E9430DCF62EE72ED82EC92E53
:10DD10000115110509F48CC0F801808180FD0AC04D
:10DD2000D1018C9180FD06C083C0FDA0E9A4D9A8D3
:10DD3000CEAC83C0F801808181608083C8010E94DD
:10DD40007C96811171C0F801618172818381948117
:10DD50000E9430DC2B013C019B01AC0160E070E0D3
:10DD600080E89FE30E94A1DA4B015C019B01AC01BA
:10DD70006F2D7E2D8D2D9C2D0E9400D669837A8378
:10DD80008B839C832DA139A549A95EADC501B40142
:10DD90000E9400D6698B7A8B8B8B9C8BAE014F5F78
:10DDA0005F4FBE016F5E7F4FC8010E9442AAF8011B
:10DDB000E95BFF4F80818823B9F120911E063091E5
:10DDC0001F0640912006509121063796608171818F
:10DDD000828193810E9400D620916A1130916B114B
:10DDE00040916C1150916D110E9400D64B015C0165
:10DDF0009B01AC01C301B2010E9400D60E940EDB60
:10DE0000F801E65BFF4F71836083A50194016F2DDC
:10DE10007E2D8D2D9C2D0E9400D60E940EDBF801D8
:10DE2000E45BFF4F71836083D8018C918E7F8C936C
:10DE30008F2C9E2CAD2CBC2C81018BA18F5F8F7001
:10DE40008BA3FDA2E9A6D9AACEAE79CAF101808141
:10DE500081608083C8010E947C9681116FC0D101CE
:10DE600011966D917D918D919C9114970E9430DC5B
:10DE70006B017C019B01AC0160E070E080E89FE3F6
:10DE80000E94A1DA2B013C012DEC3CEC4CE45DE35B
:10DE90000E9400D669837A838B839C839401A501B9
:10DEA000C301B2010E9400D6698B7A8B8B8B9C8B4D
:10DEB000AE014F5F5F4FBE016F5E7F4FC1010E9499
:10DEC00042AAF101E95BFF4F80818823B9F12091DB
:10DED0001E0630911F06409120065091210637966C
:10DEE00060817181828193810E9400D620916A11A4
:10DEF00030916B1140916C1150916D110E9400D6C0
:10DF00004B015C019B01AC01C701B6010E9400D628
:10DF10000E940EDBF101E65BFF4F718360832DEC05
:10DF20003CEC4CE45DE3C501B4010E9400D60E94C4
:10DF30000EDBF101E45BFF4F71836083F1018081AF
:10DF40008E7F808304CA28E6269DF001279DF00D70
:10DF50001124E259FE4E808181FD43C0C114D104D9
:10DF600041F0D6011596CD90DD90ED90FC9018977C
:10DF700008C08BE0C82E87EDD82E83E2E82E8BE315
:10DF8000F82EB8E6B69DF001B79DF00D1124E259C8
:10DF9000FE4E81899289A389B489BC01CD01905834
:10DFA0009B01AC010E94C5D9F801258536854785BE
:10DFB00050890E9400D69B01AC01C701B6010E94A6
:10DFC000C4D9E62E872E982EA92E262F372F482F1C
:10DFD000592F6DA57DA189A599A90E949BD587FF81
:10DFE00004C0EDA48DA099A4A9A82E2D382D492DEB
:10DFF0005A2DC201B1010E949BD5882309F427CE76
:10E00000F8E6F69DC001F79D900D11249C01225960
:10E010003E4E6901D9018C9181608C93C8010E94A8
:10E020007C96882329F0F60180818E7F80830FCE35
:10E030008E2D982DA92DBA2DF60185839683A78361
:10E04000B08705CED6018C9181FD52C0D6011596C0
:10E050002D913D914D915C9118972DA73EA74FA70B
:10E0600058AB1501B5E02B0E311CF80145805680E8
:10E0700067807084A30192016DA57EA58FA598A9E4
:10E080000E949BD587FF34C0F60181899289A389BC
:10E09000B489BC01CD0190589B01AC010E94C5D947
:10E0A000D6011D962D913D914D915C9150970E9406
:10E0B00000D69B01AC016DA57EA58FA598A90E94F5
:10E0C000C4D96B017C019B01AC01C301B2010E9468
:10E0D000EBDB18166CF4D8018C9181608C93C50130
:10E0E0000E947C968823E1F0F80180818E7F8083F6
:10E0F00018E6189DF001199DF00D1124E259FE4E0D
:10E100002185328543855485658176818781908517
:10E110000E949BD58111D2CD0BA100930A0ACECDCE
:10E12000D101CD92DD92ED92FC9213970BA1009359
:10E130000A0ADECFC858DF4F0FB6F894DEBF0FBE15
:10E14000CDBFDF91CF911F910F91FF90EF90DF90A6
:10E15000CF90BF90AF909F908F907F906F905F9087
:10E160004F903F902F90089580910B0A90910C0A48
:10E17000891B8F708F3019F40E945A58F5CF809107
:10E180000B0A8F5F8F70E0910B0A98E69E9FF0015B
:10E190001124E259FE4EDF011D929A95E9F798E0AD
:10E1A00090834091310A5091320A6091330A709104
:10E1B000340A458B568B678B708F4091350A50918E
:10E1C000360A6091370A7091380A418F528F638FF7
:10E1D000748F4091390A50913A0A60913B0A7091CC
:10E1E0003C0A458F568F678F70A340913D0A50912E
:10E1F0003E0A60913F0A7091400A41A352A363A373
:10E2000074A320910B0A90910C0A291303C094E681
:10E210009093080A80930B0A80916F00826080932C
:10E220006F00089590910B0A80910C0A981306C014
:10E230008091581090915910892B19F00E945A58CA
:10E24000F1CF0895CF93DF9381E50E942051882379
:10E25000C1F080910C0490910D04009739F04AE0D0
:10E2600050E060E070E00E941AD403C060E070E00B
:10E27000CB0160933E0670933F06809340069093D7
:10E28000410683E50E942051882351F00E94E95005
:10E29000609346067093470680934806909349061C
:10E2A00084E50E942051882351F00E94E950609338
:10E2B000420670934306809344069093450688E592
:10E2C0000E942051882351F00E94E95060930E066D
:10E2D00070930F06809310069093110689E50E94B3
:10E2E0002051882351F00E94E950609312067093E8
:10E2F000130680931406909315068AE50E94205118
:10E300008823E9F00E94E95060931606709317067F
:10E3100080931806909319062DEC3CEC4CEC5DE3D1
:10E320000E949BD518165CF0EEE8F8E18491EF01AD
:10E330002196882321F00E948551FE01F7CF85E4C4
:10E340000E942051882351F00E94E95060931A06E0
:10E3500070931B0680931C0690931D06DF91CF914E
:10E360000895FF920F931F93CF93DF93F82E092FF9
:10E37000162FE9E8F8E18491EF012196882321F036
:10E380000E948551FE01F7CFEF2DF02F8491EF0110
:10E390002196882321F00E948551FE01F7CFE7E8FE
:10E3A000F8E18491EF012196882321F00E948551A4
:10E3B000FE01F7CF612F70E080E090E00E944E55A3
:10E3C0008AE0DF91CF911F910F91FF900C948551BE
:10E3D0004F925F926F927F928F929F92AF92BF9275
:10E3E000CF92DF92EF92FF92CF93DF9320910E04B2
:10E3F00030910F0440911004509111046091290450
:10E4000070912A0480912B0490912C040E94C5D90C
:10E41000AB01BC0184E898E10E942BB72091120463
:10E4200030911304409114045091150460912D040F
:10E4300070912E0480912F04909130040E94C5D9D0
:10E44000AB01BC0180E898E10E942BB72091160433
:10E4500030911704409118045091190460913104CF
:10E460007091320480913304909134040E94C5D994
:10E47000AB01BC018CE798E10E942BB740913504B9
:10E4800050913604609137047091380488E798E120
:10E490000E942BB780916F00982F927081FF05C06A
:10E4A00080916F008D7F80936F0040902510509079
:10E4B000261060902710709028108090291090905E
:10E4C0002A10A0902B10B0902C10C0902D10D0903E
:10E4D0002E10E0902F10F0903010992329F08091A9
:10E4E0006F00826080936F00EEE6F8E18491EF01A7
:10E4F0002196882321F00E948551FE01F7CFC301A8
:10E50000B2010E944E55EAE6F8E18491EF012196AE
:10E51000882321F00E948551FE01F7CFC501B40187
:10E520000E944E55E6E6F8E18491EF01219688239A
:10E5300021F00E948551FE01F7CFC701B6010E946C
:10E540004E558AE0DF91CF91FF90EF90DF90CF9012
:10E55000BF90AF909F908F907F906F905F904F9003
:10E560000C9485512F923F924F925F926F927F92BF
:10E570008F929F92AF92BF92CF92DF92EF92FF92D3
:10E580000F931F93CF93DF93CDB7DEB762970FB68C
:10E59000F894DEBF0FBECDBF80914B0683FDA4C1B2
:10E5A00083E50E9469518C87811106C082E50E9433
:10E5B0006951882309F498C10E94E9500E9409DB3F
:10E5C0006E3671050CF08DC170933C0460933B0472
:10E5D0000E94008E0E94E95020E030E040EA50E4C2
:10E5E0000E94EBDB181614F40E940D90EAE5F8E1A6
:10E5F0008491FB83EA83882371F0082E000C990B29
:10E600000E9488874A815B814F5F5F4F5B834A83AB
:10E61000FA018491F0CF8DE090E00E9488878AE033
:10E6200090E00E94888781E0809334021092C505B3
:10E630008091C40580935C101A821B821C821D820B
:10E64000188619861A861B8619821D86FCE3FE87AA
:10E650002CE12F8736E4388B312C212C40E8498B74
:10E660005FEB5A8B812C912C540160913B0470918B
:10E670003C04072E000C880B990B0E94A1D57B014E
:10E680008C019B01AC01632D722D89899A890E94AE
:10E690009BD5882341F120913D0430913E04409167
:10E6A0003F04509140048C85B70181110CC0C80112
:10E6B0000E949BD5881F8827881F89833E2C2F2C7A
:10E6C000098B1A8B10C0C8010E949BD587FF06C01A
:10E6D000EEE5F8E18491FB83EA83E7C03E2C2F2C22
:10E6E000098B1A8B19820E9410C56B017C01DC0119
:10E6F000CB01288539854A855B85821B930BA40B4A
:10E70000B50BB7FD3BC0D701C60188519C4FAF4F39
:10E71000BF4F88879987AA87BB870E94468DE2E60C
:10E72000F8E184913F019FEF691A790A882321F06B
:10E730000E948551F301F5CF81149104A104B10425
:10E74000B9F0D501C401805F984DAF4FBF4FBC01F8
:10E75000CD016C197D098E099F0928EE33E040E058
:10E7600050E00E9489D9CA01B9010E944E5503C0E8
:10E770008FE30E9485518AE00E9485510E945A5879
:10E780000E9410C56093C6057093C7058093C805A5
:10E790009093C905A0913D04AE83B0913E04BF8320
:10E7A00000913F04109140040E94D3302E813F819C
:10E7B000A801632D722D89899A890E94C4D92B01E1
:10E7C0003C0120E030E0A9010E94EBDB87FF04C0A0
:10E7D00077FA709477F8709481149104A104B104CD
:10E7E00059F420E030E040E85FE3C301B2010E9449
:10E7F0009BD587FF0DC00AC020E030E040E450E424
:10E80000C301B2010E94EBDB181614F44601570154
:10E81000E981EE2391F12A813B814C815D812115B3
:10E8200031054105510541F0D701C601821B930B0B
:10E83000A40BB50BB7FD21C02E813F81A8016D85CA
:10E840007E858F8598890E94C4D920E030E040EC15
:10E850005FE30E949BD587FD3BCFD701C601805A5D
:10E860009541AF4FBF4F8A839B83AC83BD839E810D
:10E870009D87AF81AE870F87188B809134028823E4
:10E8800009F426CF81149104A104B10409F4EDCE5A
:10E89000B0E1CB1AB7E2DB0AE108F108C818D908E1
:10E8A000EA08FB08F7FE14CFE0CE882361F0082EBB
:10E8B000000C990B0E948887EA81FB813196FB83CB
:10E8C000EA838491F2CF8DE090E00E9488878AE00D
:10E8D00090E00E9488878091340281E08093C50592
:10E8E00003C06EE670E070CE62960FB6F894DEBF9D
:10E8F0000FBECDBFDF91CF911F910F91FF90EF9091
:10E90000DF90CF90BF90AF909F908F907F906F904F
:10E910005F904F903F902F9008959F92AF92BF923B
:10E92000CF92DF92EF92FF920F931F93CF93DF93DB
:10E930008FE4A82E82E0B82E00EE15E0C9E2D4E004
:10E940009EE0C92E94E0D92E2AE1E22E24E0F22E98
:10E95000912CF50181915F010E942051882309F1DA
:10E960000E94E950F7012081211104C020911E046A
:10E97000222339F0288139814A815B810E94C5D9DF
:10E980000AC0F3E09F1639F0F601208131814281FF
:10E9900053810E94C4D9F801608371838283938379
:10E9A00009C088819981AA81BB81F8018083918304
:10E9B000A283B38393940C5F1F4F2496F4E0CF0E91
:10E9C000D11C2FEFE21AF20A84E09812C2CF86E43B
:10E9D0000E9469518823C9F00E94E95020E030E08C
:10E9E000A9010E94EBDB181684F40E94E95020E094
:10E9F00030E040E752E40E94A1DA60934B0270934A
:10EA00004C0280934D0290934E02DF91CF911F9163
:10EA10000F91FF90EF90DF90CF90BF90AF909F90BD
:10EA200008952F923F924F925F926F927F929F92A2
:10EA3000AF92BF92CF92DF92EF92FF920F931F930C
:10EA4000CF93DF93CDB7DEB764970FB6F894DEBFF0
:10EA50000FBECDBF1A012B01922EF32EC82ED12C42
:10EA6000F601ED55F84EE491AA24A3941E160CF479
:10EA7000A12CBB24B39420E030E0A901C201B10174
:10EA80000E94EBDB18160CF0B12CCC0CDD1CCC0C6E
:10EA9000DD1CC601875D9B4F3C01FC011082118289
:10EAA000128213820E947250F301208231824282CC
:10EAB0005382E090C40520E030E0A901B801892D1F
:10EAC0009F2D0E949BD581110AC0F601E459F74D94
:10EAD00085919591A591B4918C019A2EFB2EC80138
:10EAE000A92DBF2D898B9A8BAB8BBC8B8091310468
:10EAF00090913204A0913304B091340440912D04DC
:10EB000050912E0460912F047091300400912904DB
:10EB100010912A0420912B0430912C0409831A832C
:10EB20002B833C834D835E836F83788789879A87A5
:10EB3000AB87BC871D861E861F86188AAE01475F7D
:10EB40005F4FBE016B5F7F4FCE0101960E94BDAE4D
:10EB5000CE010D966C018E010F5E1F4F25E334E050
:10EB6000AE01475F5F4FBE016B5F7F4F0C970E9406
:10EB7000EE6058DBAB1459F080917906882319F0C8
:10EB80001092790604C088EF97E10E9415586496A8
:10EB90000FB6F894DEBF0FBECDBFDF91CF911F91AE
:10EBA0000F91FF90EF90DF90CF90BF90AF909F902C
:10EBB0007F906F905F904F903F902F900895EF92CD
:10EBC000FF921F93CF93DF9385EBE82E80E1F82E21
:10EBD00015E0C0E0D0E020E030E0A901F701EC0F43
:10EBE000FD1F60817181828193810E949BD581117B
:10EBF0000CC02496C431D10571F7115084E1E80EA0
:10EC0000F11C1111E6CF80E001C081E0DF91CF91CE
:10EC10001F91FF90EF900895CF939091FD17981753
:10EC2000C1F0C82FFFDAC11112C041E354E06DE218
:10EC300074E089E294E00E94BDAE80E08093FD170D
:10EC4000882339F089E294E0CF910C9459B8B7DF6A
:10EC5000F5CFCF9108958F929F92AF92BF92EF928E
:10EC6000FF920F931F93CF93DF9300D01F92CDB7E6
:10EC7000DEB7182F809128048770873069F48FE4FD
:10EC80000E946951882319F00E94DA5003C08FE472
:10EC90000E9420518111BCC0C5DA80E0BDDF8091A7
:10ECA0004B0290914C02A0914D02B0914E02809384
:10ECB000530690935406A0935506B0935606809140
:10ECC000020290910302909352068093510684E6CB
:10ECD00090E0909303028093020281E080936806A3
:10ECE00011111BC088E50E942051F82E89E50E9471
:10ECF0002051082F8AE50E942051E82EF11006C00D
:10ED0000011109C0811107C0F02E0CC0002319F0B9
:10ED1000F02E182F08C010E006C0FF24F39401E085
:10ED2000EE24E39411E00E947B5182E50E94695138
:10ED3000882361F00E94E9504B015C0120E030E043
:10ED4000A9010E949BD5882371F106C0812C912CCA
:10ED500080EAA82E80E4B82E111104C0F11002C080
:10ED6000002391F18092E8059092E905A092EA05CE
:10ED7000B092EB05A50194016091310470913204C9
:10ED800080913304909134040E949BD587FF0BC07F
:10ED900019821A821B821C82BE016F5F7F4F88EE30
:10EDA00095E00E947BC2111105C0F11003C0011152
:10EDB00006C00AC080E00E94BD561123C1F381E065
:10EDC0000E94BD56111102C0EE2019F082E00E948F
:10EDD000BD560E94725080916706809368068091AC
:10EDE000530690915406A0915506B0915606809313
:10EDF0004B0290934C02A0934D02B0934E0280912F
:10EE00005106909152069093030280930202E0DA39
:10EE10000F900F900F900F90DF91CF911F910F9156
:10EE2000FF90EF90BF90AF909F908F900895CF92FA
:10EE3000DF92EF920F931F93CF93DF93CDB7DEB79F
:10EE400060970FB6F894DEBF0FBECDBFE090C4054B
:10EE5000E9E2F4E080859185A285B38544815581FE
:10EE600066817781008111812281338109831A8330
:10EE70002B833C834D835E836F83788789879A8752
:10EE8000AB87BC871D861E861F86188AAE01475F2A
:10EE90005F4FBE016B5F7F4FCE0101960E94BDAEFA
:10EEA000CE010D966C010BE412E025E334E0AE01D7
:10EEB000475F5F4FBE016B5F7F4F0C970E94EE6014
:10EEC00060960FB6F894DEBF0FBECDBFDF91CF9135
:10EED0001F910F91EF90DF90CF9008950F931F93A4
:10EEE000CF93DF9394E0899FE00111248E01025FAC
:10EEF0001B4FFE01E759F94FDE01AD52BA4F2D917C
:10EF00003D914D915C9160817181828193810E94DC
:10EF1000C5D9F8016083718382839383FE01E05237
:10EF2000F84E85919591A591B491FE01E455FA4F63
:10EF300080839183A283B383FE01E451F84E8591CF
:10EF40009591A591B491CB5EDD4F88839983AA8377
:10EF5000BB83DF91CF911F910F9108952F923F9224
:10EF60004F925F926F927F928F929F92AF92BF92D9
:10EF7000CF92DF92EF92FF920F931F93CF93DF9385
:10EF8000CDB7DEB762970FB6F894DEBF0FBECDBF28
:10EF90008DE690E00E9412558111C5C180914B060B
:10EFA00083FDC1C183E50E9469518C87811106C030
:10EFB00082E50E94695189838823B1F00E94E9505B
:10EFC0000E9409DBCB010E9426860E94E95020E0C6
:10EFD00030E044EB52E40E949BD518160CF49EC11D
:10EFE0000E942F9021E02983EAE4F8E184918F01C7
:10EFF000882351F0082E000C990B0E9488870F5F20
:10F000001F4FF8018491F4CF8DE090E00E94888733
:10F010008AE090E00E9488870E948BB9F981FF23E3
:10F0200009F481C181E0809334021092C5051A82EF
:10F030001B821C821D82188619861A861B861982DD
:10F040001D862CE32E873CE13F8746E4488B312C1C
:10F05000212C50E8598B8FEB8A8B812C912C5401F9
:10F060006091410470914204072E000C880B990BAB
:10F070000E94A1D57B018C019B01AC01632D722DF7
:10F0800089899A890E949BD5882359F1209143044C
:10F090003091440440914504509146049C85B70149
:10F0A000802F91110CC0912F0E949BD5881F88271B
:10F0B000881F89833E2C2F2C098B1A8B12C0912F0D
:10F0C0000E949BD587FF08C080913402E2E5F8E1F9
:10F0D0008491FB83EA83E7C03E2C2F2C098B1A8B8B
:10F0E00019820E9410C56B017C01DC01CB012885CF
:10F0F00039854A855B85821B930BA40BB50BB7FD45
:10F100003BC0D701C60188519C4FAF4FBF4F888786
:10F110009987AA87BB870E94468DE6E5F8E184912E
:10F120003F019FEF691A790A882321F00E948551D7
:10F13000F301F5CF81149104A104B104B9F0D50114
:10F14000C401805F984DAF4FBF4FBC01CD016C191A
:10F150007D098E099F0928EE33E040E050E00E94CF
:10F1600089D9CA01B9010E944E5503C08FE30E949C
:10F1700085518AE00E9485510E945A580E9410C50C
:10F180006093C6057093C7058093C8059093C90521
:10F19000A0914304AE83B0914404BF830091450421
:10F1A000109146040E94D3302E813F81A801632D27
:10F1B000722D89899A890E94C4D92B013C0120E0D3
:10F1C00030E0A9010E94EBDB87FF04C077FA70945E
:10F1D00077F8709481149104A104B10459F420E0EB
:10F1E00030E040E85FE3C301B2010E949BD587FF96
:10F1F0000DC00AC020E030E040E450E4C301B20199
:10F200000E94EBDB181614F446015701E981EE2346
:10F2100091F12A813B814C815D81211531054105A8
:10F22000510541F0D701C601821B930BA40BB50B0E
:10F23000B7FD21C02E813F81A8016D857E858F8518
:10F2400098890E94C4D920E030E040EC5FE30E943E
:10F250009BD587FD39CFD701C601805A9541AF4F65
:10F26000BF4F8A839B83AC83BD839E819D87AF8183
:10F27000AE870F87188B80913402882309F424CF3E
:10F2800081149104A104B10409F4EACEB0E1CB1ACF
:10F29000B7E2DB0AE108F108C818D908EA08FB0858
:10F2A000F7FE12CFDDCE882361F0082E000C990BFB
:10F2B0000E948887EA81FB813196FB83EA838491EF
:10F2C000F2CF8DE090E00E9488878AE090E00E9473
:10F2D00088878091970E8130E9F4EEE4F8E184911B
:10F2E000FB83EA83882371F0082E000C990B0E949F
:10F2F00088874A815B814F5F5F4F5B834A83FA0156
:10F300008491F0CF8DE090E00E9488878AE090E0C1
:10F310000E94888781E08093C50505C00E940D90FA
:10F3200031E0398361CE62960FB6F894DEBF0FBE2E
:10F33000CDBFDF91CF911F910F91FF90EF90DF90A4
:10F34000CF90BF90AF909F908F907F906F905F9085
:10F350004F903F902F900895EF92FF920F931F933D
:10F36000CF93DF93CDB7DEB76D970FB6F894DEBFBE
:10F370000FBECDBF80918A0A882309F486C082E53A
:10F380009CE00E9459BF82E59CE00E94BFA21092BF
:10F39000880A1092870A80918A0A882309F475C026
:10F3A00000913218109133180E94B189B801CE0132
:10F3B0004C960E94C58B8C01892B09F466C06C8D1C
:10F3C0007D8D6115710511F06C5F7F4F19821C8274
:10F3D00022E0A801CE0101960E9452A8811102C02C
:10F3E000F12C14C0CE0101960E941F898823C1F31D
:10F3F00061E0CE0101960E94C8A2009789F325EE34
:10F40000FC0120831C820E9402BDF82ECE010196D1
:10F410000E947551FF2009F1E5E1F8E184917F0137
:10F420009FEFE91AF90A882321F00E948551F7011C
:10F43000F5CFF80181918F01882319F00E94855141
:10F44000F8CF8AE00E9485511092030D1092040DAE
:10F450001092050D1092060D18C0E3E2F8E18491B8
:10F460007F019FEFE91AF90A882321F00E94855154
:10F47000F701F5CFF80181918F01882319F00E94DF
:10F480008551F8CF8EE20E9485516D960FB6F894A3
:10F49000DEBF0FBECDBFDF91CF911F910F91FF90C7
:10F4A000EF900895CF93DF938B3D9240B1F0E7E664
:10F4B000FBE18491EF012196882321F00E94855180
:10F4C000FE01F7CFE0ECF8E18491EF01219688236B
:10F4D00031F00E948551FE01F7CF80E001C081E04C
:10F4E000DF91CF9108952F923F924F925F926F924A
:10F4F0007F928F929F92AF92BF92CF92DF92EF92C4
:10F50000FF920F931F93CF93DF93CDB7DEB7C7570B
:10F51000D1090FB6F894DEBF0FBECDBF2DB63EB6F3
:10F52000A7961FAE1EAEA79784E690E0A9969FAF60
:10F530008EAFA99701E09E012B593F4F44E050E068
:10F54000BE01655A7F4FCE0189599F4F0E949DBBD6
:10F550009E012B593F4F42E050E0BE0167597F4F5B
:10F56000CE0189599F4F0E949DBB43E050E0BE01F0
:10F57000655A7F4F87ED92E00E944CDD892B09F49C
:10F580003FC06F968FAD6F97882339F08FE36C96ED
:10F590008FAF6C976D961FAE6D97ECE7FBE1849192
:10F5A0007F012FEFE21AF20A811103C0E3E8F9E1CB
:10F5B00004C00E948551F701F2CF84917F013FEF93
:10F5C000E31AF30A882321F00E948551F701F5CF51
:10F5D000BE01655A7F4F8AE799E10E9461B7ECE668
:10F5E000F9E184917F019FEFE91AF90A882321F05C
:10F5F0000E948551F701F5CF81E08093570654C5ED
:10F60000EDB7FEB7E696FFAFEEAFE6976B961CAE92
:10F610001DAE1EAE1FAE6B97A7961FAE1EAEA79770
:10F6200001E09E012B593F4F41E050E0BE0160597F
:10F630007F4FCE0189599F4F0E949DBB80E1E3E53A
:10F64000F2E0DE01919601900D928A95E1F780E15A
:10F65000E3E6F2E0DE01519601900D928A95E1F722
:10F6600080E1E3E7F2E0DE01119601900D928A95C8
:10F67000E1F7E1964FADE19750E04D5F5F4F440FEA
:10F68000551F440F551F2DB73EB7241B350B0FB622
:10F69000F8943EBF0FBE2DBF8DB79EB701967C017B
:10F6A00000E09E012B593F4FBC01CE0189599F4F6D
:10F6B0000E949DBB9E012B593F4F44E050E06EE3FA
:10F6C00076E0CE0189599F4F0E949DBBE1968FAC99
:10F6D000E197912C93E0890E911C880C991C880C61
:10F6E000991CEDB7FEB7E819F9090FB6F894FEBFFB
:10F6F0000FBEEDBF2DB73EB72F5F3F4F69018DB7EE
:10F700009EB7881999090FB6F8949EBF0FBE8DBF9A
:10F71000EDB7FEB731965F019E012B593F4FA40113
:10F72000B601CE0189599F4F0E949DBB9E012B5966
:10F730003F4FA401B501CE0189599F4F0E949DBB47
:10F7400010915806112309F4A7C000E09E012B591F
:10F750003F4F44E050E066E276E0CE0189599F4F8A
:10F760000E949DBB9E012B593F4F44E050E06AE24E
:10F7700076E0CE0189599F4F0E949DBB9E012B5977
:10F780003F4F44E050E062E276E0CE0189599F4F5E
:10F790000E949DBB9E012B593F4F44E050E066E420
:10F7A00076E0CE0189599F4F0E949DBB9E012B5947
:10F7B0003F4F44E050E062E476E0CE0189599F4F2C
:10F7C0000E949DBB9E012B593F4F40E150E06EE0EF
:10F7D00076E0CE0189599F4F0E949DBB9E012B5917
:10F7E0003F4F44E050E0BE01695A7F4FCE01895936
:10F7F0009F4F0E949DBB9E012B593F4F4CE050E014
:10F8000069E676E0CE0189599F4F0E949DBB9E011B
:10F810002B593F4F44E050E062E271E1CE0189593B
:10F820009F4F0E949DBB9E012B593F4F44E050E0EB
:10F83000BE01695A7F4FCE0189599F4F0E949DBBDF
:10F8400001E09E012B593F4F41E050E0BE0161595C
:10F850007F4FCE0189599F4F0E949DBB9E012B591E
:10F860003F4F41E050E0BE0162597F4FCE018959C0
:10F870009F4F0E949DBB11118AC06B968CAD9DADB0
:10F88000AEADBFAD6B978093B1109093B210A093C3
:10F89000B310B093B4107BC0E1968FADE19790E0C8
:10F8A00002962EE236E0E4963FAF2EAFE497B50124
:10F8B000DE011196EEE58E2EE1E19E2EAE014F5E49
:10F8C0005F4FFEE3AF2EF1E1BF2EE896FFAEEEAE46
:10F8D000E8977E0131E2E30EF11C20E030E0821770
:10F8E00093072CF0E896EEADFFADE89701C0F70165
:10F8F0004080518062807380F50141925192619203
:10F9000071925F018217930714F0F60101C0FA01AA
:10F910004080518062807380F401419251926192E3
:10F9200071924F018217930734F0FB0140805180A0
:10F930006280738005C04D905D906D907C901397B0
:10F94000E496EEADFFADE4974192519261927192CF
:10F95000E496FFAFEEAFE4972F5F3F4F6C5F7F4FB2
:10F960001496F4E0CF0ED11C4C5F5F4FE896EEADDD
:10F97000FFADE8973496E896FFAFEEAFE897F4E076
:10F98000EF0EF11C2430310509F0A9CFDECEE09650
:10F990008FADE097853099F4AF968FADAF978530F6
:10F9A00071F400E09E012B593F4F44E650E065EBB7
:10F9B00070E1CE0189599F4F0E949DBB24C0111157
:10F9C00002C00E94AAAFE0968FADE097AF96CFAC91
:10F9D000AF978C9D60011124E12CF12CEC14FD04F7
:10F9E00091F000E09E012B593F4F44E050E0BE01F2
:10F9F000695A7F4FCE0189599F4F0E949DBB2FEFBF
:10FA0000E21AF20AEBCF00E09E012B593F4F44E08F
:10FA100050E0BE016D5A7F4FCE0189599F4F0E9421
:10FA20009DBB1AE0115079F000E09E012B593F4F29
:10FA300044E050E0BE01695A7F4FCE0189599F4F83
:10FA40000E949DBBEFCF01E09E012B593F4F41E04B
:10FA500050E0BE0163597F4FCE0189599F4F0E94EC
:10FA60009DBB9E012B593F4F41E050E0BE016459C0
:10FA70007F4FCE0189599F4F0E949DBB00E09E01A0
:10FA80002B593F4F44E050E0BE01635C7F4FCE01F5
:10FA900089599F4F0E949DBB9E012B593F4F44E0C7
:10FAA00050E0BE016F5C7F4FCE0189599F4F0E948D
:10FAB0009DBBAE968FADAE97AD96CFACAD978C9DFE
:10FAC00060011124E12CF12C00E09E012B593F4FE5
:10FAD000CE14DF0471F044E050E0BE01695A7F4F5C
:10FAE000CE0189599F4F0E949DBB3FEFE31AF30A55
:10FAF000EBCF41E050E0BE016F587F4FCE018959F6
:10FB00009F4F0E949DBB9E012B593F4F41E050E00B
:10FB1000BE0165597F4FCE0189599F4F0E949DBB01
:10FB20009E012B593F4F44E050E0BE01695A7F4F80
:10FB3000CE0189599F4F0E949DBB9E012B593F4F7B
:10FB400044E050E0BE01695A7F4FCE0189599F4F72
:10FB50000E949DBB9E012B593F4F44E050E066E25E
:10FB600071E1CE0189599F4F0E949DBB9E012B5987
:10FB70003F4F44E050E0BE01615B7F4FCE018959A9
:10FB80009F4F0E949DBB9E012B593F4F44E050E088
:10FB9000BE01655B7F4FCE0189599F4F0E949DBB7F
:10FBA0009E012B593F4F44E050E0BE01695B7F4FFF
:10FBB000CE0189599F4F0E949DBB10E000E09E013D
:10FBC0002B593F4F44E050E0BE01695A7F4FCE01B0
:10FBD00089599F4F0E949DBB111110C06B96CCACF0
:10FBE000DDACEEACFFAC6B9720E030E84BE355E4C6
:10FBF000C701B6010E949BD5811103C054E0F52EC8
:10FC000033C080915806811108C0C0924A10D0922A
:10FC10004B10E0924C10F0924D1000E09E012B59D9
:10FC20003F4F44E050E066E470E1CE0189599F4FB8
:10FC30000E949DBB9E012B593F4F44E050E06EE473
:10FC400070E1CE0189599F4F0E949DBB9E012B59A7
:10FC50003F4F44E050E0BE01695A7F4FCE018959C1
:10FC60009F4F0E949DBB12C0FA94FF2079F000E0E4
:10FC70009E012B593F4F44E050E0BE01695A7F4F2F
:10FC8000CE0189599F4F0E949DBBEECF1F5F15305B
:10FC900009F094CF00E09E012B593F4F42E050E025
:10FCA000BE016D597F4FCE0189599F4F0E949DBB68
:10FCB0009E012B593F4F44E050E0BE01695A7F4FEF
:10FCC000CE0189599F4F0E949DBB6B96CCACDDAC99
:10FCD000EEACFFAC6B9720E030E84BE355E4C70196
:10FCE000B6010E949BD5882329F180915806811185
:10FCF00008C0C0924210D0924310E0924410F0929B
:10FD0000451000E09E012B593F4F44E050E06EE368
:10FD100070E1CE0189599F4F0E949DBB9E012B59D6
:10FD20003F4F44E050E06AE370E1CE0189599F4FB4
:10FD30000E949DBB00E09E012B593F4F42E050E0E6
:10FD4000BE016F597F4FCE0189599F4F0E949DBBC5
:10FD50009E012B593F4F41E050E0BE016F587F4F4D
:10FD6000CE0189599F4F0E949DBB19E0115000E0C0
:10FD70009E012B593F4F112359F044E050E0BE0142
:10FD8000695A7F4FCE0189599F4F0E949DBBEECF8C
:10FD900041E050E069E171E1CE0189599F4F0E9435
:10FDA0009DBBF12C00E09E012B593F4F44E050E0F9
:10FDB000BE01695A7F4FCE0189599F4F0E949DBB5A
:10FDC00010915806111110C0F1100EC06B968CAD39
:10FDD0009DADAEADBFAD6B9780931E1190931F117B
:10FDE000A0932011B0932111F39485E0F812DACF9B
:10FDF000111102C00E94A9B64CE0F42EFA94F11041
:10FE000003C03CE0F32E0FC000E09E012B593F4F92
:10FE100042E050E0BE01615A7F4FCE0189599F4FA9
:10FE20000E949DBBEBCFFA9400E09E012B593F4FFF
:10FE3000FF2059F044E050E0BE016D5B7F4FCE01E2
:10FE400089599F4F0E949DBBEECF46E050E0BE0116
:10FE5000635C7F4FCE0189599F4F0E949DBB9E01DD
:10FE60002B593F4F44E050E06EE176E0CE018959D6
:10FE70009F4F0E949DBB9E012B593F4F4CE050E08D
:10FE8000BE016F5C7F4FCE0189599F4F0E949DBB81
:10FE90002CE1F22EFA94F11003C094E0F92E1DC06B
:10FEA00000E09E012B593F4F44E050E0BE01695AEB
:10FEB0007F4FCE0189599F4F0E949DBBEBCF00E041
:10FEC0009E012B593F4F44E050E0BE01695A7F4FDD
:10FED000CE0189599F4F0E949DBBFA94F110EFCF3C
:10FEE0008BE0F82EFA94FF2079F000E09E012B5968
:10FEF0003F4F44E050E0BE01695A7F4FCE0189591F
:10FF00009F4F0E949DBBEECFA9968EAD9FADA99746
:10FF100084569109C7DA80935706882309F1ECE7E4
:10FF2000FBE184917F019FEFE91AF90A882321F010
:10FF30000E948551F701F5CFA9966EAD7FADA997C7
:10FF40006456710984E699E10E9448B76BED72E04E
:10FF50008CE599E10E9448B78AE00E94855199C0DA
:10FF6000A7962EAD3FADA797AB968EAD9FADAB9745
:10FF70002817390709F44BC081E080935706E7E65C
:10FF8000FBE184917F012FEFE21AF20A811103C095
:10FF9000ECE3F9E104C00E948551F701F2CF8491AE
:10FFA0007F013FEFE31AF30A882321F00E94855175
:10FFB000F701F5CFAB966EAD7FADAB9780E090E0EB
:10FFC0004AE00E94A754E7E3F9E184917F019FEFA3
:10FFD000E91AF90A882321F00E948551F701F5CF2B
:10FFE000A7966EAD7FADA79780E090E04AE00E94B3
:10FFF000A754E7E2F9E184917F012FEFE21AF20AB8
:020000021000EC
:10000000882309F446C00E948551F701F4CF1111ED
:1000100042C0ECE7FBE184917F013FEFE31AF30A72
:10002000811103C007ED12E004C00E948551F70161
:10003000F2CFF80181918F01882319F00E94855138
:10004000F8CFA9966EAD7FADA997645671098AE085
:1000500099E10E9448B7A7964EAD5FADA79760E0C3
:1000600070E08DEF98E10E940EB7EAEFF8E184911D
:100070007F012FEFE21AF20A811107C08091570623
:10008000811109C00E945CBC06C00E948551F70125
:10009000EECF112399F3E6968EAD9FADE6970FB69E
:1000A000F8949EBF0FBE8DBF80915806811102C08B
:1000B0000E9477B09091570681E089270FB6F89497
:1000C0003EBE0FBE2DBEC958DF4F0FB6F894DEBF3F
:1000D0000FBECDBFDF91CF911F910F91FF90EF9099
:1000E000DF90CF90BF90AF909F908F907F906F9058
:1000F0005F904F903F902F90089581E08093580635
:10010000F2D9109258068111EEC90E94E6B481E03E
:1001100008958F929F92AF92BF92CF92DF92EF920B
:10012000FF920F931F93CF93DF93CDB7DEB7CA5AD9
:10013000D1090FB6F894DEBF0FBECDBFE9961CAE55
:100140001DAE1EAE1FAEE9978091F7039091F803A4
:10015000A091F903B091FA03ED968CAF9DAFAEAFCD
:10016000BFAFED97C556DF4F19821882CB59D040EB
:1001700084E690E0C356DF4F99838883CD59D04001
:10018000109257069E0125563F4F44E050E0BE01B5
:1001900067587F4FCE0183569F4F0E94E9BBC356DD
:1001A000DF4F88819981CD59D0400296C356DF4FE9
:1001B00099838883CD59D040C556DF4F1982188264
:1001C000CB59D04081E0CD55DF4F8883C35AD04012
:1001D0009E0125563F4F41E050E0BE016D557F4FD7
:1001E000CE0183569F4F0E94E9BB9E0125563F4F8B
:1001F00040E150E06EE371E1CE0183569F4F0E94D3
:10020000E9BB9E0125563F4F44E050E06EE376E0A7
:10021000CE0183569F4F0E94E9BB9E0125563F4F5A
:1002200040E150E06EE571E1CE0183569F4F0E94A0
:10023000E9BB9E0125563F4F40E150E06EE276E07B
:10024000CE0183569F4F0E94E9BB9E0125563F4F2A
:1002500044E050E066E276E0CE0183569F4F0E9474
:10026000E9BB9E0125563F4F44E050E06AE276E04C
:10027000CE0183569F4F0E94E9BB9E0125563F4FFA
:1002800044E050E062E276E0CE0183569F4F0E9448
:10029000E9BB9E0125563F4F44E050E066E476E01E
:1002A000CE0183569F4F0E94E9BB9E0125563F4FCA
:1002B00044E050E062E476E0CE0183569F4F0E9416
:1002C000E9BB9E0125563F4F40E150E06EE076E0ED
:1002D000CE0183569F4F0E94E9BB8AE097EDA3EAC7
:1002E000BCE3E9968CAF9DAFAEAFBFAFE9979E017F
:1002F00025563F4F44E050E0BE016B587F4FCE0182
:1003000083569F4F0E94E9BB9E0125563F4F4CE00C
:1003100050E069E676E0CE0183569F4F0E94E9BB2C
:100320008091FE179091FF17A0910018B0910118CD
:10033000C358DF4F88839983AA83BB83CD57D040AE
:100340009E0125563F4F44E050E0BE0163587F4F69
:10035000CE0183569F4F0E94E9BB85E0CC55DF4F0D
:100360008883C45AD040CB55DF4F8883C55AD040CC
:100370009E0125563F4F44E050E061EB70E1CE0115
:1003800083569F4F0E94E9BB9E0125563F4F41E097
:1003900050E0BE016C557F4FCE0183569F4F0E94A7
:1003A000E9BB9E0125563F4F41E050E0BE016B5531
:1003B0007F4FCE0183569F4F0E94E9BB9E01255679
:1003C0003F4F44E650E065EB70E1CE0183569F4F0E
:1003D0000E94E9BBCF57DF4F188219821A821B8215
:1003E000C158D0409E0125563F4F44E050E0BE0129
:1003F0006F577F4FCE0183569F4F0E94E9BBE9960E
:100400001CAE1DAE1EAE1FAEE9971AE0115071F082
:100410009E0125563F4F44E050E0BE016B587F4F90
:10042000CE0183569F4F0E94E9BBF0CF83E0CA55AF
:10043000DF4F8883C65AD040C955DF4F8883C75ADB
:10044000D040CB57DF4F188219821A821B82C558C1
:10045000D040C757DF4F188219821A821B82C958B1
:10046000D040E9961CAE1DAE1EAE1FAEE9979E01B0
:1004700025563F4F41E050E0BE016A557F4FCE0107
:1004800083569F4F0E94E9BB9E0125563F4F41E096
:1004900050E0BE0169557F4FCE0183569F4F0E94A9
:1004A000E9BB9E0125563F4F44E050E0BE0167572F
:1004B0007F4FCE0183569F4F0E94E9BB9E01255678
:1004C0003F4F44E050E0BE016B577F4FCE01835653
:1004D0009F4F0E94E9BB0AE010E00150110971F042
:1004E0009E0125563F4F44E050E0BE016B587F4FC0
:1004F000CE0183569F4F0E94E9BBEFCFC855DF4F17
:100500001882C85AD0408FEFC755DF4F8883C95A29
:10051000D0409E0125563F4F41E050E0BE01685556
:100520007F4FCE0183569F4F0E94E9BB9E01255607
:100530003F4F41E050E0BE0167557F4FCE018356EB
:100540009F4F0E94E9BBE9961CAE1DAE1EAE1FAECA
:10055000E9979E0125563F4F44E050E0BE016B589D
:100560007F4FCE0183569F4F0E94E9BB9E012556C7
:100570003F4F44E050E0BE016B587F4FCE018356A1
:100580009F4F0E94E9BB9E0125563F4F44E050E03B
:1005900066E271E1CE0183569F4F0E94E9BB8091D4
:1005A000830290918402A0918502B0918602C35784
:1005B000DF4F88839983AA83BB83CD58D040809135
:1005C000870290918802A0918902B0918A02CF5649
:1005D000DF4F88839983AA83BB83C159D040CB5610
:1005E000DF4F19821882C559D040C956DF4F198292
:1005F0001882C759D0409E0125563F4F44E050E035
:10060000BE0163577F4FCE0183569F4F0E94E9BBC7
:100610009E0125563F4F44E050E0BE016F567F4F8C
:10062000CE0183569F4F0E94E9BB9E0125563F4F46
:1006300044E050E0BE016B567F4FCE0183569F4F82
:100640000E94E9BB10E0C12C80E8D82E8BE3E82E95
:1006500085E4F82E812C912C90E8A92E9FE3B92EE9
:10066000111138C09E0125563F4F44E050E06AE426
:1006700070E1CE0183569F4F0E94E9BB9E01255633
:100680003F4F44E050E066E470E1CE0183569F4F57
:100690000E94E9BB9E0125563F4F44E050E06EE4C6
:1006A00070E1CE0183569F4F0E94E9BBE9968CAE64
:1006B0009DAEAEAEBFAEE9979E0125563F4F44E0DA
:1006C00050E0BE016B587F4FCE0183569F4F0E9472
:1006D000E9BB2AC0E996CCAEDDAEEEAEFFAEE9973F
:1006E0009E0125563F4F44E050E0BE016B587F4FBE
:1006F000CE0183569F4F0E94E9BBE9961CAE1DAE0A
:100700001EAE1FAEE99704E0015071F09E01255620
:100710003F4F44E050E0BE016B587F4FCE018356FF
:100720009F4F0E94E9BBF0CF1F5F153009F098CFB3
:1007300084E190E0C156DF4F99838883CF59D04040
:100740009E0125563F4F42E050E0BE0161567F4F6B
:10075000CE0183569F4F0E94E9BB9E0125563F4F15
:1007600044E050E062E470E1CE0183569F4F0E9466
:10077000E9BB9E0125563F4F44E050E06EE370E137
:10078000CE0183569F4F0E94E9BB9E0125563F4FE5
:1007900044E050E06AE370E1CE0183569F4F0E942F
:1007A000E9BB80E290E0CF55DF4F99838883C15A3F
:1007B000D0409E0125563F4F42E050E0BE016F55AC
:1007C0007F4FCE0183569F4F0E94E9BBC655DF4F36
:1007D0001882CA5AD04080E2EBE8F2E0DE019D9632
:1007E00001900D928A95E1F79E0125563F4F41E019
:1007F00050E0BE0166557F4FCE0183569F4F0E9449
:10080000E9BB9E0125563F4F40E250E0BE01635DCB
:100810007F4FCE0183569F4F0E94E9BB9E01255614
:100820003F4F41E050E069E171E1CE0183569F4FB7
:100830000E94E9BB10E011110EC080911E11909131
:100840001F11A0912011B0912111E9968CAF9DAF9D
:10085000AEAFBFAFE9979E0125563F4F44E050E051
:10086000BE016B587F4FCE0183569F4F0E94E9BB5C
:100870001F5F153001F7BE01635B7F4F86E1FB010F
:1008800011928A95E9F79E0125563F4F46E150E0C7
:10089000CE0183569F4F0E94E9BB8CE2EBEAF2E067
:1008A000DE01119601900D928A95E1F79E01255681
:1008B0003F4F4CE250E0BE016F5F7F4FCE01835649
:1008C0009F4F0E94E9BBBE0161597F4F86E0FB014B
:1008D00011928A95E9F79E0125563F4F46E050E078
:1008E000CE0183569F4F0E94E9BB9E0125563F4F84
:1008F00044E050E06EE176E0CE0183569F4F0E94C7
:10090000E9BBBE016D597F4F8CE0FB0111928A95C6
:10091000E9F79E0125563F4F4CE050E0CE0183564B
:100920009F4F0E94E9BBE9961CAE1DAE1EAE1FAEE6
:10093000E9971CE1115071F09E0125563F4F44E0AC
:1009400050E0BE016B587F4FCE0183569F4F0E94EF
:10095000E9BBF0CFE9961CAE1DAE1EAE1FAEE99707
:1009600014E0115071F09E0125563F4F44E050E0D5
:10097000BE016B587F4FCE0183569F4F0E94E9BB4B
:10098000F0CFE9961CAE1DAE1EAE1FAEE9971BE080
:10099000115071F09E0125563F4F44E050E0BE01DA
:1009A0006B587F4FCE0183569F4F0E94E9BBF0CF1B
:1009B00080915706811167C0C356DF4FE880F980E8
:1009C000CD59D040F4E6EF1AF108C556DF4F8881C3
:1009D0009981CB59D040C756DF4F99838883C95935
:1009E000D04084E690E0C356DF4F99838883CD5989
:1009F000D0409E0125563F4F44E050E067ED72E045
:100A0000CE0183569F4F0E94E9BB9E0125563F4F62
:100A100042E050E0BE0167567F4FCE0183569F4FA4
:100A20000E94E9BBECE7FBE184918F010F5F1F4F50
:100A3000882321F00E948551F801F6CFB70188EE96
:100A400098E10E9448B7C756DF4F48815981C9597C
:100A5000D04060E070E08BED98E10E940EB7E8EDC9
:100A6000F8E184918F010F5F1F4F882321F00E94CE
:100A70008551F801F6CFC7010E94527A909157062E
:100A8000892B809357069091570681E08927C65598
:100A9000DF4F0FB6F894DEBF0FBECDBFDF91CF9111
:100AA0001F910F91FF90EF90DF90CF90BF90AF908C
:100AB0009F908F900895CF92DF92EF92FF920F93C5
:100AC0001F93CF93DF936C017A018B01C0E0D0E0DC
:100AD000CE15DF0581F0D8016D918D01D601ED9124
:100AE000FC910190F081E02DC6011995892B11F040
:100AF0002196EECF7E01C701DF91CF911F910F911B
:100B0000FF90EF90DF90CF9008950E94F1DC1F924C
:100B10000F920FB60F9211240BB60F922F933F93A3
:100B20004F935F936F937F938F939F93AF93BF93F5
:100B3000EF93FF9380915C0690915D06A0915E0615
:100B4000B0915F06892B8A2B8B2B59F190915B0614
:100B5000E0915906F0915A0680818927808380911F
:100B60005C0690915D06A0915E06B0915F06181636
:100B700019061A061B060CF056C080915C0690916F
:100B80005D06A0915E06B0915F060197A109B109CB
:100B900080935C0690935D06A0935E06B0935F061B
:100BA00042C080912D02ECE9F9E1E4919FEF90932E
:100BB0002D02E230C9F050F4EE2399F0E13081F5D6
:100BC00090916F009D7F90936F002AC0E43019F1DF
:100BD000E0F0E53029F5909173009D7F90937300CC
:100BE0001FC010926E001CC0909170009D7F90936A
:100BF000700091E09093B0009091B100987F946064
:100C00009093B1001092B3000BC0909171009D7F42
:100C10009093710005C0909172009D7F9093720037
:100C200060E00E94A7C3FF91EF91BF91AF919F91A8
:100C30008F917F916F915F914F913F912F910F9085
:100C40000BBE0F900FBE0F901F901895909342040B
:100C50008093410480E00C944C8E8F929F92AF92CF
:100C6000BF92CF92DF92EF92FF921F93CF93DF93C9
:100C7000C82F8BE29CE09093070A8093060A10929B
:100C8000470C82E090E0A0E0B0E08093300C9093BD
:100C9000310CA093320CB093330C1092050A1092D1
:100CA000010A1092020A1092030A1092040A8FEFAE
:100CB0009FEFDC018093FD099093FE09A093FF094B
:100CC000B093000ACC2379F1C53008F0F8C040E0B9
:100CD00060E070E0CB010E9442BD882309F4EFC0C0
:100CE00020E1C29FC00111248351984FFC01E254BE
:100CF000FE4F20812F7709F0E2C03C964081518160
:100D000062817381443651056105710508F4D7C0CD
:100D10003497C080D180E280F380C114D104E10413
:100D2000F10421F4CCC0C12CD12C760140E0C701E4
:100D3000B6010E9442BD182F882309F4C0C08091DB
:100D40000808909109088115924009F0B8C0A09157
:100D50000D08AA2309F4B3C060910B0870910C0828
:100D60006115710509F4ABC020910A08222309F42A
:100D7000A6C0A093420C2093340C80E030E041E008
:100D800050E0C82FFA01082E02C0EE0FFF1F0A9490
:100D9000E2F72E173F0739F08F5FC83091F789E0EF
:100DA00080933D0C8CC080933D0C209113083091B2
:100DB00014082115310519F040E050E008C02091D9
:100DC0002108309122084091230850912408209353
:100DD000350C3093360C4093370C5093380C460149
:100DE0005701860E971EA11CB11C8092430C909255
:100DF000440CA092450CB092460CE0910E08F09184
:100E00000F08F093490CE093480CB0E00E94ABD976
:100E1000860E971EA81EB91E80924A0C90924B0C0B
:100E2000A0924C0CB0924D0C85E0EE0FFF1F8A95FE
:100E3000E1F7E150FE4FEF2FFF27E6958E0E9F1E44
:100E4000A11CB11C80923E0C90923F0CA092400CD1
:100E5000B092410C209110083091110821153105F4
:100E600021F0A90160E070E008C040911D08509198
:100E70001E0860911F0870912008D701C6018819CB
:100E80009909AA09BB09840F951FA61FB71F04C0A3
:100E9000B695A79597958795CA95D2F78093390C03
:100EA00090933A0CA0933B0CB0933C0C853F2FE001
:100EB0009207A105B10528F48CE08093470C10E05F
:100EC0001AC0853F9F4FA105B10510F480E111C004
:100ED0008091290890912A08A0912B08B0912C08A4
:100EE00080934A0C90934B0CA0934C0CB0934D0CF8
:100EF00080E28093470C812FDF91CF911F91FF906B
:100F0000EF90DF90CF90BF90AF909F908F9008951B
:100F1000682F82EF9FE00C94094CCF92DF92EF9202
:100F2000FF921F93CF93DF9310928A0A8091BD0A9C
:100F3000882321F08AEB9AE00E94BFA210922F0C26
:100F400010922C0C85E380932B0C0E9410C5EB01B2
:100F5000A89561E080912B0C0E94D5C38BE29CE0A8
:100F60000E9420A42398229A219A209A289A85E008
:100F700080932D0C82E58CBD1DBC1AE08FEF0E9482
:100F800025A41150D9F720E030E0A90160E08BE200
:100F90009CE00E942AA4182F80932E0C813049F0E7
:100FA0000E9410C56C1B7D0B613D774060F381E0B2
:100FB00054C02AEA31E040E050E068E08BE29CE077
:100FC0000E942AA482FF03C010932F0C0EC014E0CD
:100FD0000E94B65680932E0C1150D1F78A3A11F028
:100FE00082E03BC082E080932F0C80912F0C8230F6
:100FF00021F0C12CD12C760105C0C12CD12CE12CC3
:1010000080E4F82E20E030E0A90167E38BE29CE069
:101010000E942AA4A701960169E28BE29CE00E944B
:101020002AA480932E0C882349F00E9410C56C1BC3
:101030007D0B613D774030F38AE00FC080912F0C2B
:10104000823011F520E030E0A9016AE38BE29CE0F8
:101050000E942AA4882351F088E080932C0C8BE214
:101060009CE00E9420A4ECE7FBE119C00E94B65668
:10107000807C803C19F483E080932F0C0E94B6564C
:101080000E94B6560E94B6568BE29CE00E9420A4B5
:1010900010922D0C81E0E1DD811131C015C08491E9
:1010A000EF012196882321F00E948551FE01F7CFA0
:1010B000EEE6FBE18491EF012196882309F456C006
:1010C0000E948551FE01F6CF80E0C7DD811117C077
:1010D000E7E6FBE18491EF012196882321F00E944D
:1010E0008551FE01F7CFE3E5FBE18491EF01219605
:1010F000882309F43BC00E948551FE01F6CF60E3CE
:101100007CE08AEB9AE00E946CA2811116C0E7E6AF
:10111000FBE18491EF012196882321F00E94855103
:10112000FE01F7CFE2E4FBE18491EF0121968823F1
:10113000E9F00E948551FE01F7CF81E080938A0A91
:10114000ECE7FBE18491EF012196882321F00E94D6
:101150008551FE01F7CFE6E3FBE18491EF01219693
:10116000882321F00E948551FE01F7CF8BE1EAEB45
:10117000FAE0A9EDBAE001900D928A95E1F780912D
:10118000B80A9091B90A9093D80A8093D70ADF9150
:10119000CF911F91FF90EF90DF90CF9008958091B5
:1011A000970E823041F481E29BE19093FC0780939B
:1011B000FB070E94B1510E9410C560939B0E709373
:1011C0009C0E80939D0E90939E0E80918A0A882398
:1011D00019F081E08093890A81E08093970E089549
:1011E000CF93DF931092890A83E08093970E8091CA
:1011F000E40E8823B1F0E9E1FBE18491EF0188235B
:1012000041F0082E000C990B83DE2196FE0184919B
:10121000F6CF8DE090E07CDE8AE090E0DF91CF9128
:1012200077CEEDE1FBE18491EF01882391F3082E65
:10123000000C990B6DDE2196FE018491F6CF8F9202
:101240009F92AF92BF92CF92DF92EF92FF920F9355
:101250001F93CF93DF9300D01F92CDB7DEB7FC0171
:101260008381813079F5818181FF2CC081899289C8
:10127000A389B489892B8A2B8B2B09F448C07F0161
:1012800040E050E0BA01CF010E94D5A18823D1F0FF
:10129000F70185889688A788B08CC18CD28C82E0B3
:1012A00090E0A0E0B0E0F60180839183A283B38355
:1012B0009E012F5F3F4FB501A401C6010E940BBEE6
:1012C000811102C080E03CC000E010E09801B5014F
:1012D000A401C6010E947ABD8823A1F389809A8067
:1012E000AB80BC80F6018789803141F4F8EF8F161E
:1012F000FFEF9F06A104B10460F4DACF88EF8816EF
:101300008FEF9806A8068FE0B80618F4D1CF81E0D9
:1013100017C0F701158A168A178A108E118A128A49
:10132000138A148A818180688183C7010E9459BF12
:10133000882341F240E050E0BA01C7010E94D5A1E4
:101340000F900F900F900F90DF91CF911F910F9101
:10135000FF90EF90DF90CF90BF90AF909F908F90D5
:10136000089510928C0A1092890A8091550C882356
:1013700021F082E59CE00C94BFA208952F923F9249
:101380004F925F926F927F928F929F92AF92BF9295
:10139000CF92DF92EF92FF920F931F93CF93DF9341
:1013A000CDB7DEB7C257D1090FB6F894DEBF0FBE76
:1013B000CDBF8C013B014A014DB75EB7E1965FAFEF
:1013C0004EAFE197AD961FAEAD971B0154E0250ED1
:1013D000311C7E018FE5E80EF11C95EE492E92E05E
:1013E000592EE0E4F0E0EC0FFD1F3496E396FFAFDA
:1013F000EEAFE397F3018781823008F462C1848500
:101400009585A685B7858F719927AA27BB27892B34
:101410008A2B8B2B09F055C110929A0A4AE95AE09F
:10142000BE016F5F7F4FC1010E94F1BE18160CF024
:1014300048C18C85982F9871903129F42091070D1F
:101440002150223078F42981222309F43AC1253E23
:1014500089F22E3279F220919A0A2E3259F28A704C
:1014600049F6B8C04DB75EB7AF965FAF4EAFAF9716
:10147000BE016F5F7F4FC7010E94ECBC01151105D3
:1014800021F0F801808181119BC021E081E090E092
:10149000F70101900020E9F73197EE19FF098E0F4F
:1014A0009F1F02964DB75EB7481B590B0FB6F894B5
:1014B0005EBF0FBE4DBF8DB79EB701965C01211177
:1014C00002C0B80102C06AE173E0C5010E9445DDB7
:1014D000B701C5010E9426DD6AE173E0C5010E94E3
:1014E00026DD25961FAE259728961FAE28972496B1
:1014F0001FAE1EAE249722965FAE4EAE229721E01D
:10150000A701B101E3968EAD9FADE3970E9452A86B
:1015100081112AC08091070D811126C0ECE7FBE103
:1015200084916F019FEFC91AD90A882321F00E9484
:101530008551F601F5CFE5E0FBE184916F012FEFD6
:10154000C21AD20A882321F00E948551F601F5CFF4
:101550006701F60181916F01882319F00E9485517E
:10156000F8CF8AE00E9485518BE1FE01EC5BFF4FD2
:10157000DE01959601900D928A95E1F724968EAD45
:101580009FAD24979CA38BA35AA249A240E050E0B0
:10159000BE016F5D7F4FC501F1DECE0181960E94D5
:1015A000F357CE01805C9F4F0E94F357AF964EAD2C
:1015B0005FADAF970FB6F8945EBF0FBE4DBF1ACFA9
:1015C000F80101900020E9F73197CF01801B910BC2
:1015D00020E05ECF81E0903109F080E080938B0ABB
:1015E000903141F08985873409F004CF8A858E37A0
:1015F00009F400CF8091070D813029F08230D9F1B4
:101600008111F8CE0AC08091080D9091090D0196C4
:101610009093090D8093080DEDCEBE016F5F7F4F53
:101620008DE89AE00E94ECBC0115110529F48DE8C3
:10163000C82E8AE0D82E09C06801F60181916F0199
:101640008823A9F30E948551F8CFF60181916F019B
:10165000882319F00E948551F8CF80E20E948551BD
:101660006D8D7E8D8F8D98A14AE00E94A7548AE0EF
:101670000E948551BFCEBE016F5F7F4F8DE89AE01B
:101680000E94ECBC8114910441F06DE87AE0C40141
:101690000E9413DD892B69F414C0AD96FFADAD97A0
:1016A0008F2F90E02091141030911510821793071E
:1016B00041F0AD962FADAD972F5FAD962FAFAD97A3
:1016C00099CEE1968EAD9FADE1970FB6F8949EBF8F
:1016D0000FBE8DBFCE58DF4F0FB6F894DEBF0FBEE2
:1016E000CDBFDF91CF911F910F91FF90EF90DF90D1
:1016F000CF90BF90AF909F908F907F906F905F90B2
:101700004F903F902F9008950F931F93CF93DF93A7
:10171000CDB7DEB76F970FB6F894DEBF0FBECDBF63
:101720008B0122E02093070D9093151080931410E5
:1017300089ED9AE00E941CA48BE1E9EDFAE0DE015C
:10174000159601900D928A95E1F78091D70A9091B4
:10175000D80A9C838B8385EE92E09A838983A801C3
:10176000BE016F5F7F4F80E090E008DECE01019602
:101770000E94F3576F960FB6F894DEBF0FBECDBF31
:10178000DF91CF911F910F9108952F923F924F9229
:101790005F926F927F928F929F92AF92BF92CF9201
:1017A000DF92EF92FF920F931F93CF93DF93CDB70A
:1017B000DEB76F970FB6F894DEBF0FBECDBF6C01DA
:1017C0002DB63EB61D8218861C821B8285EE92E0E5
:1017D0009A838983FB0180819E012F5F3F4F3901EE
:1017E0008F3241F085ED9AE0F60191838083F62EE9
:1017F000172F64C086EB9AE0F601918380838B01FA
:101800000F5F1F4F0115110509F456C04DB65EB6A6
:101810006FE270E0C8010E9431DD4C010817190722
:1018200008F048C07C01E01AF10AFF24C7010196C4
:101830002DB73EB7281B390B0FB6F8943EBF0FBE2D
:101840002DBF8DB79EB701965C01A701B8010E941C
:101850005ADDF501EE0DFF1D1082F60160817181E8
:101860006115710511F06C5F7F4F21E0A501CE017C
:1018700005960E9452A8811111C0B50181EF9AE12D
:101880000E9461B78EE20E9485518AE00E948551D4
:101890000FB6F8945EBE0FBE4DBE0EC0F60171824B
:1018A000608284010F5F1F4F0FB6F8945EBE0FBEBB
:1018B0004DBEA8CFF02E02C0F12C10E0C3010E9453
:1018C000F3578F2D912F0FB6F8943EBE0FBE2DBE4D
:1018D0006F960FB6F894DEBF0FBECDBFDF91CF91EC
:1018E0001F910F91FF90EF90DF90CF90BF90AF903E
:1018F0009F908F907F906F905F904F903F902F9030
:101900000895FF920F931F93CF93DF938C01EB0108
:10191000F42E80E20E9485518FEFF81611F084E5D5
:1019200001C082E40E9485518AE30E948551F8013A
:10193000608171818281938142E00E946855488173
:1019400059816A817B818DE19EE10E942BB762E023
:1019500070E080E090E0DF91CF911F910F91FF90B8
:101960000C94D8C48F929F92AF92BF92CF92DF9285
:10197000EF92FF920F931F93CF93DF93F0E2FF2E2E
:10198000E12CAE2DB0E0BD016F0D711D7595679511
:101990006E1511F0F6120BC0E0E0FCE16591749158
:1019A000072E000C880B990B0E94A1D562C09B01E9
:1019B00021503109220F331F220F331FF901EE5737
:1019C000F44E05911491AB01440F551F440F551F60
:1019D000FA01EE57F44EC591D4918017910714F493
:1019E000F62ED1CFC817D90714F4E62ECACFF901C5
:1019F000EC57F44EE590F490FA01EC57F44EC59094
:101A0000D490BC01601B710B072E000C880B990B46
:101A10000E94A1D54B015C01B6016E197F09072E0A
:101A2000000C880B990B0E94A1D59B01AC01C5014C
:101A3000B4010E9400D64B015C01C01BD10BBE015A
:101A4000DD0F880B990B0E94A1D59B01AC01C5014C
:101A5000B4010E94A1DA4B015C01B701FF0C880BB5
:101A6000990B0E94A1D59B01AC01C501B4010E9454
:101A7000C5D9DF91CF911F910F91FF90EF90DF902B
:101A8000CF90BF90AF909F908F9008950F931F932A
:101A9000CF93DF93CDB7DEB728970FB6F894DEBFAC
:101AA0000FBECDBF6091410470914204072E000C1F
:101AB000880B990B0E94A1D56D837E838F839887B5
:101AC0008091430490914404A0914504B091460450
:101AD00089839A83AB83BC834DEFBE016B5F7F4FDD
:101AE000CE0101960EDF60913B0470913C04072EFD
:101AF000000C880B990B0E94A1D56D837E838F8388
:101B0000988780913D0490913E04A0913F04B0914C
:101B1000400489839A83AB83BC834FEFBE016B5F24
:101B20007F4FCE010196EDDEE5E2FEE184918F016B
:101B30000F5F1F4F882321F00E948551F801F6CFD7
:101B4000E0915C10F0E0E65AFF4E608170E080E0CA
:101B500090E00E944E55E0E2FEE184918F010F5F1C
:101B60001F4F882321F00E948551F801F6CF609124
:101B70005B1070E080E090E00E944E5528960FB612
:101B8000F894DEBF0FBECDBFDF91CF911F910F91B3
:101B900008950F930FB70F9300916E000B7F009382
:101BA0006E0078940F930BB70F930CB70F921F92A0
:101BB0002F933F934F935F936F937F938F939F9355
:101BC000AF93BF93EF93FF931124DAD2FF91EF917C
:101BD000BF91AF919F918F917F916F915F914F9145
:101BE0003F912F911F900F900CBF0F910BBF0F9142
:101BF0000460F89400936E000F910FBF0F91189539
:101C0000CF92DF92EF92FF92C0903D04D0903E04BD
